:100000000C947E060C949D060C949D060C949D0603
:100010000C949D060C949D060C9417090C9456099B
:100020000C949D060C949D060C949D060C949D06C4
:100030000C949D060C949D060C949D060C94CC0C7F
:100040000C949D060C949D060C949D060C949D06A4
:100050000C94F4400C9416380C949D060C949D0658
:100060000C949D060C94EB380C949D060C94DF3890
:100070000C949D060C949D060C949D060C949D0674
:100080000C94A04D0C949D060C949D060C949D061A
:100090000C9429390C949D060C941D390C949D06E2
:1000A0000C949D060C949D060C949D060C949D0644
:1000B0000C949D060C949D060C949D060C949D0634
:1000C0000C949D060C949D060C949D060C949D0624
:1000D0000C949D060C949D060C949D060C949D0614
:1000E0000C949D060C94AD400C94B7400C94A34026
:1000F0000C945D400C94E8400C94D9400C94CD4095
:100100000C94C1400C949D060C949D060C949D0685
:100110000C949D060C949D060C949D060C949D06D3
:100120000A0025303278002025362E3266204F6EA8
:100130002D426F61726400202573002530327800F3
:100140002025362E3266200020257300756E6B6EDA
:100150006F776E20636D640A00256300682020209D
:10016000202020202020202020202020202020208F
:1001700020202020202020202D2068656C700A0D72
:100180000076202020202020202020202020202039
:10019000202020202020202020202020202D2076FC
:1001A000657273696F6E0A0D007520202020202073
:1001B000202020202020202020202020202020203F
:1001C00020202020202D20757074696D650A0D0097
:1001D000616573205B6F6E7C6F66665D20202020FA
:1001E0002020202020202020202020202D20696E6B
:1001F000746567726574790A0D006164632020205C
:1002000020202020202020202020202020202020EE
:100210002020202020202D2073686F7720765F69B2
:100220006E2C2061312C20613220766F6C746167F6
:1002300065730A0D0063616C69205B5B765F696EB4
:100240007C61317C61325D20766F6C746167655DC5
:10025000202D2063616C6962726174650A0D00640F
:1002600065205B6D61736B5D2020202020202020A5
:1002700020202020202020202020202D20646562A6
:1002800075670A0D0068756D202020202020202031
:10029000202020202020202020202020202020205E
:1002A000202D2068756D69646974792073656E739B
:1002B0006F720A0D0068756D70205B6F6E7C6F66E3
:1002C000665D2020202020202020202020202020AB
:1002D000202D2068756D6964697479207065726D70
:1002E0002073656E736F72207077720A0D006964F7
:1002F000205B72657365745D202020202020202003
:10030000202020202020202020202D20696420680B
:10031000616E646C696E670A0D006D637520202044
:1003200020202020202020202020202020202020CD
:100330002020202020202D206D637520696E666F9F
:100340000A0D006E65205B666C7573685D20202069
:100350002020202020202020202020202020202D90
:10036000206E65696768626F72207461626C650AED
:100370000D006C6F67205B6175746F7C6F6E7C6FB6
:1003800066665D20202020202020202020202D2097
:100390006D6F7465732064617461206F6E205553B6
:1003A000420A0D006F7720202020202020202020CE
:1003B000202020202020202020202020202020203D
:1003C0002D206F6E652D776972652073656E736F72
:1003D00072730A0D007265205B6D61736B5D202086
:1003E000202020202020202020202020202020200D
:1003F000202D206D6F7465207265706F727420738C
:10040000657474696E670A0D007269205B696E74A9
:100410005D2020202020202020202020202020209F
:1004200020202020202D207265706F727420696E4C
:1004300074657276616C0A0D007273202020202092
:1004400020202020202020202020202020202020AC
:1004500020202020202D20726164696F2073746138
:1004600074730A0D00737320202020202020202088
:10047000202020202020202020202020202020207C
:10048000202D207374617475732073756D6D6172A6
:10049000790A0D0070777231205B6F6E7C6F666633
:1004A0005D2020202020202020202020202020200F
:1004B0002D2070696E31207077720A0D007265739D
:1004C0007420656570726F6D202020202020202010
:1004D0002020202020202020202D20726573746F82
:1004E000726520656570726F6D0A0D00626F6F74C2
:1004F00020202020202020202020202020202020FC
:1005000020202020202020202D207265626F6F7413
:100510000A0D0075706772202020202020202020E6
:100520002020202020202020202020202020202DBE
:10053000207265626F6F742076696120626F6F74DC
:100540006C6F616465720A0D00557074696D652089
:10055000256420646179732C20253032643A25307B
:1005600032643A253032640A00204E657665722D79
:100570007573656420737461636B203E202564206D
:1005800062797465730A0025352E3266200025379E
:100590002E33662025372E3366002530327800252D
:1005A000730A004E65772064656275673D30782573
:1005B000580A0043757272656E74206465627567CF
:1005C0003D307825580A00445F4F5045523D307801
:1005D00025780A00445F52583D307825780A004457
:1005E0005F54583D307825780A00445F504B543DA5
:1005F0006E307825780A00445F4F573D3078257873
:100600000A00445F4C45443D307825780A00445F39
:10061000504F5745523D307825780A00445F455683
:10062000454E543D307825780A00445F50305F4C89
:1006300045443D307825780A00445F50315F4C4591
:10064000443D307825780A00445F4145533D307879
:1006500025780A00445F5057525F313D3078257845
:100660000A002563002563002563004F4B0A00251F
:1006700063007478206C656E202020202072682032
:100680006D697373202020207268207374616C651B
:100690002020207268206D6973630A00252D313097
:1006A0006C7520252D31306C7520252D31306C7501
:1006B00020252D31306C75200A002563004D4355EF
:1006C0003D2530366C780020467573653A206565A7
:1006D0003D253032782068663D25303278206C66C2
:1006E0003D25303278206C623D2530327800204F35
:1006F000534343414C3D256420002563002563009E
:100700002563002563004E6577207265706F7274F3
:100710003D307825580A005573696E672072657000
:100720006F72743D307825580A00525F49443D0984
:1007300009307825780A00525F543D090930782540
:10074000780A00525F545F4D43553D093078257853
:100750000A00525F565F4D43553D09307825780AAF
:1007600000525F50303D0909307825780A00525F09
:1007700050305F543D0909307825780A00525F50A7
:10078000313D0909307825780A00525F55505449A7
:100790004D453D09307825780A00525F52483D09A1
:1007A00009307825780A00525F565F494E3D0909A5
:1007B000307825780A00525F41313D0909307825AB
:1007C000780A00525F41323D0909307825780A00E5
:1007D000525F54313D0909307825780A00256300BD
:1007E0004E6577207265706F727420696E746572E1
:1007F00076616C3D252D64207365630A0043757234
:1008000072656E74207265706F727420696E7465A3
:100810007276616C3D252D64207365630A00256343
:10082000002563005374617475732053756D6D6199
:1008300072790A49443D004E65696768626F7220AB
:100840007461626C652073697A653D25640A0052A3
:10085000494D4520616464723D252D642E252D642B
:100860000A00526164696F205265706F727420498A
:100870006E74657276616C3D252D640A0052616468
:10088000696F205265706F7274204D61736B3D30DB
:1008900078252D780A00565F494E3D252D352E329C
:1008A000660A00565F4D43553D252D352E32660AAA
:1008B000005553425F5057523D25730A00546F74E0
:1008C000616C20696E74723A2050303D252D6C6445
:1008D0002050313D252D6C640A004C6F67206D6FF0
:1008E000646520697320006175746F0A0025730ABE
:1008F0000048554D5F5057525F414C574159533D49
:1009000025730A0044656275673D3078252D780AA5
:1009100000507772312069732025730A0025630027
:1009200025630052483D252D342E31662000545F4A
:1009300052483D252D342E31662000256300585441
:10094000414C5F5452494D3D2564004572726F72AF
:10095000203020566F6C74004572726F7220302008
:10096000566F6C74004572726F72203020566F6C37
:10097000740025352E3266200025372E336620255B
:10098000372E33660025730A0025730A0025730A83
:100990000025730A00256300256300532025642E7B
:1009A000256420636C6F636B20256C752074782040
:1009B000256C7520727820256C752072747820253E
:1009C0006C752072727820256C75207265786D695F
:1009D0007420256C752061636B747820256C7520FC
:1009E0006E6F61636B747820256C752061636B7228
:1009F0007820256C752074696D65646F7574202589
:100A00006C752062616461636B727820256C75205F
:100A1000746F6F6C6F6E6720256C7520746F6F73C9
:100A2000686F727420256C752062616473796E63DF
:100A30006820256C752062616463726320256C7583
:100A400020636F6E74656E74696F6E64726F702070
:100A5000256C752073656E64696E6764726F7020B3
:100A6000256C75206C6C747820256C75206C6C720C
:100A70007820256C750A00452025642E25642063A6
:100A80006C6F636B20256C752063707520256C7509
:100A9000206C706D20256C752069727120256C7535
:100AA00020676C656420256C7520796C6564202551
:100AB0006C7520726C656420256C75207478202517
:100AC0006C75206C697374656E20256C7520736578
:100AD0006E736F727320256C752073657269616C1B
:100AE00020256C750A000A2A2A2A2A2A2A2A426FF5
:100AF0006F74696E672025732A2A2A2A2A2A2A0AED
:100B00000052616E646F6D20455549363420616432
:100B100064726573732067656E6572617465640ADB
:100B2000004D414320616464726573732000257831
:100B30003A000A0025732025732C206368616E6ECD
:100B4000656C20257520706F776572202575002CE7
:100B500020636865636B2072617465202575204889
:100B60007A000A004F6E6C696E650A002573257362
:100B70000A006C6F63616C686F73740041544D457B
:100B800047413132387266613100020000FFFE00D9
:100B90000001454550524F4D20697320636F7272BA
:100BA0007570742C20726577726974696E6720772E
:100BB0006974682064656661756C74732E0A006ED2
:100BC000616E00696E660000407A10F35A00A072F0
:100BD0004E18090010A5D4E80000E8764817000078
:100BE000E40B54020000CA9A3B000000E1F5050046
:100BF0000080969800000040420F000000A086018F
:100C0000000000102700000000E80300000000645E
:100C100000000000000A00000000000100000000C9
:100C2000002C76D888DC674F0823DFC1DFAE59E19E
:100C3000B1B796E5E3E453C63AE651997696E8E60D
:100C4000C28426EB898C9B62ED407C6FFCEFBC9CE0
:100C50009F40F2BAA56FA5F490055A2AF75C936BF2
:100C60006CF9676DC11BFCE0E40D47FEF520E6B5AD
:100C700000D0ED902E0300943577050080841E0887
:100C80000000204E0A000000C80C333333330F98A5
:100C90006E12831141EF8D2114893BE65516CFFE6C
:100CA000E6DB18D1844B381BF77C1D901DA4BBE4F8
:100CB00024203284725E228100C9F124ECA1E53D3A
:100CC00027494E46494E4954594E414E0000204155
:100CD0000000C84200401C4620BCBE4CCA1B0E5A35
:100CE000AEC59D74CDCCCC3D0AD7233C17B7D138C7
:100CF00077CC2B329595E6241FB14F0A11241FBEE5
:100D0000CFEFD1E4DEBFCDBF16E0A0E0B2E0E4E675
:100D1000FFEC00E00BBF02C007900D92A430B107BA
:100D2000D9F718E2A4E0B6E001C01D92A23BB107DA
:100D3000E1F70E94C85A0C94B0670C940000E0914F
:100D4000CE12F0E0EF71F070E55EFC4E8083809192
:100D5000CE128F5F8093CE128091EC1F88608093BB
:100D6000EC1F42E454E0CA0161E10E94EB2A80E0FA
:100D700090E008956F927F928F929F92AF92BF9270
:100D8000CF92DF92EF92FF920F931F93CF93DF9357
:100D90004B0180910E0690910F0681FD74980E9480
:100DA00043305C0188E196E00E94E72B0AC0CE0147
:100DB0000296B4010E94C2280097E9F4CE010E9475
:100DC0008D2CEC01009799F7CCC0CE010296B401AE
:100DD0000E94B928D5018C918150888780E091E0EC
:100DE000A0E0B0E089879A87AB87BC8788E196E06E
:100DF000BE010E94562C84E00E9467319D838C8343
:100E000083E00E9467313C019F838E83F501C0809F
:100E10008885C81ADD24EE24FF24A6E0CC0CDD1C56
:100E2000EE1CFF1CAA95D1F769857A858B859C8578
:100E300020EC30E040E050E00E94B060DC01CB01EB
:100E4000892F9A2FAB2FBB27C80ED91EEA1EFB1E77
:100E5000C986DA86EB86FC86D5018C9188878091DD
:100E60000E0690910F0681FD08C08091780480FDE8
:100E700004C081FF6EC01D9B6CC0EDB7FEB77297BA
:100E80000FB6F894FEBF0FBEEDBF0DB71EB70F5FD4
:100E90001F4F80E092E092838183C5010196D801C3
:100EA00013969C938E931297F401808114968C93E1
:100EB000149715961C921597818116968C93169708
:100EC00017961C92D5018C91F801808711868C8130
:100ED0009D819387828775866486BB27AF2D9E2D63
:100EE0008D2D97878687C701B60124E630E040E064
:100EF00050E00E94B060672F782F892F99270E94B9
:100F0000F660DC01CB01F801918B808B0E94866436
:100F1000209194048DB79EB742960FB6F8949EBF69
:100F20000FBE8DBF2223A9F000D000D0EDB7FEB7D1
:100F3000319688E999E0ADB7BEB712969C938E932F
:100F40001197228313820E9498640F900F900F9044
:100F50000F9080910E0690910F0681FF0BC0749A3E
:100F600009C089EA94E00E94742BEC01009709F013
:100F70002CCFEFCFDF91CF911F910F91FF90EF908A
:100F8000DF90CF90BF90AF909F908F907F906F90A9
:100F9000089587EE93E08115910511F00197F1F71F
:100FA00008950F931F93CF93DF93C0EADFE10CE323
:100FB00012E088819981009739F12DB73EB728500A
:100FC00030400FB6F8943EBF0FBE2DBFEDB7FEB751
:100FD0003196ADB7BEB712961C930E9311974A8106
:100FE0005B816C817D8142835383648375839783A6
:100FF00086830E9486642DB73EB7285F3F4F0FB6A9
:10100000F8943EBF0FBE2DBF26963FE1CC3DD307DF
:1010100081F6DF91CF911F910F910895E0EAFFE1F2
:101020001182108236968FE1EC3DF807C9F70895DA
:10103000CF93DF93C0EADFE1E881F981309761F176
:1010400040910406509105066091060670910706CE
:101050008091120690911306A0911406B091150686
:10106000841B950BA60BB70B4A815B816C817D813C
:10107000840F951FA61FB71F8A839B83AC83BD83F4
:10108000181619061A061B063CF0099519821882D3
:101090001A821B821C821D8226968FE1CC3DD807C6
:1010A00059F68091040690910506A0910606B0912C
:1010B00007068093120690931306A0931406B0932C
:1010C0001506DF91CF910895CF93DF93EC018881CE
:1010D0009981009729F027E080379207A9F40BC087
:1010E00080E296E060E870E00E947F2D80E797E064
:1010F000998388830DC080E296E00E94AA2D009714
:1011000039F00E941808ECCF1982188283E001C0E0
:1011100081E0DF91CF910895DC01E0EAFFE180E01A
:1011200090E0208131812115310591F4FC01EE0F11
:10113000FF1FE80FF91FEE0FFF1FE056F04E42832E
:10114000538364837583B183A08381E090E0089525
:10115000019636968A30910521F780E090E0089557
:1011600080EB98E040EA50E060E070E00E948C087C
:1011700080EB98E040EA50E060E070E00E948C086C
:101180000097B9F180910E0690910F0687FF31C04C
:10119000409104065091050660910606709107067D
:1011A0008DB79EB70A970FB6F8949EBF0FBE8DBF3E
:1011B000EDB7FEB731968EE592E0ADB7BEB71296A9
:1011C0009C938E931197428353836483758380EA43
:1011D00090E0A0E0B0E086839783A087B1870E946B
:1011E00086648DB79EB70A960FB6F8949EBF0FBE61
:1011F0008DBF0895882369F06D987598ED9A809158
:101200006A00886080936A008091680081608093A2
:1012100068006E987698EE9A80916A00806280935A
:101220006A008091680081608093680008951F9231
:101230000F920FB60F9211248F939F93AF93BF938A
:101240008091680080FF29C080919C1F90919D1F14
:10125000019690939D1F80939C1F8091941B909169
:10126000951BA091961BB091971B0196A11DB11DD6
:101270008093941B9093951BA093961BB093971B00
:1012800080910E0690910F0690FF07C0749882E03F
:1012900090E09093A2048093A104BF91AF919F919D
:1012A0008F910F900FBE0F901F9018951F920F9265
:1012B0000FB60F9211248F939F93AF93BF9380919A
:1012C000680080FF29C080919E1F90919F1F01960A
:1012D00090939F1F80939E1F8091981B9091991BC4
:1012E000A0919A1BB0919B1B0196A11DB11D8093EB
:1012F000981B9093991BA0939A1BB0939B1B809172
:101300000E0690910F0691FF07C0739882E090E05F
:101310009093A2048093A104BF91AF919F918F916C
:101320000F900FBE0F901F90189580937C008091B6
:101330007B00877F80937B0080917C00806C809312
:101340007C0085E080937A0080917A0080688093A9
:101350007A0080917B0087FFFCCF80917B0085FF26
:10136000FCCF80917A00806480937A0080917A002B
:1013700086FDFCCF109279001092780084E090E016
:1013800060E070E020917A00206420937A00209140
:101390007A0026FDFCCF2091780030917900620F11
:1013A000731F019779F710927C0080917A008F77F4
:1013B00080937A00769567957695679580E090E0C2
:1013C0000E949B5F462F572F682F792FCB01BA01C0
:1013D000089580E00E94950920919D0430919E041B
:1013E00040919F045091A0040E944D6021EE3AE785
:1013F00044E95EE30E94CB5E462F572F682F792F7A
:10140000CB01BA01089580E180935101809351018D
:101410009091510195FF03C08F5F8F31B9F76BE455
:10142000869FB0011124882777FD8095982F0E9410
:101430009D5F20E030E64FE954E40E94CB5E462FEA
:10144000572F682F792FCB01BA0120E030E04AE70F
:1014500054E40E94335F462F572F682F792FCB011A
:10146000BA01089580917C0482FF4DC080917B0079
:10147000886080937B0089EC80937C0085E080937A
:101480007A0080917A00806880937A0080917B0056
:1014900087FFFCCF80917B0085FFFCCF80917A0095
:1014A000806480937A0080917A0086FDFCCF8091E1
:1014B0007A00806480937A0080917A0086FDFCCF68
:1014C000609178007091790080E090E00E949B5FCD
:1014D00027ED33EA40E95FE30E944D6026E636E6F9
:1014E00048E853E40E94CA5EDC01CB018093C2123B
:1014F0009093C312A093C412B093C51280917A0046
:101500008F7780937A000895CF92DF92EF92FF92C7
:101510001F93CF93DF93CDB7DEB729970FB6F8941B
:10152000DEBF0FBECDBF6C01109208068FEF89831E
:1015300057EDE52E52E1F52E10E03FC0183009F4CA
:1015400040C0CE010196BE016E5F7F4F0E942A33DC
:1015500089818F3F11F08E3F19F48093080631C0C6
:10156000CE010296C114D10479F40E9443338093D2
:10157000E91FDE011296E1EEFFE188E09D91919373
:101580008150E1F711E01DC00E944333F7018083D1
:10159000DE01129620E030E0C70108974D91FC0172
:1015A000E20FF31F40832F5F3F4F28303105B1F723
:1015B0001F5F89E090E0E80EF91E8981882309F019
:1015C000BDCF812F29960FB6F894DEBF0FBECDBFD9
:1015D000DF91CF911F91FF90EF90DF90CF90089512
:1015E00000D080E291E0EDB7FEB7928381830E9444
:1015F00098640F900F9008952F923F924F925F92B0
:101600006F927F928F929F92AF92BF92CF92DF9212
:10161000EF92FF920F931F93CF93DF9300D000D0F0
:10162000CDB7DEB78C01009741F489E290E06BE220
:1016300070E04AE250E027E00AC08130910549F4A9
:1016400089E290E06BE270E04AE250E026E00E941E
:10165000FF31C8010E94840A39E0832E36E0932EC0
:10166000800E911ED4018C930115110599F017ED90
:10167000A12E12E1B12E00E010E08BE3682E81E094
:10168000782E90E4492E91E0592E28E4222E21E074
:10169000322E10C181EE9FE10E946634FC01BF0131
:1016A000882777FD8095982F0E949D5FF82EE92E60
:1016B00001EE1FE1AA24BB24B2E2CB2EB1E0DB2E67
:1016C000D8018D918D0100D000D0EDB7FEB73196D5
:1016D000ADB7BEB71296DC92CE9211978283138279
:1016E0006B837C830E9498640894A11CB11C0F90AA
:1016F0000F900F900F906B817C81B8E0AB16B10416
:10170000F9F600D000D000D00DB71EB70F5F1F4F05
:1017100087E291E0EDB7FEB7928381839701862F30
:10172000972FA32FBE2DBC01CD0120E030E048EC67
:1017300052E40E94335FDC01CB01F8018283938382
:10174000A483B5830E9498642DB73EB72A5F3F4FAC
:101750000FB6F8943EBF0FBE2DBF8091E91F8823BE
:1017600019F081E892E002C08AE892E000D000D04F
:1017700027E331E0ADB7BEB712963C932E93119795
:1017800014969C938E9313970E9498640F900F90D9
:101790000F900F900E94F00A94C0C80163E0880F78
:1017A000991F6A95E1F7800F911F81539D4E0E940A
:1017B0006634FC01BF01882777FD8095982F0E9431
:1017C0009D5F6C0120E030E0A8EFEA2EAFEFFA2E2B
:1017D000EA0CFB1C00D000D0ADB7BEB71196EDB738
:1017E000FEB772826182F701E20FF31F80811296C9
:1017F0008C93129713961C9229833A836B837C8374
:101800000E94986429813A812F5F3F4F0F900F907B
:101810000F900F906B817C8128303105D9F600D074
:1018200000D000D0EDB6FEB60894E11CF11CADB7B7
:10183000BEB712965C924E921197862F972FAC2DC1
:10184000BD2DBC01CD0120E030E048EC52E40E9407
:10185000335FDC01CB01F70182839383A483B583DB
:101860000E9498642DB73EB72A5F3F4F0FB6F89499
:101870003EBF0FBE2DBFD5018C91882319F081E8A2
:1018800092E002C08AE892E000D000D0EDB7FEB747
:1018900032822182948383830E9498640F900F90F8
:1018A0000F900F900E94F00A0F5F1F4F29E030E069
:1018B000A20EB31ED4018C9190E0081719070CF406
:1018C0006CCF0F900F900F900F90DF91CF911F91E1
:1018D0000F91FF90EF90DF90CF90BF90AF909F90CF
:1018E0008F907F906F905F904F903F902F900895D2
:1018F000CF93DF9300D0CDB7DEB78091E21F89830D
:101900008091E81F8A83CE0101960E94D4280F900F
:101910000F90DF91CF910895CF93DF93EC018091E9
:10192000E11F8F3FB1F58091E21F8F3F91F58091CC
:10193000E31F8F3F71F58091E41F8F3F51F5809138
:10194000E51F8F3F31F58091E61F8F3F11F58091A4
:10195000E71F8F3FF1F48091E81F8F3FD1F489E2B8
:1019600090E06BE270E04AE250E027E00E94FF3135
:1019700080E090E00E94840AC75FD94F888381EE9F
:101980009FE160E070E049E050E00E94DE650E9467
:10199000780CDF91CF9108951F920F920FB60F929E
:1019A0000BB60F9211242F933F934F935F936F9336
:1019B0007F938F939F93AF93BF93EF93FF93809108
:1019C000EC1F82608093EC1F8091A1049091A2048F
:1019D0001816190614F4749A739A80910E06909151
:1019E0000F0685FF02C07498739880910406909149
:1019F0000506A0910606B09107060196A11DB11D2E
:101A00008093040690930506A0930606B0930706FC
:101A10008091A3049091A40401979093A4048093CF
:101A2000A304009709F064C08091160690911706F0
:101A30009C012F5F3F4F309317062093160640916D
:101A40003F1B5091401B6091411B7091421B4F5FA7
:101A50005F4F6F4F7F4F40933F1B5093401B6093EE
:101A6000411B7093421B20E130E03093A40420938B
:101A7000A3042091780420FD02C01D9B05C0109294
:101A80000C0610920B0606C021E030E030930C06E5
:101A900020930B0620917A0430917B0421153105A7
:101AA000A1F00296B9010E94CF60009771F4779877
:101AB00080910E0690910F0693FF07C0749884E002
:101AC00090E09093A2048093A1042115310581F048
:101AD0008091160690911706B9010E94CF60009779
:101AE00039F48AE294E062E140E050E00E94EB2A9F
:101AF000FF91EF91BF91AF919F918F917F916F91E6
:101B00005F914F913F912F910F900BBE0F900FBEA1
:101B10000F901F9018958091CE129091531B891BA6
:101B200008950E948B0D882379F0E091531BF0E01B
:101B3000EF71F070E55EFC4E808190E02091531BC8
:101B40002F5F2093531B08958FEF9FEF0895CF933E
:101B5000DF93EC0110921106109210068881998192
:101B6000009731F022E0873D920709F0B7C009C025
:101B70000E948B0D882341F487ED92E0998388833E
:101B8000B1C0613109F0AEC0F89478940E94910D13
:101B900090E090932906809328068D3009F47CC04C
:101BA0008F3F31F38231910569F18F37910521F033
:101BB0008830910509F053C080912A0690912B0638
:101BC000181619060CF060C06091AC287091AD2811
:101BD00088E090E00E945A646091AC287091AD2832
:101BE00080E290E00E945A646091AC287091AD2828
:101BF00088E090E00E945A6480912A0690912B061A
:101C000001973EC06091AC287091AD288DE090E0C6
:101C10000E945A6410922D0610922C0614C08C5A01
:101C2000944EFC0180816091AC287091AD2890E0C9
:101C30000E945A6480912C0690912D0601969093F3
:101C40002D0680932C0680912C0690912D062091D4
:101C50002A0630912B06821793070CF315C060916A
:101C6000AC287091AD280E945A6480912A06909108
:101C70002B0620912806FC01EC5AF44E2083019695
:101C800090932B0680932A0680912A0690912B062A
:101C90008F33910509F06CCF1092531B1092CE1226
:101CA00080912A0690912B06FC01EC5AF44E10828A
:101CB000909311068093100610922B0610922A061C
:101CC0008091EA1F9091EB1F009709F451CF60912A
:101CD0001E0640E050E00E94EB2A4ACF198218828B
:101CE00083E001C081E0DF91CF91089578948091E5
:101CF0000B0690910C06009719F483B7817F03C0FF
:101D000083B7817F866083BFF89483B7816083BF88
:101D10007894889583B78E7F83BF78940895CF9306
:101D2000DF93EC0188819981009721F027E08D37BE
:101D3000920789F40E94760E8091BC099091BD09AA
:101D400065E840E050E00E94EB2A8DE797E0998338
:101D5000888381E003C01982188283E0DF91CF91EC
:101D60000895FF920F931F93CF93DF93729A809100
:101D7000780483FD06C0C0E5D0E00E94C907219722
:101D8000E1F78EE40E94E434882309F08BC0C0E5BB
:101D9000D0E00E94C9072197E1F78FE40E94E43464
:101DA0000E944C35C82F8295869586958370813028
:101DB000A9F44091471B5091481B6091491B7091B9
:101DC0004A1B4F5F5F4F6F4F7F4F4093471B5093AE
:101DD000481B6093491B70934A1B16C08230A0F0C9
:101DE00040914B1B50914C1B60914D1B70914E1BB1
:101DF0004F5F5F4F6F4F7F4F40934B1B50934C1B78
:101E000060934D1B70934E1B0E944C351C2F1F730B
:101E100000E0080F111D0E944C35F82E0E94563527
:101E2000DF2D90E0C92FC80FD11DD695C795D69547
:101E3000C7950E9433358091780483FF7298B8016A
:101E400080E090E00E949B5F20E134E048EC5BE39F
:101E50000E944D60DC01CB0180933B1390933C13B7
:101E6000A0933D13B0933E13BE0180E090E00E942A
:101E70009B5F24EA3CEF44E25CE30E944D6020E07B
:101E800030E040E252E40E94CA5EDC01CB01809364
:101E9000ED1F9093EE1FA093EF1FB093F01F80E013
:101EA00090E015C08091431B9091441BA091451B6D
:101EB000B091461B0196A11DB11D8093431B9093C9
:101EC000441BA093451BB093461B81E090E0DF913B
:101ED000CF911F910F91FF9008950E94320A809137
:101EE0007C0490917D0490FF02C00E94B10E80910D
:101EF0007C0490917D0491FF0CC00E94E909DC01F3
:101F0000CB018093DC1F9093DD1FA093DE1FB09365
:101F1000DF1F08957298729A8EE40E94E43480EA7A
:101F20000E943B3580E00E943B3580E00E943B35BB
:101F30008FE40E94E4340E944C3582958695869504
:101F400083708130A9F44091471B5091481B6091E8
:101F5000491B70914A1B4F5F5F4F6F4F7F4F4093FC
:101F6000471B5093481B6093491B70934A1B16C034
:101F70008230A0F040914B1B50914C1B60914D1B47
:101F800070914E1B4F5F5F4F6F4F7F4F40934B1BC6
:101F900050934C1B60934D1B70934E1B00D000D090
:101FA000EDB7FEB731962BE832E0ADB7BEB712966B
:101FB0003C932E931197828313820E9486640F9024
:101FC0000F900F900F908EE40E94E43480E80E94FE
:101FD0003B3580E00E943B3580E00E943B350E940B
:101FE000333580E090E0089500D08CE491E0ADB707
:101FF000BEB712969C938E9311970E94986420917D
:1020000094040F900F902223A9F000D000D0EDB7D8
:10201000FEB7319689E591E0ADB7BEB712969C93B5
:102020008E931197228313820E9498640F900F90D1
:102030000F900F90089500D08CE591E0EDB7FEB7BA
:10204000928381830E94986481E891E0EDB7FEB7A6
:10205000928381830E94986489EA91E0EDB7FEB78C
:10206000928381830E94986480ED91E0EDB7FEB782
:10207000928381830E9498648AEF91E0EDB7FEB766
:10208000928381830E94986485E392E0EDB7FEB766
:10209000928381830E9498648FE592E0EDB7FEB74A
:1020A000928381830E94986485E892E0EDB7FEB741
:1020B000928381830E94986485EB92E0EDB7FEB72E
:1020C000928381830E9498648EEE92E0EDB7FEB712
:1020D000928381830E9498648AE193E0EDB7FEB712
:1020E000928381830E94986483E493E0EDB7FEB706
:1020F000928381830E94986482E793E0EDB7FEB7F4
:10210000928381830E94986484EA93E0EDB7FEB7DE
:10211000928381830E94986485ED93E0EDB7FEB7CA
:10212000928381830E94986489E094E0EDB7FEB7C2
:10213000928381830E94986489E394E0EDB7FEB7AF
:10214000928381830E94986485E694E0EDB7FEB7A0
:10215000928381830E94986484E994E0EDB7FEB78E
:10216000928381830E9498648DEB94E0EDB7FEB773
:10217000928381830E9498648CEE94E0EDB7FEB761
:10218000928381830E94986483E195E0EDB7FEB766
:10219000928381830E9498640F900F9008958BE939
:1021A00092E00E94BF6408954F925F926F927F9277
:1021B0008F929F92AF92BF92CF92DF92EF92FF9257
:1021C0000F931F93CF93DF9300D000D0CDB7DEB72E
:1021D00060913F1B7091401B8091411B9091421B6D
:1021E00080903F1B9090401BA090411BB090421BE1
:1021F00040903F1B5090401B6090411B7090421BD1
:1022000020913F1B3091401B4091411B5091421B3C
:1022100029833A834B835C834DB75EB74A50504065
:102220000FB6F8945EBF0FBE4DBF0DB71EB70F5F60
:102230001F4F29E435E0EDB7FEB732832183A0E8D4
:10224000CA2EA1E5DA2EA1E0EA2EF12CA701960113
:102250000E94F660F80133832283C501B401A7010F
:1022600096010E94F660B0E1CB2EBEE0DB2EE12CA1
:10227000F12CA70196010E94F660332727FD3095C7
:10228000F80135832483C301B201A70196010E949E
:10229000F6602CE3C22ED12CE12CF12CA701960183
:1022A0000E94F660332727FD3095F8013783268397
:1022B00069817A818B819C81A70196010E94F660D9
:1022C000772767FD7095F801718760870E94986491
:1022D0002DB73EB7265F3F4F0FB6F8943EBF0FBEF7
:1022E0002DBF0F900F900F900F90DF91CF911F9106
:1022F0000F91FF90EF90DF90CF90BF90AF909F90A5
:102300008F907F906F905F904F900895E2EBF8E28E
:102310008081918122E482349207B9F000D000D00C
:1023200089E695E0ADB7BEB712969C938E93119750
:10233000E25BF8421496FC93EE9313970E94986424
:102340000F900F900F900F9008953A96B1E4E53FEB
:10235000FB07F0F20895EF92FF920F931F93CF9334
:10236000DF930E94E909DC01CB0100D000D000D04E
:1023700027E835E0EDB7FEB732832183838394836A
:10238000A583B6830E9498648DB79EB706960FB654
:10239000F8949EBF0FBE8DBF81E00E9495092091E9
:1023A000990430919A0440919B0450919C040E949E
:1023B0004D608B01D82FC92F82E00E949509AB0197
:1023C000BC01EDB7FEB73A970FB6F894FEBF0FBE4B
:1023D000EDBFEDB6FEB60894E11CF11C2EE835E029
:1023E000328321839E01802F912FA32FB22FF701DB
:1023F00082839383A483B583CB01BA012091950492
:102400003091960440919704509198040E944D6039
:10241000DC01CB01F70186839783A087B1870E94F7
:1024200098648DB79EB70A960FB6F8949EBF0FBEFC
:102430008DBF0E94F00ADF91CF911F910F91FF9005
:10244000EF900895EF92FF920F931F93CF93DF9336
:10245000882389F081EE9FE16FEF70E049E050E062
:102460000E94106481EE9FE160E070E049E050E07E
:102470000E94DE6522C001EE1FE1C0E0D0E03AE933
:10248000E32E35E0F32ED8018D918D0100D000D0E0
:10249000EDB7FEB73196ADB7BEB71296FC92EE928D
:1024A0001197828313820E94986421960F900F9057
:1024B0000F900F90C830D10531F70E94F00ADF91DC
:1024C000CF911F910F91FF90EF900895CF92DF92DF
:1024D000EF92FF92609192047091930480E090E0FB
:1024E0000E9402646CEB72E00E941764009709F08E
:1024F00077C08FE892E090937D0480937C048CE712
:1025000094E06DE070E042E050E00E94DE658CE314
:1025100090E090937B0480937A048AE794E06BE0E8
:1025200070E042E050E00E94DE6582E090E090932F
:1025300079048093780488E794E069E070E042E0F1
:1025400050E00E94DE6510920F0610920E068EE09B
:1025500096E06BE170E042E050E00E94DE650F2EF5
:10256000F2E2CF2EFFEFDF2EFCECEF2EFBE3FF2E8F
:10257000F02DC0929904D0929A04E0929B04F092BC
:102580009C0489E994E063E170E044E050E00E943B
:10259000DE65C0929504D0929604E0929704F09282
:1025A000980485E994E06FE070E044E050E00E9418
:1025B000DE658DEE97E4AAE8BCE380939D049093DA
:1025C0009E04A0939F04B093A0048DE994E067E17A
:1025D00070E044E050E00E94DE6581E00E9422123B
:1025E000FF90EF90DF90CF9008952F923F924F92FF
:1025F0005F926F927F928F929F92AF92BF92CF9293
:10260000DF92EF92FF920F931F93CF93DF9300D04F
:10261000CDB7DEB79A838983DC018D919C911197A8
:10262000009711F00C9445216091920470919304ED
:1026300084E59BE10E94026484E59BE160E470E034
:102640000E942064009759F46091AC287091AD28E5
:102650008AE090E00E945A6481E00C944B21813022
:10266000910549F42090541B3324442455246624B6
:1026700077244301BEC18230910599F43091541BF7
:102680002091551B932F80E0820F911D1C01892FF3
:10269000880F880B482E582E682E782E882E982E5C
:1026A000A8C18330910509F09CC02091541B8090F3
:1026B000551BB090561B30E040E050E060E070E009
:1026C00080E090E000E10E940B5A922EA32E142F7E
:1026D000F52EE62EC72E282ED92E282D30E040E0EC
:1026E00050E060E070E080E090E008E00E940B5A6B
:1026F000290DB1E0291508F0B0E03A0DE1E03A15F6
:1027000008F0E0E0B30FF1E0B31708F0F0E0EF2BD2
:10271000410F31E0411708F030E0E40FF1E0E41739
:1027200008F0F0E03F2B5F0D41E05F1508F040E05E
:10273000A32FA50F31E0A51708F030E0432B6E0D55
:1027400031E06E1508F030E0F42FF60F41E0F61797
:1027500008F040E0342B7C0D41E07C1508F040E0AF
:10276000532F570F31E0571708F030E0432B820DFD
:1027700031E0821508F030E0480F61E0481708F0BA
:1027800060E0362BD90ED30EB20E81E0B21608F0FF
:1027900080E0182F1B0F71E01B1708F070E07E0F10
:1027A00061E07E1708F060E06A0F31E06A1708F018
:1027B00030E03F0F21E03F1708F020E0250F91E0C7
:1027C000251708F090E0940F81E0941708F080E05E
:1027D0002B2C312E472E562E632E722E892E982E9C
:1027E000FDC08430910509F0FBC02091541B8090FE
:1027F000551BA090561BB090571B30E040E050E0B6
:1028000060E070E080E090E008E10E940B5A722ED8
:10281000932E142FF52EE62EC72E282ED92E282DD6
:1028200030E040E050E060E070E080E090E000E107
:102830000E940B5A270DF1E0271508F0F0E0390D42
:10284000E1E0391508F0E0E0F30FA1E0F31708F03C
:10285000A0E0EA2B410F31E0411708F030E0E40F2F
:10286000A1E0E41708F0A0E03A2B5F0D41E05F150E
:1028700008F040E0B32FB50F31E0B51708F030E0B5
:10288000432B6E0D31E06E1508F030E0A42FA60F3B
:1028900041E0A61708F040E0342B7C0D41E07C15A8
:1028A00008F040E0532F570F31E0571708F030E0A1
:1028B000432B820D31E0821508F030E0480F61E0D3
:1028C000481708F060E0362BD90ED30E222E2B0CC1
:1028D00081E0221608F080E0B82EBF0E81E0BF161E
:1028E00008F080E0982E9E0E81E09E1608F080E0B1
:1028F000C82ECB0E11E0CB1608F010E01A0F81E0C5
:102900001A1708F080E0F82EF50E81E0F51608F0B1
:1029100080E0E82EE40E81E0E41608F080E0D80EB6
:102920002A2D30E040E050E060E070E080E090E090
:1029300008E00E940B5A220DE1E0221508F0E0E0C9
:102940003B0DF1E03B1508F0F0E0E30FA1E0E317E9
:1029500008F0A0E0FA2B490D31E0491508F030E00D
:10296000F40FA1E0F41708F0A0E03A2B5C0D41E071
:102970005C1508F040E0A32FA50F31E0A51708F083
:1029800030E0432B610F31E0611708F030E0542F45
:10299000560F41E0561708F040E0342B7F0D41E020
:1029A0007F1508F040E0632F670F31E0671708F0EC
:1029B00030E0432B8E0D31E08E1508F030E0480FEB
:1029C00071E0481708F070E0372BD90E222E3E2E0A
:1029D0004F2E5A2E652E762E842E932E9D0C09C0D6
:1029E0008AE0282E3324442455246624772488241E
:1029F00099240E94F00AB2E62B1689F4E5E63E1609
:102A000071F4F4E64F1659F4552049F4662039F470
:102A1000772029F4882019F4992009F40DC5910133
:102A2000A201B301C401B2E6AB2E15E6B12E04E655
:102A3000C02EDD24EE24FF2400E010E00E94855A21
:102A4000823008F099C187E7281681F49FE639168D
:102A500069F4442059F4552049F4662039F477206C
:102A600029F4882019F4992009F4D3C79101A2010F
:102A7000B301C401F7E7AF2EAFE6BA2ECC24DD24B4
:102A8000EE24FF2400E010E00E94855A823008F016
:102A9000B6C0A4E62A1689F4B1E63B1671F44420C8
:102AA00061F4552051F4662041F4772031F48820F8
:102AB00021F4992011F40C94AA209101A201B301F0
:102AC000C40104E6A02EE1E6BE2ECC24DD24EE24D3
:102AD000FF2400E010E00E94855A823008F046C0D2
:102AE000E5E72E1679F4332069F4442059F4552093
:102AF00049F4662039F4772029F4882019F49920C4
:102B000009F4BAC5F6E72F1679F4332069F44420A6
:102B100059F4552049F4662039F4772029F48820A7
:102B200019F4992009F4B7C588E6281611F00C9419
:102B30004321332011F00C944321442011F00C94D4
:102B40004321552011F00C944321662011F00C9480
:102B50004321772011F00C944321882011F00C942C
:102B60004321992011F00C94432163C594E6291662
:102B700081F4A9E63A1669F4442059F4552049F441
:102B8000662039F4772029F4882019F4992009F473
:102B900053C5B5E62B1681F4EEE63E1669F44420E3
:102BA00059F4552049F4662039F4772029F4882017
:102BB00019F4992009F487C7F5E62F1611F00C9443
:102BC000432184E6381611F00C944321442011F07F
:102BD0000C944321552011F00C944321662011F0F0
:102BE0000C944321772011F00C944321882011F09C
:102BF0000C944321992011F00C9443211DC493E7B8
:102C0000291689F4A2E73A1671F4442061F455209C
:102C100051F4662041F4772031F4882021F4992082
:102C200011F40C94361F9101A201B301C401B3E762
:102C3000AB2E12E7B12ECC24DD24EE24FF2400E0DD
:102C400010E00E94855A823008F04AC0B5E62B1683
:102C500079F43B1469F4442059F4552049F4662072
:102C600039F4772029F4882019F4992009F494C7BD
:102C7000E9E62E1689F4F2E73F1671F4442061F478
:102C8000552051F4662041F4772031F4882021F456
:102C9000992011F40C94DD1E83E3281611F00C9496
:102CA000432191E7391611F00C944321442011F08F
:102CB0000C944321552011F00C944321662011F00F
:102CC0000C944321772011F00C944321882011F0BB
:102CD0000C944321992011F00C9443210C94AA20C8
:102CE000A3E62A1691F4B4E63B1679F4E1E64E1613
:102CF00061F4552051F4662041F4772031F48820A6
:102D000021F4992011F40C94AA20F3E72F1689F4EA
:102D100085E6381671F491E6491659F4552049F4C0
:102D2000662039F4772029F4882019F4992009F4D1
:102D3000C1C4A3E72A1611F00C9443213A1611F0EE
:102D40000C944321442011F00C944321552011F0A0
:102D50000C944321662011F00C944321772011F04C
:102D60000C944321882011F00C944321992011F0F8
:102D70000C9443210C94451FB4E72B1689F4EFE61D
:102D80003E1671F44E1661F4F2E65F1649F46620C1
:102D900039F4772029F4882019F4992009F4C6C45D
:102DA0009101A201B301C40104E7A02EEFE6BE2EFB
:102DB000FFE6CF2EA2E6DA2EEE24FF2400E010E09C
:102DC0000E94855A823008F0A8C085E7281689F449
:102DD00093E6391671F4ADE64A1659F4552049F4D4
:102DE000662039F4772029F4882019F4992009F411
:102DF00091C59101A201B301C401A5E7AA2EB3E6D2
:102E0000BB2E1DE6C12EDD24EE24FF2400E010E0E1
:102E10000E94855A8230B0F52C1489F43A1479F462
:102E2000B8E64B1661F4552051F4662041F4772042
:102E300031F4882021F4992011F40C94B920E7E6AC
:102E40002E1689F4FFE63F1671F48CE6481659F405
:102E5000552049F4662039F4772029F4882019F4A4
:102E6000992009F497C492E7291611F00C94432194
:102E7000391611F00C944321A5E64A1611F00C9472
:102E8000432136C0B1E32B1681F43B1671F4E1E720
:102E90004E1659F4552049F4662039F4772029F468
:102EA000882019F4992009F435C5F0E72F1689F424
:102EB00085E6381671F492E7491659F4552049F41D
:102EC000662039F4772029F4882019F4992009F430
:102ED00063C6A0E32A1611F00C944321B1E33B161C
:102EE00011F00C944321E1E74E1611F00C944321AC
:102EF000552011F00C944321662011F00C944321CD
:102F0000772011F00C944321882011F00C94432178
:102F1000992011F00C9443219AC4F0E72F1691F4F4
:102F20008DE6381679F495E7491661F4A8E65A1645
:102F300049F4662039F4772029F4882019F499207F
:102F400009F48DC59101A201B301C40110E7A12EBE
:102F50000DE6B02EE5E7CE2EF8E6DF2EEE24FF24B8
:102F600000E010E00E94855A823008F04DC02A141B
:102F700089F4BCE63B1671F4E5E64E1659F45D148F
:102F800049F4662039F4772029F4882019F499202F
:102F900009F44FC3F1E62F1691F48DE6381679F453
:102FA00095E7491661F4A8E65A1649F4662039F403
:102FB000772029F4882019F4992009F43FC5B9E64F
:102FC0002B1611F00C944321ECE63E1611F00C94F4
:102FD0004321F1E64F1611F00C94432183E6581675
:102FE00011F00C944321662011F00C9443217720BA
:102FF00011F00C944321882011F00C944321992066
:1030000011F00C944321B0C094E7291691F4A3E782
:103010003A1679F4B5E64B1661F4E2E75E1649F428
:10302000662039F4772029F4882019F4992009F4CE
:10303000B0C59101A201B301C401E4E7AE2EF3E7EC
:10304000BF2EA5E6CA2EB2E7DB2EEE24FF2400E059
:1030500010E00E94855A823020F5F1E32F1611F01E
:103060000C9443213D1411F00C94432187E748163A
:1030700011F00C94432190E7591611F00C94432160
:10308000662011F00C944321772011F00C94432119
:10309000882011F00C944321992011F00C944321C5
:1030A0003BC0A2E72A1691F4B7E63B1679F4E0E7B5
:1030B0004E1661F4F5E75F1649F4662039F477207F
:1030C00029F4882019F4992009F433C38CE62816D2
:1030D00011F00C94432191E6391611F00C94432120
:1030E000A4E74A1611F00C944321B8E75B1611F0DF
:1030F0000C944321662011F00C944321772011F0A9
:103100000C944321882011F00C944321992011F054
:103110000C9443210C9409216091920470919304C2
:1031200080E090E00E9402648C0163EC72E00E94F7
:103130001764009719F477980C944521C80166EC40
:1031400072E00E941764009719F4779A0C94452155
:10315000779903C083EC92E002C086EC92E000D045
:1031600000D02FE935E0AAC46091920470919304D5
:1031700080E090E00E9402648C016DEC72E00E949D
:103180001764009709F043C0609192047091930412
:1031900080E090E00E9402648C01009711F40C948E
:1031A000452160ED72E00E941764009729F482E2E5
:1031B0009FEFACECBBE318C0C8010E94F5626B0145
:1031C0007C0120E030E040E050E00E942F5F882347
:1031D000D1F081E00E9495099B01AC01C701B601C5
:1031E0000E94335FDC01CB018093990490939A0491
:1031F000A0939B04B0939C0489E994E063E170E0A0
:1032000044E050E075C200D08BE499E09DC0C80155
:1032100066ED72E00E941764009709F045C0609166
:1032200092047091930480E090E00E9402648C010B
:10323000009711F40C94452160ED72E00E94176430
:10324000009729F482E29FEFACECBBE318C0C80101
:103250000E94F5626B017C0120E030E040E050E02C
:103260000E942F5F8823C1F082E00E9495099B0194
:10327000AC01C701B6010E94335FDC01CB01809332
:10328000950490939604A0939704B093980485E9CD
:1032900094E06FE070E0B4CF00D088E599E0EDB73E
:1032A000FEB79283818356C0C80169ED72E00E9427
:1032B0001764009709F053C06091920470919304D1
:1032C00080E090E00E9402648C01009711F40C945D
:1032D000452160ED72E00E941764009729F48DEE9D
:1032E00097E4AAE8BCE320C0C8010E94F5626B0124
:1032F0007C0120E030E040E050E00E942F5F882316
:1033000001F180E00E9495094B015C01C701B60103
:1033100021EE3AE744E95EE30E94CA5EA50194010A
:103320000E94335FDC01CB0180939D0490939E0447
:10333000A0939F04B093A0048DE994E067E170E04E
:103340005FCF00D085E699E0ADB7BEB712969C93EB
:103350008E9311970E9498640F900F9096C70E94C9
:10336000E909AB01BC0100D000D000D082E799E0B0
:10337000EDB7FEB79283818343835483658376835D
:103380000E949864EDB7FEB736960FB6F894FEBF6C
:103390000FBEEDBF81E00E94950920919904309104
:1033A0009A0440919B0450919C040E944D606B01D3
:1033B000182F092F82E00E949509AB01BC018DB73F
:1033C0009EB70A970FB6F8949EBF0FBE8DBFEDB69D
:1033D000FEB60894E11CF11C89E799E0ADB7BEB7D1
:1033E00012969C938E93119798018C2D9D2DA32F4F
:1033F000B22FF70182839383A483B583CB01BA01F3
:10340000209195043091960440919704509198042E
:103410000E944D60DC01CB01F70186839783A08772
:10342000B1870E9498648DB79EB70A960FB6F8943C
:103430009EBF0FBE8DBF24C760919204709193040C
:1034400080E090E00E940264009771F160E070E01B
:1034500040E150E00E94B461AB01BC0180910E06D6
:1034600090910F068417950799F150930F0640939A
:103470000E068EE096E06BE170E042E050E00E94C4
:10348000DE6580910E0690910F0600D000D023EAF1
:1034900035E0ADB7BEB712963C932E9311971496B4
:1034A0009C938E9313970EC080910E0690910F06F9
:1034B00000D000D023EB35E0EDB7FEB73283218397
:1034C000948383830E9498640F900F900F900F90C5
:1034D0000E94F00A00D000D087EC95E0ADB7BEB7EF
:1034E00012969C938E93119781E090E014969C9392
:1034F0008E9313970E94986484ED95E0EDB7FEB724
:103500009283818382E090E0948383830E94986415
:103510008FED95E0ADB7BEB712969C938E93119741
:1035200084E090E014969C938E9313970E94986485
:103530008AEE95E0EDB7FEB79283818388E090E054
:10354000948383830E94986487EF95E0ADB7BEB7FC
:1035500012969C938E93119780E190E014969C9321
:103560008E9313970E94986482E096E0EDB7FEB7C1
:103570009283818380E290E0948383830E949864A5
:103580008EE096E0ADB7BEB712969C938E931197DE
:1035900080E490E014969C938E9313970E94986415
:1035A0008CE196E0EDB7FEB79283818380E890E0EE
:1035B000948383830E9498648AE296E0ADB7BEB795
:1035C00012969C938E93119780E091E014969C93B1
:1035D0008E9313970E94986489E396E0EDB7FEB747
:1035E0009283818380E092E0948383830E94986435
:1035F00088E496E0ADB7BEB712969C938E93119770
:1036000080E094E014969C938E9313970E949864A4
:1036100084E596E0EDB7FEB79283818380E098E081
:10362000948383830E9498640F900F900F900F9063
:103630002CC60E941B1029C66091920470919304BD
:1036400080E090E00E94026460ED72E00E941764E6
:10365000009711F481E001C080E00E9422122091C5
:103660009404222309F411C600D000D0EDB7FEB7B0
:10367000319682E696E0C4C50E94D410209194044D
:10368000222309F402C600D000D0EDB7FEB7319670
:1036900085E696E0B5C50E94CF10209194042223C0
:1036A00009F4F3C500D000D0EDB7FEB7319688E637
:1036B00096E0A6C5609192047091930480E090E03A
:1036C0000E9402648C0163EC72E00E941764009710
:1036D00091F48091780490917904846090937904B6
:1036E0008093780488E794E069E070E042E050E07D
:1036F0000E94DE65CAC5C80166EC72E00E941764CC
:103700009C0180917804909179042115310511F480
:103710008B7FE4CF82FF03C083EC92E002C086EC93
:1037200092E000D000D025E839E0C8C10C94000038
:10373000ACC500D08BE696E0ADB7BEB712969C93B1
:103740008E9311970E949864209194040F900F908B
:103750002223A9F000D000D0EDB7FEB731968FE656
:1037600096E0ADB7BEB712969C938E9311972283C5
:1037700013820E9498640F900F900F900F9088E131
:103780000FB6F89480936000109260000FBE0C9406
:10379000007C7BC5609192047091930480E090E07E
:1037A0000E9402647C0163EC72E00E94176400973F
:1037B00049F40E94263B80917804909179048160BD
:1037C0008D7F8CCFC70166EC72E00E941764009772
:1037D00041F40E94173C80917804909179048C7F89
:1037E0007DCF0EED12E0C701B8010E94176400976B
:1037F00049F40E94173C80917804909179048E7F5F
:1038000082606CCF8091780481FF0BC000D000D023
:1038100089E899E0EDB7FEB792838183148303832F
:1038200001CF80FF03C083EC92E002C086EC92E0FF
:1038300000D000D02DE839E0ADB7BEB712963C936A
:103840002E93119714969C938E931397EBCE00D0E2
:1038500082E796E0EDB7FEB7928381830E94986479
:103860008DB79EB740970FB6F8949EBF0FBE8DBF21
:10387000EDB7FEB731968CE996E0ADB7BEB71296BC
:103880009C938E93119780914F1B9091501BA09108
:10389000511BB091521B82839383A483B583809183
:1038A000431B9091441BA091451BB091461B8683FE
:1038B0009783A087B1878091471B9091481BA09167
:1038C000491BB0914A1B82879387A487B587809153
:1038D0004B1B90914C1BA0914D1BB0914E1B8687AA
:1038E0009787A08BB18B0E94986420919404EDB7C8
:1038F000FEB772960FB6F894FEBF0FBEEDBF22233F
:1039000009F4C3C400D000D0EDB7FEB731968AEBFE
:1039100096E076C4F89409E081E090E0FC01009321
:103920005700C895F02C20E030E0F90100935700D3
:10393000C895E02C7894F89423E030E0F9010093E6
:103940005700C895102D82E090E0FC0100935700CD
:10395000C895002D789400D000D000D02DEB36E033
:10396000EDB7FEB73283218380911713909118131E
:10397000A0911913B0911A1383839483A583B683FE
:103980000E94986400D000D0EDB7FEB7319687EC66
:1039900096E0ADB7BEB712969C938E9311970283B3
:1039A000138214831582E6821782F08611860E94A4
:1039B0009864EDB7FEB73A960FB6F894FEBF0FBE07
:1039C000EDBF0E9486112091660000D000D0EDB7B7
:1039D000FEB731968EEE96E0ADB7BEB712969C93C9
:1039E0008E931197228313820E9498640F900F90F8
:1039F0000F900F900E94F00A20919404222309F462
:103A000044C400D000D0EDB7FEB731968AEF96E0FF
:103A1000F7C380E090E00E94FC0A81E090E00E9401
:103A2000FC0A20919404222309F42FC400D000D072
:103A3000EDB7FEB731968DEF96E0E2C30E948A0F94
:103A40000E94F00A20919404222309F41EC400D09D
:103A500000D0EDB7FEB7319680E097E0D1C360911A
:103A600092047091930480E090E00E9402648C01C3
:103A700063EC72E00E941764009731F4809178043F
:103A80009091790488602ACEC80166EC72E00E94A9
:103A900017649C0180917804909179042115310577
:103AA00011F4877F1BCE83FF03C083EC92E002C03A
:103AB00086EC92E000D000D021E939E0EDB7FEB706
:103AC00032832183ADCD609192047091930480E0A4
:103AD00090E00E94026463EE72E00E941764009717
:103AE00029F4109219061092180646C088E196E053
:103AF0000E94E72B7C0109EE12E03BC08DB79EB718
:103B00000C970FB6F8949EBF0FBE8DBFEDB7FEB7F2
:103B10003196ADB7BEB712961C930E931197D7018D
:103B200012968C9112978283138213968C9113971D
:103B30008483158218968C91189786831782149621
:103B40008D919C9115979187808716968D919C9168
:103B50001797938782870E948664EDB7FEB73C96DD
:103B60000FB6F894FEBF0FBEEDBFC7010E948D2CAB
:103B70007C01E114F10411F620919404222309F44C
:103B800084C300D000D0EDB7FEB7319683E097E054
:103B900037C30E94661279C36091920470919304B6
:103BA00080E090E00E940264009731F160E070E0F4
:103BB00040E150E00E94B461DC01CB0190937D04B0
:103BC00080937C0400D000D04DB75EB74F5F5F4F4D
:103BD00026E037E0EDB7FEB732832183FA01938305
:103BE00082830E9498640F900F900F900F908CE743
:103BF00094E06DE070E07ACD00D000D087E197E0EE
:103C0000ADB7BEB712969C938E93119780917C04AA
:103C100090917D0414969C938E9313970E949864C0
:103C20000F900F900F900F900E94F00A00D000D0DC
:103C30008AE297E0EDB7FEB79283818381E090E05E
:103C4000948383830E94986487E397E0ADB7BEB7FF
:103C500012969C938E93119782E090E014969C9319
:103C60008E9313970E94986483E497E0EDB7FEB7B4
:103C70009283818384E090E0948383830E9498649C
:103C800082E597E0ADB7BEB712969C938E931197DD
:103C900088E090E014969C938E9313970E9498640A
:103CA00081E697E0EDB7FEB79283818380E190E0F3
:103CB000948383830E9498648EE697E0ADB7BEB785
:103CC00012969C938E93119780E290E014969C93A9
:103CD0008E9313970E9498648DE797E0EDB7FEB737
:103CE0009283818380E490E0948383830E9498642C
:103CF0008AE897E0ADB7BEB712969C938E93119762
:103D000080E890E014969C938E9313970E94986499
:103D10008AE997E0EDB7FEB79283818380E091E076
:103D2000948383830E94986487EA97E0ADB7BEB717
:103D300012969C938E93119780E092E014969C9338
:103D40008E9313970E94986486EB97E0EDB7FEB7C9
:103D50009283818380E094E0948383830E949864BB
:103D600083EC97E0ADB7BEB712969C938E931197F4
:103D700080E098E014969C938E9313970E94986429
:103D800080ED97E0EDB7FEB79283818380E090E10C
:103D9000948383830E949864209194040F900F90E1
:103DA0000F900F90222309F470C200D000D0EDB71D
:103DB000FEB731968DED97E023C260919204709129
:103DC000930480E090E00E940264009751F160E06B
:103DD00070E04AE050E00E94B461DC01CB019093B6
:103DE0007B0480937A0400D000D04DB75EB74F5F5C
:103DF0005F4F20EE37E0EDB7FEB732832183FA0143
:103E0000938382830E9498640F900F900F900F907D
:103E10008AE794E06BE070E042E050E00E94DE65EB
:103E200018C000D000D08DEF97E0ADB7BEB71296A6
:103E30009C938E93119780917A0490917B041496B1
:103E40009C938E9313970E9498640F900F900F90FD
:103E50000F9020919404222309F417C200D000D0BF
:103E6000EDB7FEB731968EE198E0CAC10E94042EEC
:103E700020919404222309F408C200D000D0EDB7A9
:103E8000FEB7319681E298E0BBC100D084E298E0B1
:103E9000EDB7FEB7928381830E9498640F900F90D4
:103EA00080E00E9422120E94D41000D000D087E34C
:103EB00098E0ADB7BEB712969C938E93119780E4AD
:103EC00090E014969C938E9313970E94986400D070
:103ED000EDB7FEB731968FE498E0ADB7BEB7129656
:103EE0009C938E9311978091F11F8283138280910E
:103EF000F21F848315820E9498640F900F9082E6CF
:103F000098E0EDB7FEB79283818380917A04909117
:103F10007B04948383830E9498648DE798E0ADB717
:103F2000BEB712969C938E93119780917C049091CA
:103F30007D0414969C938E9313970E9498640F901F
:103F40000F900F900F900E94E909AB01BC0100D0C7
:103F500000D000D086E998E0EDB7FEB79283818368
:103F600043835483658376830E949864EDB7FEB7DC
:103F700036960FB6F894FEBF0FBEEDBF0E94320A10
:103F80000E94030AAB01BC0100D000D000D083EA3C
:103F900098E0ADB7BEB712969C938E931197EDB78C
:103FA000FEB743835483658376830E9498648DB7FC
:103FB0009EB706960FB6F8949EBF0FBE8DBF1D9B91
:103FC00003C08AEC92E002C086EC92E000D000D000
:103FD00021EB38E0ADB7BEB712963C932E93119704
:103FE00014969C938E9313970E9498648091941BCF
:103FF0009091951BA091961BB091971B4091981B97
:104000005091991B60919A1B70919B1B00D000D01E
:1040100000D00DB71EB70F5F1F4F2DEB38E0EDB787
:10402000FEB732832183F80182839383A483B5830F
:1040300046835783608771870E949864EDB7FEB707
:1040400038960FB6F894FEBF0FBEEDBF8AED98E02C
:10405000928381830E949864809178040F900F90DE
:1040600081FF0EC000D087EE98E0ADB7BEB71296C4
:104070009C938E9311970E9498640F900F9017C095
:1040800080FF03C083EC92E002C086EC92E000D097
:1040900000D02DEE38E0EDB7FEB732832183948354
:1040A00083830E9498640F900F900F900F908091DF
:1040B000780483FF03C083EC92E002C086EC92E0B8
:1040C00000D000D021EF38E0ADB7BEB712963C93D8
:1040D0002E93119714969C938E9313970E94986435
:1040E00080910E0690910F0624E039E0EDB7FEB7FF
:1040F00032832183948383830E9498640F900F906E
:104100000F900F90779903C083EC92E002C086EC89
:1041100092E000D000D021E139E0ADB7BEB71296F1
:104120003C932E93119714969C938E9313970E9411
:104130009864209194040F900F900F900F90222379
:1041400009F4A3C000D000D0EDB7FEB731968DE1E1
:1041500099E056C00E94AB1120919404222309F4E7
:1041600094C000D000D0EDB7FEB7319680E299E060
:1041700047C00E94B10E00D000D000D083E299E089
:10418000EDB7FEB79283818380913B1390913C13EE
:10419000A0913D13B0913E1383839483A583B6838E
:1041A0000E9498648EE299E0ADB7BEB712969C93D8
:1041B0008E9311978091ED1F9091EE1FA091EF1FAC
:1041C000B091F01FEDB7FEB783839483A583B683C8
:1041D0000E9498648DB79EB706960FB6F8949EBF5E
:1041E0000FBE8DBF0E94F00A20919404222309F48F
:1041F0004CC000D000D0EDB7FEB731968BE399E00C
:10420000ADB7BEB712969C938E93119722831382FB
:1042100009CA609192047091930480E090E00E943A
:10422000026460E173E00E9417640097A1F460915A
:1042300092047091930480E090E00E9402640097E1
:1042400021F10E94F962803100F590915201982B82
:10425000909352011AC08091520100D000D02EE3F9
:1042600039E0EDB7FEB73283218390E08F70907014
:10427000948383830E9498640F900F900F900F9007
:104280000E94F00A02C00E94F40FA981BA8111961F
:104290001C921E9283E00F900F90DF91CF911F919F
:1042A0000F91FF90EF90DF90CF90BF90AF909F90D5
:1042B0008F907F906F905F904F903F902F900895D8
:1042C000F89491E2E0E0F0E0909357008491E2E00E
:1042D000F0E0909357004491E4E0F0E090935700B1
:1042E000E49190E0A0E0B0E0DC019927882750E05D
:1042F00060E070E0762F652F542F4427840F951FC0
:10430000A61FB71F8E0F911DA11DB11D80931713FE
:1043100090931813A0931913B0931A1378940895D7
:10432000CF93DF9300D000D000D0CDB7DEB7CE0161
:1043300001966DE070E042E050E00E94C065898126
:104340009A812FEF8F3F920749F48CE794E06DE05C
:1043500070E042E050E00E94DE6504C090937D046E
:1043600080937C04CE0101966BE070E042E050E067
:104370000E94C06589819A812FEF8F3F920779F45F
:104380008CE390E090937B0480937A048AE794E036
:104390006BE070E042E050E00E94DE6504C0909364
:1043A0007B0480937A04CE01019669E070E042E0DC
:1043B00050E00E94C06589819A812FEF8F3F92075C
:1043C00079F482E090E0909379048093780488E710
:1043D00094E069E070E042E050E00E94DE6504C0D5
:1043E0009093790480937804CE0101966BE170E09C
:1043F00042E050E00E94C06589819A812FEF8F3F93
:10440000920769F410920F0610920E068EE096E065
:104410006BE170E042E050E00E94DE6504C09093E2
:104420000F0680930E0681EE9FE160E070E049E0A8
:1044300050E00E94C0650E94780CCE01039663E1B3
:1044400070E044E050E00E94C0658B819C81AD81AA
:10445000BE818F3F2FEF92072FEFA2072FEFB207FA
:1044600049F489E994E063E170E044E050E00E949F
:10447000DE6508C089E994E063E170E044E050E063
:104480000E94C065CE0103966FE070E044E050E00A
:104490000E94C0658B819C81AD81BE818F3F2FEFD3
:1044A00092072FEFA2072FEFB20749F485E994E0B6
:1044B0006FE070E044E050E00E94DE6508C085E9EE
:1044C00094E06FE070E044E050E00E94C065CE01EF
:1044D000039667E170E044E050E00E94C0658B8184
:1044E0009C81AD81BE818F3F2FEF92072FEFA207F6
:1044F0002FEFB20749F48DE994E067E170E044E002
:1045000050E00E94DE6508C08DE994E067E170E04C
:1045100044E050E00E94C06526960FB6F894DEBFD6
:104520000FBECDBFDF91CF9108956C9A6B9A6A9AB6
:104530006F9A729A749A739A779A809880B3897FE7
:1045400080BB87E080937E00549A0E9460210E9485
:10455000902181E00E94FA0880E090E00E948C0C9B
:104560000E94DE340895CF93DF93EC018881998116
:10457000009731F027E08136920709F077C06DC0CF
:104580000E9495228091780480FD02C00E94173C11
:10459000809170008C7F809370008091B600806263
:1045A0008093B6001092B20082E08093B1008091B7
:1045B000B60090E0877090700097C9F78091700006
:1045C0008160809370000E940E080E94B00880E015
:1045D00090E06FE976E00E94E9390E94CF1080E018
:1045E0000E9422120E94803E80931A060E94D93CAB
:1045F00080931B0600D000D000D0EDB7FEB73196F7
:1046000025E133E0ADB7BEB712963C932E931197D8
:104610008283138280911A06848315820E948664A5
:1046200010921D0610921C068DB79EB706960FB607
:10463000F8949EBF0FBE8DBF8EE694E09093EB1F63
:104640008093EA1F83E290E090931F0680931E06FA
:1046500081E697E0998388830DC0633259F48CE139
:1046600096E060E070E00E94F512E6CF19821882B1
:1046700083E001C081E0DF91CF91089585369105F7
:1046800064F120910E0630910F0620FF10C000D07B
:1046900000D027E233E0EDB7FEB732832183948365
:1046A00083830E9486640F900F900F900F908091EB
:1046B0004F1B9091501BA091511BB091521B019622
:1046C000A11DB11D80934F1B9093501BA093511BB4
:1046D000B093521B81E090E0089580E090E008954F
:1046E0004F925F926F927F928F929F92AF92BF9202
:1046F000CF92DF92EF92FF920F931F93CF93DF93AE
:10470000CDB7DEB7CA57D0400FB6F894DEBF0FBEA4
:10471000CDBF2C01633851F48EE296E0EB966FAF7B
:10472000EB970E942529EB966FADEB97D2018D9107
:104730009C911197009731F0B6E0843A9B0709F0FD
:10474000F7C40EC08EE296E061E870E045EA54E0FE
:104750000E940A2984EA96E0F20191838083EFC4E3
:10476000623109F0ECC40E946D0F80917C0480FFDF
:1047700060C000D000D000D0EDB7FEB7319672E037
:10478000C72ED12CCC0EDD1EADB7BEB71296DC9273
:10479000CE92119788E790E0938382838BE393E036
:1047A000958384830E94ED648C0181EEA82E8FE1B5
:1047B000B82EEDB7FEB736960FB6F894FEBF0FBE13
:1047C000EDBFEE24FF2498E7892E912C2FE3622E73
:1047D00023E0722ED5012D915D01EDB7FEB738971C
:1047E0000FB6F894FEBF0FBEEDBF3196C601800F25
:1047F000911FADB7BEB712969C938E93119793827B
:10480000828275826482268317820E94ED64080F7B
:10481000191F0894E11CF11CEDB7FEB738960FB6CE
:10482000F894FEBF0FBEEDBFF8E0EF16F10491F66D
:1048300002C000E010E080917C0490917D0400971C
:1048400081F12DB73EB7285030400FB6F8943EBFE7
:104850000FBE2DBFEDB7FEB73196CE010296800F89
:10486000911FADB7BEB712969C938E93119788E7B0
:1048700090E09383828384E493E0958384838091A2
:104880000B0690910C06978386830E94ED64080FB7
:10489000191FEDB7FEB738960FB6F894FEBF0FBEDE
:1048A000EDBF80917C0481FF51C089E290E06BE212
:1048B00070E04AE250E027E00E94FF3181EE9FE184
:1048C0000E9466342DB73EB72A5030400FB6F89498
:1048D0003EBF0FBE2DBFEDB6FEB60894E11CF11C25
:1048E0009E012E5F3F4F200F311FADB7BEB712960E
:1048F0003C932E93119728E730E0F701338322830E
:104900002BE433E0358324839C01B901882777FDAC
:104910008095982F0E949D5F20E030E048EC52E4A3
:104920000E94335FDC01CB01F70186839783A08768
:10493000B1870E94ED64080F191F2DB73EB7265F9F
:104940003F4F0FB6F8943EBF0FBE2DBF80917C0441
:1049500090917D0494FF54C089E290E06BE270E096
:104960004AE250E026E00E94FF3181E090E00E94A0
:10497000840A80930A068FEC92E10E946634ADB7F8
:10498000BEB71A970FB6F894BEBF0FBEADBFEDB657
:10499000FEB60894E11CF11C9E012E5F3F4F200FD4
:1049A000311F12963C932E93119728E730E0F701C0
:1049B0003383228325E533E0358324839C01B901C9
:1049C000882777FD8095982F0E949D5F20E030E03A
:1049D00048EC52E40E94335FDC01CB01F70186838F
:1049E0009783A087B1870E94ED64080F191F2DB728
:1049F0003EB7265F3F4F0FB6F8943EBF0FBE2DBFA8
:104A000080917C0482FF35C08DB79EB70A970FB6A0
:104A1000F8949EBF0FBE8DBFEDB7FEB73196CE01A5
:104A20000296800F911FADB7BEB712969C938E93DE
:104A3000119788E790E09383828380E693E09583E3
:104A400084838091C2129091C312A091C412B0913C
:104A5000C51286839783A087B1870E94ED64080FF3
:104A6000191FEDB7FEB73A960FB6F894FEBF0FBE0A
:104A7000EDBF80917C0483FF32C00E94030AAB012A
:104A8000BC012DB73EB72A5030400FB6F8943EBF58
:104A90000FBE2DBFEDB7FEB73196CE010296800F47
:104AA000911FADB7BEB712969C938E93119788E76E
:104AB00090E0938382838EE693E09583848346839C
:104AC0005783608771870E94ED64080F191FEDB747
:104AD000FEB73A960FB6F894FEBF0FBEEDBF8091B9
:104AE0007C0484FF36C04091941B5091951B6091CB
:104AF000961B7091971B2DB73EB72A5030400FB6CA
:104B0000F8943EBF0FBE2DBFEDB7FEB73196CE0174
:104B10000296800F911FADB7BEB712969C938E93ED
:104B2000119788E790E0938382838CE793E09583E5
:104B3000848346835783608771870E94ED64080FE2
:104B4000191FEDB7FEB73A960FB6F894FEBF0FBE29
:104B5000EDBF80917C0485FF72C0A0907A04B09074
:104B60007B04A114B10409F46AC04091941B5091D4
:104B7000951B6091961B7091971BC090C612D090A8
:104B8000C712E090C812F090C9122DB73EB72A5054
:104B900030400FB6F8943EBF0FBE2DBF8DB69EB607
:104BA0000894811C911CCE010296800F911FADB715
:104BB000BEB712969C938E93119788E790E0F4010C
:104BC0009383828385E893E0958384834C195D0900
:104BD0006E097F09CB01BA010E949B5F6B017C01CA
:104BE000B50180E090E00E949B5F9B01AC01C70192
:104BF000B6010E94335FDC01CB01F4018683978309
:104C0000A087B1870E94ED64080F191F8091941B43
:104C10009091951BA091961BB091971B8093C61203
:104C20009093C712A093C812B093C9122DB73EB784
:104C3000265F3F4F0FB6F8943EBF0FBE2DBF809149
:104C40007C0486FF3BC04091981B5091991B60915A
:104C50009A1B70919B1B8DB79EB70A970FB6F8945D
:104C60009EBF0FBE8DBFEDB7FEB73196CE01029647
:104C7000800F911FADB7BEB712969C938E9311977C
:104C800088E790E09383828382E993E0958384832D
:104C900046835783608771870E94ED64080F191F50
:104CA000EDB7FEB73A960FB6F894FEBF0FBEEDBF54
:104CB000C8010E943E23009709F040C280917C0405
:104CC00087FF3CC040913F1B5091401B6091411BAE
:104CD0007091421B2DB73EB72A5030400FB6F89462
:104CE0003EBF0FBE2DBFEDB7FEB73196CE01029687
:104CF000800F911FADB7BEB712969C938E931197FC
:104D000088E790E0938382838BE993E095838483A3
:104D100046835783608771870E94ED64080F191FCF
:104D2000EDB7FEB73A960FB6F894FEBF0FBEEDBFD3
:104D3000C8010E943E23009709F000C280917C04C4
:104D400090917D0490FF3CC02DB73EB72A50304073
:104D50000FB6F8943EBF0FBE2DBFEDB7FEB731962C
:104D6000CE010296800F911FADB7BEB712969C93ED
:104D70008E93119788E790E09383828384EA93E08F
:104D80009583848380913B1390913C13A0913D13B4
:104D9000B0913E1386839783A087B1870E94ED640C
:104DA000080F191FEDB7FEB73A960FB6F894FEBF7D
:104DB0000FBEEDBFC8010E943E23009709F0BEC19F
:104DC00080917C0490917D0491FF3CC02DB73EB74B
:104DD0002A5030400FB6F8943EBF0FBE2DBFEDB73E
:104DE000FEB73196CE010296800F911FADB7BEB7C8
:104DF00012969C938E93119788E790E09383828319
:104E00008FEA93E0958384838091DC1F9091DD1F6E
:104E1000A091DE1FB091DF1F86839783A087B187A3
:104E20000E94ED64080F191FEDB7FEB73A960FB652
:104E3000F894FEBF0FBEEDBFC8010E943E2300974D
:104E400009F07CC180917C0490917D0492FF4CC05C
:104E500081E00E949509AB01BC012DB73EB72A50F5
:104E600030400FB6F8943EBF0FBE2DBFEDB6FEB674
:104E70000894E11CF11CCE010296800F911FADB782
:104E8000BEB712969C938E93119788E790E0F70136
:104E9000938382838CEB93E095838483CB01BA0167
:104EA0002091990430919A0440919B0450919C0464
:104EB0000E944D60DC01CB01F70186839783A087B8
:104EC000B1870E94ED64080F191F2DB73EB7265F0A
:104ED0003F4F0FB6F8943EBF0FBE2DBFC8010E94D2
:104EE0003E23009709F02AC180917C0490917D04B3
:104EF00093FF4BC082E00E949509AB01BC018DB7C6
:104F00009EB70A970FB6F8949EBF0FBE8DBFEDB641
:104F1000FEB60894E11CF11CCE010296800F911F91
:104F2000ADB7BEB712969C938E93119788E790E029
:104F3000F7019383828389EC93E095838483CB018B
:104F4000BA012091950430919604409197045091B4
:104F500098040E944D60DC01CB01F70186839783A2
:104F6000A087B1870E94ED64080F191F2DB73EB7C7
:104F7000265F3F4F0FB6F8943EBF0FBE2DBFC8014E
:104F80000E943E23009709F0D9C0779A80910E06BF
:104F900090910F0693FD749A80910E0690910F06E2
:104FA00082FD08C08091780480FD04C081FF31C07B
:104FB0001D9B2FC000D000D086ED93E0ADB7BEB7EB
:104FC00012969C938E931197CE01029614969C9301
:104FD0008E9313970E948664209194040F900F90F3
:104FE0000F900F902223A9F000D000D0EDB7FEB7AC
:104FF000319685E999E0ADB7BEB712969C938E9332
:105000001197228313820E9498640F900F900F9043
:105010000F90809139068983FE01E00FF11F128203
:1050200062E0E62EF12CE00EF11E00D000D08DEDF6
:1050300093E0EDB7FEB792838183F482E3820E940E
:1050400086640F900F900F900F90CE010196B701DC
:105050000E940B318091780482FF49C08EE794E072
:10506000BE016F5F7F4FA7012CE93BE10E946035D5
:1050700080910E0690910F0692FF39C04CE9C42E24
:105080004BE1D42E00E010E057EEA52E53E0B52EF4
:10509000D6018D916D0100D000D0EDB7FEB73196ED
:1050A000ADB7BEB71296BC92AE92119782831382AF
:1050B0000E9486640F5F1F4F0F900F900F900F900C
:1050C0000031110529F78AE090E00E94B86400D011
:1050D00000D08CEE93E0EDB7FEB792838183F4822B
:1050E000E3820E9486640F900F900F900F90809142
:1050F0000E0690910F0682FD73980E94263B8EE269
:1051000096E00E94282980910B0690910C0600974A
:1051100011F00E94173C809139068F5F8093390609
:1051200080910E0690910F0682FF14CB739A12CBDA
:10513000D20111961C921E9283E002C001C081E050
:10514000C658DF4F0FB6F894DEBF0FBECDBFDF915C
:10515000CF911F910F91FF90EF90DF90CF90BF9074
:10516000AF909F908F907F906F905F904F90089539
:105170000895FC01DB018C91808311968C9111972D
:1051800081830895FC01DB0190818C91981741F493
:1051900021E030E0918111968C911197981711F0D0
:1051A00020E030E0C9010895BC0181EF9FE10E9439
:1051B000B9280895DC011996ED91FC911A970280A7
:1051C000F381E02D309709F0099508950F931F930F
:1051D000CF93DF9300D0CDB7DEB78C0188E10E947A
:1051E0007A31BC01CE0101960E94B928D8011996E6
:1051F000ED91FC911A970190F081E02DC801BE015C
:105200006F5F7F4F09950F900F90DF91CF911F91A6
:105210000F910895EF92FF920F931F93CF93DF9317
:10522000EC018B017A0143EB54E00E943629FA86A7
:10523000E986C80167EB74E00E949429DF91CF9161
:105240001F910F91FF90EF9008950E944F290895AC
:10525000CF93DF93EC0188E161EF7FE10E94703131
:10526000CE010E945229DF91CF910895EF92FF92D3
:105270000F931F93CF93DF93EC018B017A010E9470
:105280007029F886EF82C8016BEB74E00E949429C4
:10529000DF91CF911F910F91FF90EF9008950E94A1
:1052A000792908950E948F410895DC011796ED91A8
:1052B000FC9118970190F081E02D09950895DC018B
:1052C0001796ED91FC9118970280F381E02D3097AD
:1052D00009F0099508958AEB99E00E94E32B08955F
:1052E000FC01738362838AEB99E0BF010E94562C14
:1052F0000895BC018AEB99E00E94212C0895CF9378
:10530000DF93EC018AEB99E00E94E72B08C0FC01D7
:10531000228133812C173D0721F00E948D2C0097AC
:10532000B1F7DF91CF9108950F931F93CF93DF9340
:105330008B010E947F29EC01009731F01D830C83C3
:10534000C8010E94D2438E83DF91CF911F910F91AC
:1053500008951F93CF93DF93EC01162F888580FF6C
:105360001DC0EC81FD813097C9F0D093BD09C09379
:10537000BC0982E08887CE0106960995992787FDAA
:10538000909502978230910510F0133829F4CE01E0
:10539000BE010E94D22902C081E08887DF91CF91AF
:1053A0001F910895CF92DF92EF92FF920F931F9378
:1053B000CF93DF93EC017B01C090BC09D090BD0975
:1053C0000091BE091091BF09F80103C00190F0815E
:1053D000E02DEC17FD0719F03097C1F746C0209774
:1053E00009F443C08885882309F118860BC0C017CB
:1053F000D10729F0C80167E8AE010E94A929F80188
:10540000008111810115110591F7EC81FD81309723
:1054100069F0CE15DF0551F0D093BD09C093BC09EA
:10542000CE01069663E840E050E00995E091BE09A0
:10543000F091BF09CE17DF0791F48881998190938D
:10544000BF098093BE090DC0808191818C179D0793
:1054500029F4888199819183808303C0FC0130976E
:1054600099F7D092BD09C092BC09DF91CF911F91ED
:105470000F91FF90EF90DF90CF9008951F93CF93FF
:10548000DF931092C009C091BE09D091BF0911E00D
:105490000EC08985882341F018871986CE0162E8FD
:1054A00040E050E00E94A9290990D881C02D2097A2
:1054B00081F7DF91CF911F9108958091C109982FB5
:1054C0009F5F9093C10908956091BC097091BD09D7
:1054D0000E94D22908958AE88093C1091092C209D6
:1054E0001092C3091092BF091092BE091092BD0913
:1054F0001092BC0908958091C009882311F00E9480
:105500003E2A7091C309772309F455C02091C2093E
:1055100030E0F901EE0FFF1FEE0FFF1FE20FF31F48
:10552000EC53F64F60816093640A4181528150933D
:10553000660A4093650A838194819093680A8093F8
:10554000670A2F5F3F4F2F7130702093C20971504F
:105550007093C309009741F58091BE099091BF09EE
:1055600018C08091C009882311F00E943E2A409102
:10557000650A5091660A8091690A90916A0A609161
:10558000640A0E94A929E091690AF0916A0A80815F
:10559000918190936A0A8093690A8091690A909137
:1055A0006A0A0097F1F607C0613819F421E0FC019E
:1055B00020870E94A9298091C0092091C30990E009
:1055C000820F911D08958091C0092091C30990E038
:1055D000820F911D08959C017091C3097032D9F01A
:1055E0008091C209870F8F7180936B0A90E0FC0154
:1055F000EE0FFF1FEE0FFF1FE80FF91FEC53F64FE2
:10560000608352834183348323837F5F7093C30914
:1056100080E090E0089581E090E00895CF93DF93DB
:10562000C091BC09D091BD090E94A929D093BD09A0
:10563000C093BC09DF91CF910895FC01AB0190911B
:10564000BE098091BF09A92FB82F03C00D90BC914E
:10565000A02DAE17BF0791F01097C1F7309771F0EA
:1056600090838183F093BF09E093BE0981E0808736
:1056700017821682CF0161E80E940E2B0895FC016B
:10568000009741F080858150823020F481E081874D
:105690008093C009089521E030E0FC0180858823D3
:1056A00011F420E030E0C9010895CF93DF93EC01BD
:1056B0004A815B818C819D8160E070E00E94106472
:1056C0002A813B8188819981289FA001299F500DC3
:1056D000389F500D11248E819F8160E070E00E9400
:1056E0001064DF91CF910895DC0112962D913C91C9
:1056F000139780E090E01DC01496ED91FC911597F2
:10570000E80FF91F4081442399F421E020832D9173
:105710003C911197829FA001839F500D929F500D45
:10572000112416968D919C911797840F951F0895BB
:1057300001968217930701F780E090E00895FC013D
:1057400046815781A281B38120E030E019C046171D
:10575000570781F4A481B581A20FB31F8C9118164D
:1057600014F481508C930480F581E02DE20FF31F37
:105770008081089580819181480F591F2F5F3F4F8D
:105780002A173B0721F78FEF0895FC0146815781C7
:1057900064177507A8F0A081B18182819381A89FC9
:1057A0009001A99F300DB89F300D1124240F351F93
:1057B00081E090E06217730728F080E090E00895A0
:1057C00080E090E00895FC01118210820895FC01B0
:1057D000808191810895FB0120813181FC01318319
:1057E00020830895FC0180819181009711F4089530
:1057F000C901FC012081318121153105C9F70895C6
:10580000DC01ED91FC911197309729F40BC0DF0179
:105810000190F081E02D808191810097C1F7119670
:105820001C921E92CF010895DC01ED91FC9111971D
:10583000309729F08081918111969C938E93CF01AE
:105840000895CF93DF93EC01E881F9813097B9F0A7
:10585000A0E0B0E002C0DF01FC0180819181E61789
:10586000F70759F4109719F49983888303C01196A8
:105870009C938E931182108202C0009761F7DF9192
:10588000CF9108950F931F93CF93DF938C01EB017A
:105890000E94212CF8018081918199838883D18392
:1058A000C083DF91CF911F910F9108950F931F93A4
:1058B000CF93DF938C01EB010E94212C1982188277
:1058C000C8010E94F22B009711F4F80101C0FC01FD
:1058D000D183C083DF91CF911F910F910895DC0197
:1058E000ED91FC91119780E090E004C00196019049
:1058F000F081E02D3097D1F70895FB01BA01309780
:1059000019F40E94422C089580819181DA01119648
:105910009C938E93518340830895009721F0FC015E
:1059200080819181089580E090E0089580916C0AD3
:1059300090916D0A009729F410926F0A10926E0AE6
:1059400008950E949738BC01E0916C0AF0916D0AAD
:105950004281538180819181480F591F461B570B0B
:105960000CC08281938120813181820F931F861B1D
:10597000970B8417950708F4AC010480F581E02D9E
:10598000309779F7460F571F50936F0A40936E0A6E
:10599000089589EC94E00E943F2B0895EF92FF92C6
:1059A0000F931F93CF93DF937C01FC018081918142
:1059B000009729F08A35910509F06DC00BC010924F
:1059C0006D0A10926C0A8AE590E0F701918380835A
:1059D00081E065C0673859F5A0916C0AB0916D0AF5
:1059E00004C014960D90BC91A02D109741F316960B
:1059F0008D919C9117978417950799F3A0936C0A42
:105A0000B0936D0A0DC0868197818417950739F48C
:105A10008481958115969C938E931497FD01DF01E7
:105A20001496ED91FC911597309769F7CCCF6238B9
:105A300051F6C0916C0AD0916D0A00E010E028C0C8
:105A4000CE010E94B7470097F1F08E819F8168E8F0
:105A5000AE010E94EB2A0097A1F41F821E828C8166
:105A60009D810115110521F0F8019583848304C0FF
:105A700090936D0A80936C0A1D821C820E94962C62
:105A8000D8CF0E94C92C9C818D818E01C92FD82F1F
:105A90002097B1F698CFF7011182108283E0DF9151
:105AA000CF911F910F91FF90EF900895CF93DF93C7
:105AB000EC010E94C92C8E819F8130916C0A20914B
:105AC0006D0A009759F0E32FF22F06C0EC17FD077F
:105AD00089F00480F581E02D3097C1F78091BC09F1
:105AE0009091BD099F838E833C832D83D0936D0A53
:105AF000C0936C0A0E94962CDF91CF910895CF93AA
:105B0000DF93EC010E949747CE010E94562DDF9152
:105B1000CF910895CF93DF93EC010E94A347CE016C
:105B20000E94562DDF91CF910895CF93DF93EC0122
:105B30000E94AD47CE010E94562DDF91CF9108956E
:105B4000FC0180819181860F971F918380830E9441
:105B5000962C089521E030E0FC0186819781009722
:105B600011F020E030E0C9010895FC012281338169
:105B700080819181280F391FC9010895FC0180811E
:105B80009181089581E090E020916C0A30916D0A36
:105B90002115310511F480E090E0089580916C0AA0
:105BA00090916D0A009729F080916E0A90916F0A8A
:105BB000089580E090E00895CF93DF93EC01E091A9
:105BC0006C0AF0916D0A8E179F0741F48C819D81BC
:105BD00090936D0A80936C0A14C0FC01309731F0E9
:105BE000848195818C179D07C1F707C01D821C8297
:105BF0001F821E82DF91CF9108958C819D819583B4
:105C000084830E94962CF2CFCF93DF93D091F11F23
:105C1000C091F21F0E94C338AB01BC018DB79EB783
:105C2000825590400FB6F8949EBF0FBE8DBFEDB762
:105C3000FEB731968BE999E0ADB7BEB712969C934B
:105C40008E931197D2831382C48315824683578320
:105C5000608771878091E4219091E521A091E621F0
:105C6000B091E72182879387A487B5878091E82147
:105C70009091E921A091EA21B091EB218687978745
:105C8000A08BB18B8091EC219091ED21A091EE2120
:105C9000B091EF21828B938BA48BB58B8091F021F7
:105CA0009091F121A091F221B091F321868B978BF5
:105CB000A08FB18F8091F4219091F521A091F621D0
:105CC000B091F721828F938FA48FB58F8091F821A7
:105CD0009091F921A091FA21B091FB21868F978FA5
:105CE000A0A3B1A38091FC219091FD21A091FE2160
:105CF000B091FF2182A393A3A4A3B5A38091002216
:105D000090910122A0910222B091032286A397A331
:105D1000A0A7B1A78091042290910522A09106220C
:105D2000B091072282A793A7A4A7B5A780910822C4
:105D300090910922A0910A22B0910B2286A797A7E1
:105D4000A0ABB1AB80910C2290910D22A0910E22BC
:105D5000B0910F2282AB93ABA4ABB5AB8091102274
:105D600090911122A0911222B091132286AB97AB91
:105D7000A0AFB1AF8091142290911522A09116226C
:105D8000B091172282AF93AFA4AFB5AFEDB7FEB716
:105D9000FF968091182290911922A0911A22B09119
:105DA0001B2280839183A283B383EDB7FEB7ED5BA3
:105DB000FF4F80911C2290911D22A0911E22B09134
:105DC0001F2280839183A283B383EDB7FEB7E95B83
:105DD000FF4F8091202290912122A0912222B09108
:105DE000232280839183A283B383EDB7FEB7E55B63
:105DF000FF4F8091242290912522A0912622B091DC
:105E0000272280839183A283B383EDB7FEB7E15B42
:105E1000FF4F8091282290912922A0912A22B091AF
:105E20002B2280839183A283B3830E949864D091B4
:105E3000F11FC091F21F8DB79EB78E5A9F4F0FB6BC
:105E4000F8949EBF0FBE8DBF0E94C338AB01BC014A
:105E5000ADB7BEB7D2970FB6F894BEBF0FBEADBFF9
:105E6000EDB7FEB7319687E79AE012969C938E9332
:105E70001197D2831382C483158246835783608728
:105E8000718780912C2290912D22A0912E22B09189
:105E90002F2282879387A487B587809130229091A3
:105EA0003122A0913222B091332286879787A08B2E
:105EB000B18B8091342290913522A0913622B091FD
:105EC0003722828B938BA48BB58B80913822909153
:105ED0003922A0913A22B0913B22868B978BA08FDA
:105EE000B18F80913C2290913D22A0913E22B091B1
:105EF0003F22828F938FA48FB58F80914022909103
:105F00004122A0914222B0914322868F978FA0A375
:105F1000B1A38091442290914522A0914622B09154
:105F2000472282A393A3A4A3B5A380914822909172
:105F30004922A0914A22B0914B2286A397A3A0A701
:105F4000B1A78091542290915522A0915622B091F0
:105F5000572282A793A7A4A7B5A780915822909112
:105F60005922A0915A22B0915B2286A797A7A0AB95
:105F7000B1AB0E9498648DB79EB7C2960FB6F894E5
:105F80009EBF0FBE8DBFDF91CF91089580E38093B8
:105F9000740A0895CF93DF936091740A70E0C0E3B0
:105FA000D0E0C61BD70B6958754FAE010E9407643D
:105FB000CE01DF91CF910895CF92DF92EF92FF92C1
:105FC0000F931F93CF93DF937C01C090720AD09000
:105FD000730A6091740A70E08601005D1F4F061B12
:105FE000170B01381105D8F4C0E3D0E0C61BD70B5E
:105FF0006958754FAE010E940764C7018C0F9D1F41
:106000006091750A7091760A2091700A3091710A38
:10601000620F731FA6010E940764C80102C080E0DE
:1060200090E0DF91CF911F910F91FF90EF90DF9063
:10603000CF9008959091740A980F9093740A0895E0
:106040004091720A5091730A9C014817590798F0C1
:106050008091700A9091710A820F931F9093710A38
:106060008093700A421B530B5093730A4093720A39
:1060700081E090E0089580E090E008959093730AA5
:106080008093720A08958091700A9091710A8955DF
:10609000954F08958091740A90E08958954F08951E
:1060A00081E090E02091750A3091760A4AE0273A23
:1060B000340711F480E090E008950E94503000977A
:1060C00069F087EA9AE06091750A7091760A4091CA
:1060D000720A5091730A0E94076408954091700AF1
:1060E0005091710A41155105C1F08091720A909149
:1060F000730AC096A7EABAE020E330E007C0FD01CA
:10610000E40FF51F60816D932F5F3F4F281739070C
:10611000B4F31092710A1092700A08958091750A72
:106120009091760A08958091720A9091730A089569
:106130009091740A80E3891B089520E38091740A8A
:10614000281B8091720A9091730A820F911D089505
:106150001F93CF93DF93EC011091740A812F90E08D
:106160008C179D076CF00E949D308C0F9D1F81380D
:10617000910530F41C1B1093740A81E090E002C07A
:1061800080E090E0DF91CF911F910895CF93DF934E
:10619000EBEFFFE11192119280E2EB32F807D1F7B9
:1061A000C0E0D0E0CE01880F991F8D50904E61EB7A
:1061B00074E00E94B9282196C430D10599F7DF9187
:1061C000CF9108951092710A1092700A1092730A7A
:1061D0001092720A80E38093740A87EA9AE090939F
:1061E000760A8093750A0E94C63008950F931F9314
:1061F000CF93DF93EC018B010E94E230D093760ABB
:10620000C093750A1093730A0093720ADF91CF91BD
:106210001F910F910895EF92FF920F931F93CF93C9
:10622000DF9300D0CDB7DEB78C0169837A830E94FB
:10623000E2306981E62E7A81F72E81E8E816F104D2
:1062400018F030E8E32EF12C8091750A9091760ACF
:10625000B801A7010E940764F092730AE092720AE3
:10626000C7010F900F90DF91CF911F910F91FF9079
:10627000EF900895FC01ABEFBFE180E30D90019238
:106280008150E1F7FB01A3EFBFE188E00D9001929F
:106290008150E1F70895ABEFBFE1FC0180E301908D
:1062A0000D928150E1F7A3EFBFE1FB0188E001907F
:1062B0000D928150E1F70895E82FF0E0EE0FFF1FF7
:1062C000E550F04E7183608381E090E00895E82FFF
:1062D000F0E0EE0FFF1FE550F04E808191810895B0
:1062E00090E0880F991F8D53904E0E94B92881E04D
:1062F00090E0089590E0880F991F8D53904E089577
:106300008115910511F00197F1F70895E0912E2084
:10631000F0912F20908180912D2089230895E09184
:106320002B20F0912C20808190912D20892B80832F
:10633000E0913020F0913120808190912D20892BA7
:1063400080830895E0912B20F0912C209081809102
:106350002D20809589238083E0913020F091312099
:10636000908180912D2080958923808308951F93AB
:10637000CF93DF93E0912B20F0912C20908180919E
:106380002D20809589238083E0913020F091312069
:10639000808190912D20892B80838FEB93E00E9448
:1063A00080311FB7F894E0913020F0913120908136
:1063B00080912D2080958923808383E890E00E943E
:1063C0008031E0912E20F0912F20D081C0912D209E
:1063D0001FBF78948BE393E00E948031E0912E20E0
:1063E000F0912F20808190912D20892319F08D2FFD
:1063F0008C2301C081E0DF91CF911F9108955093CC
:1064000031204093302070932C2060932B20909368
:106410002F2080932E2081E090E002C0880F991FEA
:106420002A95E2F780932D200E94B7310895CF93EB
:10643000DF93C82FDFB7F894E0913020F09131203E
:10644000808190912D20892B808383E090E00E94B1
:106450008031CC2351F0E0913020F09131209081B7
:1064600080912D2080958923808387E190E00E9490
:106470008031E0912E20F0912F20808190912D206D
:10648000892309F4C0E089E590E00E948031E09121
:106490003020F0913120908180912D2080958923AA
:1064A0008083DFBF8BE390E00E9480318C2FDF91EF
:1064B000CF910895CF93DF93C82FD8E08C2F8170B0
:1064C0000E941732C6958111C068D150B9F78C2F40
:1064D000DF91CF9108958FEF0E945A320895DF9295
:1064E000EF92FF920F931F93CF93DF93182FEB013F
:1064F0000E94B731882381F580EF0E945A32EE2442
:1065000000E498E0D92E81E00E941732F82E81E055
:106510000E941732882319F0FF2069F020C0FF2065
:1065200051F4011728F0888180FF05C0101719F079
:10653000E02EFF24F3948F2D0E94173288818695D8
:106540008883FF2011F0806888830150DA94D9F69F
:1065500021960023B1F605C0EE24EA9402C08EEF26
:10656000E82E8E2DDF91CF911F910F91FF90EF902C
:10657000DF9008950F931F93CF93DF93182FEB01B4
:106580000E94B731209751F085E50E945A3208E009
:1065900089910E945A320150D9F703C08CEC0E94B5
:1065A0005A32812F0E945A32DF91CF911F910F9161
:1065B00008950F931F93CF93DF93E82FDB01EA0138
:1065C000B9014C9150E011969C91119780E0482BB5
:1065D000592BE03181F4CA018E7F33E0880F991F77
:1065E0003A95E1F716962C9116974CE050E0421B35
:1065F0005109480F591F57FF06C081E08883509505
:1066000041955F4F01C01882E83299F414968C913D
:10661000149790E09C01207630702036310549F0C7
:1066200086FF02C04E7F05C085FF02C04C7F01C0BF
:10663000487FCA0124E0969587952A95E1F7FB01EA
:1066400080834F70F801408380E0DF91CF911F91EC
:106650000F9108950F931F93CF93DF93EC018B015C
:106660008881B8010E946F32888381508D3F30F459
:10667000F8018081883211F0803191F7DF91CF915C
:106680001F910F910895CF93DF93EC010E94B731D2
:1066900084EBBE010E94BA3281E00E941732C82FFB
:1066A0000E94B73181E0CC2309F480E0DF91CF91E3
:1066B00008951F93CF93DF93182FEB010E94B731FA
:1066C0000E948631882349F084E4BE010E94BA32D8
:1066D000113029F00E948F3102C082E001C080E0B9
:1066E000DF91CF911F9108956F927F928F929F9229
:1066F000BF92CF92DF92EF92FF920F931F93CF93AF
:10670000DF93CDB7DEB729970FB6F894DEBF0FBE83
:10671000CDBF7C014B013A0169010E94B7318EEB7C
:10672000B7010E94BA328E010F5F1F4FE9E0BE2E03
:106730000E946B32F80181938F01BA94C9F7CE01A0
:10674000019669E070E00E94854D882361F4F701AD
:106750008081BE016F5F7F4FA401930186010E947B
:10676000D93280E001C083E029960FB6F894DEBFED
:106770000FBECDBFDF91CF911F910F91FF90EF9092
:10678000DF90CF90BF909F908F907F906F900895F3
:106790008F929F92AF92BF92CF92DF92EF92FF9231
:1067A0000F931F93CF93DF93CDB7DEB729970FB623
:1067B000F894DEBF0FBECDBFD82E5B014A01790130
:1067C0008EEB60E070E00E94BA328E010F5F1F4FC7
:1067D000F9E0CF2E0E946B32F80181938F01CA94A9
:1067E000C9F7CE01019669E070E00E94854D8823CB
:1067F00059F48D2DBE016F5F7F4FA5019401870174
:106800000E94D93280E001C083E029960FB6F89447
:10681000DEBF0FBECDBFDF91CF911F910F91FF90D3
:10682000EF90DF90CF90BF90AF909F908F900895A2
:10683000EF92FF921F93CF93DF93CDB7DEB72897E8
:106840000FB6F894DEBF0FBECDBF182F262FDE0186
:106850001196E3EDF4E088E001900D928150E1F7AC
:10686000E42EFF24E7FCF09441E752E0E49EC001EF
:10687000E59E900DF49E900D112464E670E00E9458
:10688000E360CB0134E6239F90011124820F931F14
:10689000FE01319640E0219130E0E216F30611F45A
:1068A000019603C04F5F4830B1F7112319F090955E
:1068B00081959F4F28960FB6F894DEBF0FBECDBFCF
:1068C000DF91CF911F91FF90EF9008950F931F9349
:1068D000CF93DF93CDB7DEB72B970FB6F894DEBF1B
:1068E0000FBECDBF182F092F885F612F792F0E940F
:1068F0005933882309F048C066E471E48FE090E0E2
:106900000E94D134812F902FBE016D5F7F4FAE0169
:106910004E5F5F4F9E012F5F3F4F0E94743388236D
:1069200099F5DE011496E3EDF4E088E001900D9214
:106930008150E1F7E9814E2F50E021E732E0429F9C
:10694000C001439F900D529F900D112464E670E0AA
:106950000E94E360CB013A8124E6329F900111242A
:10696000820F931FDE01149620E03D91E31711F48E
:10697000019603C02F5F2830C1F72B81222331F00D
:10698000909581959F4F02C084E391E22B960FB6BC
:10699000F894DEBF0FBECDBFDF91CF911F910F9155
:1069A0000895DC01CB0181159105A105B10529F000
:1069B00081509040A040B040D9F708951092B9009E
:1069C00080E28093B800089594EA9093BC0090917F
:1069D000BC0097FFFCCF9091B900987F983011F0E0
:1069E000903199F48093BB0084E88093BC0080913F
:1069F000BC0087FFFCCF9091B900987F983139F0A7
:106A000081E0903429F480E0089581E0089580E0E9
:106A1000089544EA34E824E94093BC009091BC0016
:106A200097FFFCCF9091B900987F983011F090318A
:106A300099F78093BB003093BC009091BC0097FF06
:106A4000FCCF9091B900987F903211F0983539F4CD
:106A50002093BC009091BC0094FDFCCFDDCF089545
:106A60000E94E434089584E98093BC008091BC00C6
:106A700084FDFCCF08958093BB0084E88093BC0024
:106A80008091BC0087FFFCCF9091B900987F81E096
:106A9000983209F480E0089584EC8093BC008091E2
:106AA000BC0087FFFCCF8091BB00089584E88093F1
:106AB000BC008091BC0087FFFCCF8091BB00089593
:106AC000FC0180E1919190933F018150D9F7809131
:106AD0003C018F7D80933C0180913C01877F8093B6
:106AE0003C01FB0180E1919190933E018150D9F7E7
:106AF00080913C01806880933C0180913D0180FF42
:106B0000FCCF4051504080913C01806280933C0119
:106B100080913C01877F80933C0112C0FB0180E1A2
:106B2000919190933E018150D9F780913C0180680A
:106B300080933C0180913D0180FFFCCF405150404B
:106B4000141615065CF3F90180E190913E019193D2
:106B50008150D9F781E090E00895E6E4F1E080818A
:106B600020819081308182958695869583702295CB
:106B70002F70822B832B92959F70892B0895DF9223
:106B8000EF92FF920F931F93CF93DF9300D0CDB777
:106B9000DEB780E06CE046E00E945B3989E18093DB
:106BA000C4001092C50082E08093C00080E00E9483
:106BB000FD390E94873884B784B784B784B784B717
:106BC000E2EBF8E222E432E4318320833A968DB797
:106BD0009EB70A97E817F907B8F300D000D086EE01
:106BE0009AE0ADB7BEB712969C938E9311978BED3A
:106BF00094E014969C938E9313970E9498640F9040
:106C00000F900F900F900E94B6490E946B2A89EC5A
:106C100094E060E070E00E941D2B0E944948E091E2
:106C20002605F091270509950E94AD3590E00E9458
:106C3000F349CE0101960E94B937882359F000D05C
:106C400081E09BE0EDB7FEB7928381830E94986458
:106C50000F900F90CE0101960E94D4280E94C33756
:106C60008C010E94C837BC01C801AE014F5F5F4F65
:106C70000E94F73C0E9426370E94DC3C0E94CD37E0
:106C80000E94783E00D081E29BE0ADB7BEB712967D
:106C90009C938E9311970E94986400D0EDB7FEB735
:106CA00031960EE21BE0ADB7BEB712961C930E9361
:106CB00011978A81828313820E949864EDB7FEB790
:106CC0003196ADB7BEB712961C930E93119789817A
:106CD000828313820E9498640F900F9082E39BE05E
:106CE000EDB7FEB7928381830E9498640F900F9056
:106CF0000E94F949E091A905F091AA050995E09152
:106D00009005F09191050995E0915205F091530598
:106D1000099500918E0510918F05E090A705F090E0
:106D2000A8050E94D93CD82E0E94803E2DB73EB7C0
:106D30002A5030400FB6F8943EBF0FBE2DBFEDB7BE
:106D4000FEB7319624E33BE0ADB7BEB712963C9355
:106D50002E93119713830283F582E482D6821782E1
:106D6000808711860E949864E091B305F091B40584
:106D70002DB73EB7265F3F4F0FB6F8943EBF0FBE0C
:106D80002DBF3097D1F00995BC0100D000D08FE421
:106D90009BE0ADB7BEB712969C938E93119780E897
:106DA00090E00E94CF60EDB7FEB7748363830E94CA
:106DB00098640F900F900F900F9000D082E69BE0A8
:106DC000ADB7BEB712969C938E9311970E949864AC
:106DD0000F900F908BEE95E060E070E00E941D2B0D
:106DE00084EF93E00E947B4700D084E69BE0EDB700
:106DF000FEB7928381830E9498640F900F900F904A
:106E00000F90DF91CF911F910F91FF90EF90DF9046
:106E1000089500D000D000D0EDB7FEB731962CE633
:106E20003BE0ADB7BEB712963C932E931197938378
:106E30008283758364830E9498648DB79EB706969B
:106E40000FB6F8949EBF0FBE8DBF08950F931F938A
:106E5000CF93DF93CDB7DEB7A0970FB6F894DEBF20
:106E60000FBECDBF82E290E00E94D865082F282F88
:106E70002B50203108F0982F9095891709F46DC098
:106E800000D082E99BE0ADB7BEB712969C938E937B
:106E900011970E9498648E010F5F1F4F0F900F9003
:106EA000D80180E090E0FC01E657F44FE491ED93C7
:106EB000019688309105B9F7F894CE0101966EE3FA
:106EC00070E048E050E00E94DE65D80180E090E08C
:106ED000FC01E458F44FE491ED9301968E30910556
:106EE000B9F7CE01019660E370E04EE050E00E94F9
:106EF000DE6580E090E0FC01EE58F44FE491D801AB
:106F0000ED938D0101968A309105A9F7CE01019686
:106F100066E270E04AE050E00E94DE6580E290E0C8
:106F20006DEC7BEA0E94F6658EE190E060E070E037
:106F30000E94F6658DE190E060E00E94E86584E2E1
:106F400090E060E070E00E94F6650AE182E290E085
:106F50006AE175EE0E94F6657894802FA0960FB6D0
:106F6000F894DEBF0FBECDBFDF91CF911F910F917F
:106F70000895F8946EE370E042E050E00E94C0652E
:106F8000789480E0089580E290E00E94D8650895AA
:106F90008EE190E00E94D86508958DE190E00E9416
:106FA000D065089540914020509141206091422049
:106FB0007091432090E0A0E0B0E0480F591F6A1F95
:106FC0007B1F409340205093412060934220709358
:106FD000432040913C2050913D2060913E20709193
:106FE0003F20480F591F6A1F7B1F40933C2050933E
:106FF0003D2060933E2070933F202091E02122238A
:10700000A1F0409138205091392060913A20709140
:107010003B20480F591F6A1F7B1F40933820509315
:10702000392060933A2070933B2008951F920F926D
:107030000FB60F920BB60F9211242F933F934F93DD
:107040005F936F937F938F939F93AF93BF93EF93D0
:10705000FF9380912B0B90912C0B019690932C0B0E
:1070600080932B0B80912A0B8F5F80932A0B8038A3
:10707000A9F410922A0B8091402090914120A09178
:107080004220B09143200196A11DB11D8093402064
:1070900090934120A0934220B09343208091E0211F
:1070A0008823E1F08091290B8F5F8093290B803832
:1070B000A9F41092290B8091382090913920A09149
:1070C0003A20B0913B200196A11DB11D809338203C
:1070D00090933920A0933A20B0933B200E94C22D78
:1070E000009711F00E94C92CFF91EF91BF91AF91D1
:1070F0009F918F917F916F915F914F913F912F91D0
:107100000F900BBE0F900FBE0F901F901895F89424
:107110001092B60016BC83EF87BD82E084BD94E078
:1071200095BD95B395BB80936E007894089580913A
:107130002B0B90912C0B20912B0B30912C0B821749
:107140009307A9F7089507C022E330E0000021501B
:107150003040E1F701970097B9F708950F931F9317
:10716000CF93DF938C010E949738EC010E949738EF
:107170008C1B9D0B80179107C8F3DF91CF911F9156
:107180000F91089508950F931F930091402010913F
:1071900041202091422030914320809140209091C5
:1071A0004120A0914220B0914320081719072A07D7
:1071B0003B0759F7B801C9011F910F9108951F921C
:1071C0000F920FB60F9211241092F1040F900FBE80
:1071D0000F901F9018951F920F920FB60F920BB63B
:1071E0000F9211242F933F934F935F936F937F934D
:1071F0008F939F93AF93BF93EF93FF93E091E70437
:10720000F091E8048081E091F204F091F30430976A
:1072100009F00995FF91EF91BF91AF919F918F91E7
:107220007F916F915F914F913F912F910F900BBE86
:107230000F900FBE0F901F9018951F920F920FB6D0
:107240000F9211241092FE040F900FBE0F901F900A
:1072500018951F920F920FB60F920BB60F92112432
:107260002F933F934F935F936F937F938F939F934E
:10727000AF93BF93EF93FF93E091F404F091F50483
:107280008081E091FF04F0910005309709F00995A5
:10729000FF91EF91BF91AF919F918F917F916F91EE
:1072A0005F914F913F912F910F900BBE0F900FBEAA
:1072B0000F901F90189590E02DE030E0829FF00134
:1072C000839FF00D929FF00D1124E951FB4FA28195
:1072D000B3811C92A481B5816C93A681B78188ED9E
:1072E0008C93A085B1854C931286148613860895DD
:1072F00090E02DE030E0829FF001839FF00D929F9F
:10730000F00D1124E951FB4F81E08287A081B1810A
:107310006C933A9680818823E9F70895CF93C82F1C
:107320008A3031F480916D0B6DE00E94783902C093
:107330008D3029F080916D0B6C2F0E94783980E0A0
:1073400090E0CF9108951F93CF93DF93182FEB0117
:107350000CC08A3021F4812F6DE00E947839699148
:107360006D3019F0812F0E9478398881882389F740
:10737000DF91CF911F9108950F931F93CF93DF93C8
:10738000CDB7DEB79E01265F3F4F0DE21BE0C8017F
:1073900060E470E0488559850E942A658F81B801B4
:1073A0000E94A339DF91CF911F910F9108951F93F0
:1073B000CF93DF93182FEB0104C0812F0E947839FF
:1073C0002196FE0164916623C1F7DF91CF911F9151
:1073D000089590E02DE030E0829FF001839FF00D52
:1073E000929FF00D1124E951FB4F74876387089534
:1073F000682F80E00E947839089580936D0B81E0BA
:1074000095E09093AD288093AC28089584B7877F4A
:1074100084BF88E10FB6F8948093600010926000FA
:107420000FBE08952FE088E190E00FB6F894A8957C
:10743000809360000FBE209360000895A895089582
:1074400088E10FB6F89480936000109260000FBE40
:107450000895F89428E088E190E00FB6F894A89594
:10746000809360000FBE20936000FFCF80914B207F
:1074700080914B2090E008958091390181FD10C0EA
:1074800081E491E06FE140E00E941740813059F0C3
:1074900021E030E0813111F020E030E0C9010895B1
:1074A00080E090E0089581E090E0089581E491E02B
:1074B0006FE140E00E9417400895E9E3F1E0808128
:1074C00080818D7F80838DE090E00197F1F782E4E9
:1074D00091E06FE140E023E00E94214083E090E0F2
:1074E0000197F1F708959091390191FD0AC0282F75
:1074F000803108F02FE085E491E06FE040E00E94E9
:10750000214008958091390181FD13C081E491E00B
:107510006FE140E00E941740982F8151823038F08F
:107520009F3129F0913019F081E0923019F480E018
:10753000089581E008950E94823A8823E1F3089536
:10754000CF93DF93C82F883049F0863039F08930E7
:1075500029F0863119F0893109F045C0809139014F
:1075600081FD44C00E949B3A0E94563AD82FC8170A
:10757000B9F1C83019F40E945D3A2BC0C93141F409
:107580008631A9F482E491E06FE140E029E009C08E
:10759000C63169F4893159F482E491E06FE140E049
:1075A00026E00E942140E3E0F0E03197F1F782E429
:1075B00091E06FE140E02C2F0E942140D83029F467
:1075C00089E691E00197F1F704C0E3E0F0E031973C
:1075D000F1F70E94563A8C1719F083E490E008C046
:1075E00080E490E005C082E490E002C084E490E092
:1075F000DF91CF91089580919400909195009093A0
:1076000079228093782221E02093652280913901AC
:1076100081FF15C02093DF21809194009091950007
:107620009093752280937422209363228091390174
:107630008D7F809339018091DF218823E1F786E1F6
:107640000E94A03A81E08093E02108958091E0219A
:10765000882351F480916F0B882321F081E080937F
:10766000F10B02C00E94FB3A81E090E008950E9475
:107670009B3A1092E0210E945D3A8091390182602C
:1076800080933901809163228823E9F180919400ED
:107690009091950020917422309175228217930762
:1076A000A0F48091402290914122A0914222B09179
:1076B00043228C57914EAF4FBF4F809340229093FF
:1076C0004122A0934222B093432280919400909152
:1076D0009500821B930BA0E0B0E0409140225091B6
:1076E00041226091422270914322840F951FA61F70
:1076F000B71F8093402290934122A0934222B093DF
:10770000432210926322809165228823E9F18091BF
:1077100094009091950020917822309179228217DF
:107720009307A0F48091482290914922A0914A2287
:10773000B0914B228C57914EAF4FBF4F8093482250
:1077400090934922A0934A22B0934B2280919400B7
:1077500090919500821B930BA0E0B0E040914822ED
:107760005091492260914A2270914B22840F951FBB
:10777000A61FB71F8093482290934922A0934A22C4
:10778000B0934B221092652208958091F10B8823CB
:1077900021F00E94FB3A1092F10B8091F20B8823AA
:1077A00021F00E94373B1092F20B10926F0B08955C
:1077B0000F931F93CF93DF93F82FE92FAB0181E055
:1077C00080936F0B00912422109125222091262274
:1077D000309127220F5F1F4F2F4F3F4F00932422DE
:1077E000109325222093262230932722862F8E5F06
:1077F00087FF0CC08091DD219091DE21019690934E
:10780000DE218093DD21CFEFDFEF09C020E73BE0F1
:10781000C9016F2F7E2F0E940764C0E0D0E00E9454
:10782000C53BCE01DF91CF911F910F9108958091BB
:10783000E021882399F080916F0B882321F40E9426
:10784000823A882331F481E08093F20B81E090E06A
:1078500008950E94373B80E090E0089580E090E03A
:1078600008951F93CF93DF930F92CDB7DEB78FB7F5
:10787000898380916F0B882331F5F8948091E02102
:10788000882351F08091390181FD1BC00E94823A0A
:107890008823B9F080E003C00E94263B81E09091EC
:1078A00047019E3010F010E001C01FEF882311F057
:1078B0000E94173C16FF05C089818FBF81E090E0D0
:1078C00004C089818FBF80E090E00F90DF91CF915D
:1078D0001F91089580936E0B08950E94563A82502E
:1078E000813130F4E82FF0E0E65CFA4F80810895B2
:1078F00081E0089508958FEF80934E018CE691E02A
:1079000060EF44E022E00E9421408CE290E06EE0D3
:1079100041E025E00E94214080E880936F01809142
:10792000460180936D0184E491E060E245E021E04E
:107930000E9421400895CF93DF93CDEFD3E0CE0195
:107940000197F1F70E940D40109254201092D6201A
:10795000109258211092532010925220E9E3F1E046
:1079600080818E7F808380818D7F80838DE090E019
:107970000197F1F780818160808382E491E06FE17B
:1079800040E023E00E9421402197F1F780915D01C2
:1079900080915E010E947B3C8CE195E060E070E0AC
:1079A0000E941D2B0E94FB3A81E090E0DF91CF9175
:1079B00008958091F30B0895CF93DF930F92CDB785
:1079C000DEB789830E949B3A29812093F30B88E4D8
:1079D00091E06FE140E00E9421400F90DF91CF9154
:1079E00008950E94DC3C86E00E94A03A0895FA01C6
:1079F00080936201909363016093600170936101D1
:107A00003097C1F0808180936B01818180936A01FE
:107A1000828180936901838180936801848180934E
:107A200067018581809366018681809365018781E6
:107A30008093640108958CE195E00E943F2B81E0E2
:107A400080934B2080914C2090914D2001969093F3
:107A50004D2080934C2081E090E00895CF93DF93F8
:107A600050915320252F30E0F901EE0FFF1F36957E
:107A7000322F222737952795E20FF31FEC5AFF4D3F
:107A80004081442309F4F4C02091390121FDF0C064
:107A90002091E021222309F4EBC047FF23C0852F6A
:107AA00090E0FC01EE0FFF1F9695982F8827979581
:107AB0008795E80FF91FEC5AFF4D10828091142230
:107AC00090911522A0911622B09117220196A11D26
:107AD000B11D8093142290931522A0931622B09387
:107AE0001722C6C0433018F5852F90E0FC01EE0F39
:107AF000FF1F9695982F882797958795E80FF91F70
:107B0000EC5AFF4D10828091102290911122A09189
:107B10001222B09113220196A11DB11D8093102253
:107B200090931122A0931222B0931322A1C0C42FCC
:107B3000D0E022976C177D0718F5852F90E0FC01A7
:107B4000EE0FFF1F9695982F882797958795E80F3A
:107B5000F91FEC5AFF4D108280910C2290910D225A
:107B6000A0910E22B0910F220196A11DB11D80930C
:107B70000C2290930D22A0930E22B0930F2278C076
:107B8000252F30E0B901660F771F3695322F222757
:107B900037952795620F731F6B5A7F4D50E00E94F7
:107BA000076420915320822F90E0FC01EE0FFF1F0D
:107BB0009695982F882797958795E80FF91FEC528F
:107BC000FF4D808180934420822F90E0FC01EE0FD6
:107BD000FF1F9695982F882797958795E80FF91F8F
:107BE000EC5AFF4D10822F5F20935320233010F06A
:107BF000109253208091532090E0FC01EE0FFF1F64
:107C00009695982F882797958795E80FF91FEC5A36
:107C1000FF4D8081882311F00E941B3D6091470138
:107C20006093452080914A20882311F0681710F452
:107C300060934A2084E070E00E945C3160914420AF
:107C400083E070E00E945C3180912822909129228B
:107C5000A0912A22B0912B220196A11DB11D8093E3
:107C6000282290932922A0932A22B0932B2202C08B
:107C7000C0E0D0E0CE01DF91CF910895CF93DF93A4
:107C8000EC0188819981009729F024E08B3F9207CD
:107C900039F505C08BEF94E09983888325C062385D
:107CA00019F510924B200E94E2300E94433060E8A8
:107CB00070E00E942E3D1816190644F40E943E30D2
:107CC000E091AD05F091AE050995E4CF8091482093
:107CD0009091492001969093492080934820DACFD3
:107CE0001982188283E001C081E0DF91CF9108956D
:107CF00091E090936F0B0E94733A0E94C53B0895E8
:107D00008091390181FD07C085E491E06FE040E09A
:107D10000E941740089580E108950F931F93CF9319
:107D2000DF93C82F21E020936F0BD091E021809149
:107D3000390181FF16C08091940090919500909335
:107D4000752280937422209363222093DF218091F7
:107D500039018D7F809339018091DF218823E1F7FC
:107D6000D0E00E949B3A8091E021882309F441C031
:107D7000809165228823E9F180919400909195008B
:107D8000209178223091792282179307A0F4809174
:107D9000482290914922A0914A22B0914B228C57BF
:107DA000914EAF4FBF4F8093482290934922A093AA
:107DB0004A22B0934B228091940090919500821BAF
:107DC000930BA0E0B0E0409148225091492260918D
:107DD0004A2270914B22840F951FA61FB71F8093D4
:107DE000482290934922A0934A22B0934B221092AA
:107DF000652289E10E94A03A86E00E9467310097DF
:107E000051F00E94803E082F86E00E946731815029
:107E10000E94733A02C000E010E0809194009091BB
:107E20009500909377228093762281E0809364225C
:107E3000F8948091390182608093390180913901F1
:107E40008D7F809339016C2F6E5F80E79BE00E94ED
:107E5000524078948091DA219091DB2101969093A1
:107E6000DB218093DA210E949B3A82E491E060EE6C
:107E700045E00E941740C82F86E00E9467310097B6
:107E800019F0802F0E94733ADD2319F00E94FB3A0B
:107E900002C00E94373B809164228823E9F18091DF
:107EA000940090919500209176223091772282174C
:107EB0009307A0F48091442290914522A0914622FC
:107EC000B09147228C57914EAF4FBF4F80934422C1
:107ED00090934522A0934622B0934722809194002C
:107EE00090919500821B930BA0E0B0E0409144225A
:107EF000509145226091462270914722840F951F30
:107F0000A61FB71F8093442290934522A093462238
:107F1000B0934722109264228091E021882361F07F
:107F2000809194009091950090937922809378228B
:107F300081E08093652207C082E491E06FE140E038
:107F400023E00E9421400E94C53BC130E1F0C330D4
:107F5000A9F480911C2290911D22A0911E22B09123
:107F60001F220196A11DB11D80931C2290931D22FA
:107F7000A0931E22B0931F22C2E00AC0C53029F090
:107F8000C73031F404C0C0E003C0C3E001C0C1E0A9
:107F90008C2F90E0DF91CF911F910F910895CF9397
:107FA000DF93EB010E94D83B009729F4CE010E9499
:107FB0008D3E009751F02091DD213091DE212F5F21
:107FC0003F4F3093DE212093DD21DF91CF91089543
:107FD000CF93DF938091E021882321F40E94263BF8
:107FE000C1E001C0C0E00E94563A863111F08131F3
:107FF00019F4D091470109C086E491E06FE140E0B7
:108000000E941740D82FDD0FD80FCC2311F00E940B
:10801000173C8D2FDF91CF9108951092F50B1092A0
:10802000F40BEFE6F0E08081806280830895FC012C
:108030008081862390E002C0959587954A95E2F766
:108040000895F894FC019081862F8095892330E073
:1080500002C0220F331F4A95E2F72623282B2083E4
:1080600078940895CF93DF93EC012196E0917B0102
:10807000DC01EC932E2FA0E8B1E03D913993215023
:10808000E1F7E150F0E0E058FE4F2181FC01E058BB
:10809000FF4F20838F579F4F21E0FC012083DF910A
:1080A000CF910895FC0160938001A1E8B1E061588F
:1080B00081918D936A17E1F708951F920F920FB681
:1080C0000F920BB60F9211242F933F934F935F9310
:1080D0006F937F938F939F93AF93BF93EF93FF9390
:1080E00080914701809345202091522030E0C901C2
:1080F000880F991F3695322F222737952795820FA3
:10810000931F8C5A9F4D0E943240809152208F5F66
:1081100080935220833010F0109252200E941B3D19
:10812000FF91EF91BF91AF919F918F917F916F914F
:108130005F914F913F912F910F900BBE0F900FBE0B
:108140000F901F9018951F920F920FB60F92112447
:108150000F900FBE0F901F9018951F920F920FB6A1
:108160000F9211240F900FBE0F901F9018951F9221
:108170000F920FB60F9211240F900FBE0F901F9009
:1081800018951F920F920FB60F9211241092DF21B3
:108190000F900FBE0F901F9018951F920F920FB661
:1081A0000F9211241092DF210F900FBE0F901F909D
:1081B00018951F920F920FB60F9211248F9381E0A2
:1081C00080934B208F910F900FBE0F901F901895AA
:1081D0001F920F920FB60F9211241092DF210F9071
:1081E0000FBE0F901F9018951F920F920FB60F920F
:1081F00011248F939F938091F40B9091F50B01962E
:108200009093F50B8093F40B9F918F910F900FBE7D
:108210000F901F9018950F931F93CF93DF9380912A
:10822000E8219091E921A091EA21B091EB210196FA
:10823000A11DB11D8093E8219093E921A093EA212B
:10824000B093EB210E94A3438C0186EF9BE00E9438
:10825000E72B08C0EA81FB81309709F00995CE0130
:108260000E948D2CEC010097A9F70115110519F05A
:10827000C8010E945529DF91CF911F910F91089558
:108280000E94F9490E94E2300E94BC418EE895E0CC
:108290009093E3218093E2210E94A04382E090E04A
:1082A00060E074E040E05EE12FEF31E00E94614366
:1082B0000895CF92DF92EF92FF920F931F93CF9387
:1082C000DF936C018B017A0186EF9BE00E94E72B24
:1082D00009C0EC81FD81309711F0C8010995CE01EC
:1082E0000E948D2CEC010097A1F7C601B801A701EF
:1082F0000E945F29DF91CF911F910F91FF90EF9026
:10830000DF90CF900895BC0186EF9BE00E94562C31
:108310000895BC0186EF9BE00E94212C0895CF9325
:10832000DF93EC018091E4219091E521A091E62179
:10833000B091E7210196A11DB11D8093E421909396
:10834000E521A093E621B093E721CE010E94B64338
:10835000009769F00E945D30E0919205F0919305DD
:1083600089E591E4BE01099581E090E002C080E0DA
:1083700090E0DF91CF91089588EF9BE00E94E32B7E
:1083800008950F93CF93DF93EC017B836A83188664
:108390005F834E8388EF9BE0BE010E94562CE091E4
:1083A000FA0BF091FB0B309749F04C815D818A818B
:1083B0009B81688520E030E001E00995DF91CF9155
:1083C0000F910895BC0188EF9BE00E94212C089535
:1083D0000F93DC0118961C921897E091FA0BF0911C
:1083E000FB0B309759F012968D919C91139760E09A
:1083F00040E050E020E030E000E009950F91089562
:108400000F93DC01AB0114962D913C91159781E0FF
:1084100018968C93189715967C936E931497E09109
:10842000FA0BF091FB0B309739F012968D919C91DD
:10843000139761E000E009950F9108950F93DC0117
:10844000E091FA0BF091FB0B309769F014962D91A7
:108450003C91159712968D919C91139718966C915B
:10846000A90101E009950F910895E091FC0BF091AD
:10847000FD0B309709F0099508959093FD0B8093BB
:10848000FC0B08959093FB0B8093FA0B089588EFF3
:108490009BE00E94E72B0895EF92FF920F931F93AA
:1084A000CF93DF938C01EB017A0188EF9BE00E9470
:1084B000E72B15C0DC0112962D913C9113972C17D8
:1084C0003D0759F41696ED91FC911797309749F0B6
:1084D000B801AE019701099504C00E948D2C009748
:1084E00049F7DF91CF911F910F91FF90EF90089581
:1084F0000895AF92BF92CF92DF92EF92FF920F93C7
:108500001F93CF93DF9300D0CDB7DEB75B010E94FE
:108510004330FC01E080F180FA82E982FCE0EF1652
:10852000F10418F400E010E02DC000D000D086E582
:1085300095E0EDB7FEB792838183F482E3820E94D7
:1085400086640F900F900F900F901FC00E944330D1
:10855000F801EE0FFF1FEE0FFF1FE80FF91FC2809B
:10856000D3800E9443300F5F1F4FF801EE0FFF1FB3
:10857000EE0FFF1FE80FF91F40815181C501B601C1
:108580000E944C420E151F0509F70F900F90DF91C6
:10859000CF911F910F91FF90EF90DF90CF90BF9000
:1085A000AF900895CF93DF93C9E1DCE060912F0C89
:1085B0007091300CCE0145EF52E420E030E00E9493
:1085C00056480E94F64960912F0C7091300C0E9421
:1085D000CF60BC01CE01409749E153E420E030E098
:1085E0000E945648DF91CF91089580912F0C909171
:1085F000300C20912D0C30912E0C880F991F2817CC
:10860000390708F4C9019093300C80932F0C0E9415
:10861000D24208950F93013051F48091290C90912A
:108620002A0C9093300C80932F0C0E94D2420F9111
:108630000895CF93DF930E94E2300E944330EC0113
:10864000198218820E94474220C012962D913C91B7
:108650001397FC01EE0FFF1FEE0FFF1FEC0FFD1F26
:108660003383228314962D913C9115970196FC013A
:10867000EE0FFF1FEE0FFF1FEC0FFD1F3183208356
:1086800099838883CD010E948D2CDC01888199819A
:10869000109729F018962C9118972223B1F6880F7D
:1086A000991F880F991F02960E943E3088819981F8
:1086B000009721F08EEF9BE00E942829DF91CF9157
:1086C0000895EF92FF920F931F93CF93DF93FC01D6
:1086D0008B017A01E9018EEF9BE0BF0143E755E092
:1086E0000E940A2910932A0C0093290CF0922C0C5A
:1086F000E0922B0CD0932E0CC0932D0C8AE093E4C7
:108700000E944242DF91CF911F910F91FF90EF9015
:108710000895CF93DF93C9E1DCE0CE010E94DD48EC
:10872000CE0140970E94DD48CE014B970E9425293B
:10873000DF91CF91089580912F0C9091300C089586
:108740000E946B290895CF93DF93E0917705F09114
:1087500078050995EC01009729F06A817B8181E019
:108760000E945C31CE01DF91CF9108950F931F934A
:10877000CF93DF93EC01E0917905F0917A050995AB
:108780008C016A817B8181E00E945C3181E090E014
:108790000115110511F480E090E0DF91CF911F9158
:1087A0000F910895E0917B05F0917C05099508955E
:1087B0009C0180E090E005C0F90131974081840F71
:1087C000911D2E5F3F4FF901329740814423A1F75D
:1087D0000895FC01308120E0818190E0822B932B71
:1087E00002C0880F991F6A95E2F7892F9927FA012D
:1087F000E358FA4F208130E08223932328E030E0D1
:10880000241B350B02C0969587952A95E2F70895AB
:108810006F927F928F929F92AF92BF92CF92DF9290
:10882000EF92FF920F931F93CF93DF935C013B0175
:108830008A0169012830310544F4CB01BA01A9014C
:108840000E94E943F50180834EC0790173E0F594FD
:10885000E7947A95E1F74115510521F04501C0E013
:10886000D0E005C0F301D50180E090E021C0C30154
:108870008C0F9D1FB80148E050E00E94E943F401CD
:1088800081934F012196CE15DF058CF3C701F7FECA
:1088900002C080E090E0A60147705070411551057C
:1088A00011F1E501C80FD91F860D971DB80118C039
:1088B00021912D9301968E159F05D4F3C701F7FEE4
:1088C00002C080E090E0A60147705070411551054C
:1088D00051F0E501C80FD91F860D971D60E070E0CB
:1088E0000E94E9438883DF91CF911F910F91FF9000
:1088F000EF90DF90CF90BF90AF909F908F907F9040
:108900006F9008958F929F92AF92BF92CF92DF9215
:10891000EF92FF920F931F93CF93DF9300D000D07D
:10892000CDB7DEB70E9443308C0182E090E00E9418
:108930002030009709F45FC0F801918180E0208128
:10894000820F911D0E947F297C01009709F455C078
:108950000E9443304C01F7018681482F4695469589
:10896000469550E090E08770907021E030E00097ED
:1089700011F420E030E0CA01820F931F0E942030E2
:108980000097C9F1F70104811581CC24DD242EC0A4
:10899000F801A180BB24B601A3E075956795AA955F
:1089A000E1F7680D791DA60147705070883168F0B5
:1089B000CE01039695010E940844F8018081BE0112
:1089C0006D5F7F4F0E9470310DC01A821982CE01F7
:1089D000019695010E94084469817A81F80180819D
:1089E0000E945C31CA0CDB1C0E5F1F4FF8018081B6
:1089F000882371F602C0EE24FF24C7010F900F9068
:108A00000F900F90DF91CF911F910F91FF90EF90FA
:108A1000DF90CF90BF90AF909F908F900895FC0112
:108A200050E080E190E0861B970B821B930B02C005
:108A3000440F551F8A95E2F78081852B80838181C1
:108A4000842B818308956F927F928F929F92AF9231
:108A5000BF92CF92DF92EF92FF920F931F93CF932B
:108A6000DF933C016B015A0179012830310524F470
:108A7000C301FA01408159C08901B3E015950795FA
:108A8000BA95E1F76115710521F04A01C0E0D0E027
:108A900005C0FA01D30180E090E023C0F4014191C8
:108AA0004F01C3018C0F9D1FB60128E030E00E94EA
:108AB0000F452196C017D1078CF3980117FF02C00C
:108AC00020E030E0D701A770B070109781F1F50178
:108AD000E20FF31F408150E0C6018A1B9B0B0896F2
:108AE00019C021912D93019680179107D4F3980115
:108AF00017FF02C020E030E0D701A770B0701097D8
:108B0000B1F0F501E20FF31F408150E088E090E002
:108B10008A1B9B0B02C0559547958A95E2F7C301C6
:108B2000820F931F60E070E09D010E940F45DF916E
:108B3000CF911F910F91FF90EF90DF90CF90BF905A
:108B4000AF909F908F907F906F9008956F927F92DB
:108B50008F929F92AF92BF92CF92DF92EF92FF924D
:108B60000F931F93CF93DF9300D0CDB7DEB77C0177
:108B7000DC0116968C911697282F2695269526951A
:108B800030E090E08770907001E010E0009711F401
:108B900000E010E0020F131FC80102960E94A830E7
:108BA000009709F451C00E944A30FC01D701129687
:108BB0008C911297808313968C9181830E944A3006
:108BC00032E0632E712C680E791EC30160E070E004
:108BD000A8010E941064F701E480F580CC24DD2414
:108BE0002CC0D7011196AC901197BB24860193E05D
:108BF000159507959A95E1F7060D171D27E0822E2A
:108C0000912C8C209D20883130F00E947A31AC016B
:108C1000C801B40109C00E9467319A838983C801E1
:108C2000B401AE014F5F5F4F95010E942345CA0C0E
:108C3000DB1CE2E0F0E0EE0EFF1ED7018C918823F2
:108C400081F681E090E002C080E090E00F900F900C
:108C5000DF91CF911F910F91FF90EF90DF90CF9018
:108C6000BF90AF909F908F907F906F900895E0910C
:108C7000AB05F091AC0509950895E0915405F0918C
:108C8000550509950895E091AF05F091B005099556
:108C90000895E091B105F091B2050995089580E03D
:108CA00090E008950895E0913605F0913705099513
:108CB000089580E090E008950F931F93CF93DF9382
:108CC000CDB7DEB7E0970FB6F894DEBF0FBECDBFCD
:108CD0000E9493308C010E944330602FAE014F5FA1
:108CE0005F4F0E94864F882309F446C088A99801E7
:108CF000281B3109C9010E9420300097E9F12E811B
:108D0000222379F18A859B853BEA8D3C930721F0EC
:108D10003FEF8F3F930781F5223069F088E090E0C4
:108D20000197E1E0F0E0EC0FFD1FE80FF91F23854C
:108D30002F3F21F007C082E090E0F2CF181619060D
:108D40007CF30FC089E1BE01645F7F4F0E947031E8
:108D500089E10E947A3161EF7FE10E94C228009789
:108D600059F088E1BE016A5E7F4F0E947031E09148
:108D70009405F09195050995E0960FB6F894DEBF3D
:108D80000FBECDBFDF91CF911F910F910895AF928C
:108D9000BF92CF92DF92EF92FF920F931F93CF93E8
:108DA000DF93CDB7DEB7E0970FB6F894DEBF0FBE06
:108DB000CDBF5C016B01FE01319680E3DF011D92A6
:108DC0008A95E9F781E089838CE00E9467318C8382
:108DD0001D821F828091330C89878F5F8093330CB3
:108DE00003E008878DEC9BEA9B878A8789E10E94D4
:108DF0007A3161EB74E00E94C228009731F082E082
:108E00008E838FEF8C878D8709C089E10E947A312C
:108E1000BC01CE010C960E94B9280E838DEC9BEA12
:108E20009D8B8C8BCE01469661EF7FE10E94B92825
:108E30000E9443309FA78EA70E94933088ABCE013B
:108E400001960E94974E082F90E00E94A83000974C
:108E500049F10E944A30BC01CE010196402F0E9488
:108E6000B54E00912C0510912D050E944A307C01D1
:108E70000E949D30BC01C701F8010995A114B104FD
:108E800089F0009721F08130910561F404C0C6019A
:108E900060E070E003C0C60164E070E041E050E0D3
:108EA000F5010995E0960FB6F894DEBF0FBECDBF71
:108EB000DF91CF911F910F91FF90EF90DF90CF90B6
:108EC000BF90AF9008950E94F6498093330CE091D3
:108ED0003605F091370509950895009731F0E09136
:108EE0003605F091370509950895E0913805F09120
:108EF000390509950895CF93DF93EC0104C060E034
:108F000070E00E941D2B899199910097C1F7DF9124
:108F1000CF910895CF93DF93EC0102C00E94642AA1
:108F2000899199910097D1F7DF91CF910895CF93CF
:108F3000DF93EC017B836A830E949738998388834F
:108F4000DF91CF910895FC0180819181228133814D
:108F5000820F931F918380830895CF93DF93EC0159
:108F60000E94973899838883DF91CF910895CF939A
:108F7000DF93EC010E94973828813981AC01421BB4
:108F8000530B9A012F5F3F4F81E090E04A815B8154
:108F90004217530710F080E090E0DF91CF910895E1
:108FA000CF93DF93FC01C281D38180819181C80F6F
:108FB000D91F0E9497389E01281B390BC901DF91E8
:108FC000CF910895EF92FF920F931F93CF93DF936A
:108FD0007C018A01FC0180819181009729F08B340A
:108FE000910509F049C01AC085E39CE00E94E72B77
:108FF000EC0109C06C817D81CE0102960E947F2D1B
:109000000990D881C02D2097A9F781E08093340C76
:109010008BE490E0F7019183808333C0683889F551
:1090200085E39CE00E94E72BEC0123C0CE01029671
:1090300008171907D9F485E39CE0BE010E94212C92
:109040000091BC091091BD098A859B859093BD094B
:109050008093BC09EC85FD85309719F08E859F853E
:1090600009951093BD090093BC09D2CF0990D8810E
:10907000C02D2097D9F6CCCFF7011182108283E062
:1090800001C081E0DF91CF911F910F91FF90EF9090
:1090900008951092340C85E39CE00E94E32B84EC4D
:1090A00095E060E070E00E941D2B08950F931F93E0
:1090B000CF93DF93EC010091BC091091BD091B8790
:1090C0000A875D874C873F872E878091340C8823E1
:1090D00079F084EC95E09093BD098093BC09CE01B2
:1090E00002960E947F2D1093BD090093BC0902C017
:1090F0007D836C8385E39CE0BE010E94212C85E387
:109100009CE0BE010E94562CDF91CF911F910F91E0
:1091100008950F931F93CF93DF93EC018091340C4C
:10912000882391F00091BC091091BD0984EC95E071
:109130009093BD098093BC09CE0102960E948A2DAE
:109140001093BD090093BC0985E39CE0BE010E9419
:10915000212C85E39CE0BE010E94562CDF91CF912B
:109160001F910F9108950F931F93CF93DF93EC01FD
:109170008091340C882391F00091BC091091BD09B5
:1091800084EC95E09093BD098093BC09CE010296D2
:109190000E94952D1093BD090093BC0985E39CE0C6
:1091A000BE010E94212C85E39CE0BE010E94562C4A
:1091B000DF91CF911F910F910895CF93DF93EC0131
:1091C0008091340C882329F0CE0102960E94DC2D78
:1091D00004C01F821E821986188685E39CE0BE01AA
:1091E0000E94212CDF91CF910895CF93DF93EC0162
:1091F0008091340C882329F0CE0102960E94AA2D7A
:1092000012C085E39CE00E94E72B06C08C179D07E7
:1092100041F0FC01808191810097C1F781E090E0ED
:1092200002C080E090E0DF91CF910895CF93DF936B
:10923000EAE6F2E2CCE2D2E2AEE5B2E211921192BB
:1092400019921992199219921D9282E2E238F80746
:10925000A9F7DF91CF9108950F931F93CF93DF93D9
:10926000FC01E25AFD4D20818C01000F111F000FFF
:10927000111F222311F12091940030919500E801F3
:10928000C45DDD4DFC01EE0FFF1FE659FD4D8081F1
:109290009181A901481B590BCA01A0E0B0E04881A7
:1092A00059816A817B81840F951FA61FB71F888310
:1092B0009983AA83BB8331832083F801E45DFD4D4C
:1092C0006081718182819381DF91CF911F910F9194
:1092D000089560E070E080E090E00895FC01EE0FFA
:1092E000FF1FEE0FFF1FE45DFD4D4083518362833E
:1092F00073830895EF92FF920F931F93CF93DF93A1
:10930000BEE5EB2EB2E2FB2EECE2F2E2CAE6D2E2DE
:1093100020E030E0D7018D917D018823C9F00091D4
:1093200094001091950088819981A801481B590BE0
:1093300060E070E080819181A281B381840F951FEC
:10934000A61FB71F80839183A283B38319830883E9
:109350002F5F3F4F349622962C303105D9F6DF919E
:10936000CF911F910F91FF90EF9008950E94194E99
:1093700008950F931F93FC018091370C9091380C46
:10938000338322831583048371836083F093380CC5
:10939000E093370C009719F4CB010E94334E80E024
:1093A00090E01F910F9108958091370C9091380CA7
:1093B0000097C1F01092380C1092370CDC01149613
:1093C0006D917C9115971296ED91FC9113970995EB
:1093D000E091370CF091380C309721F08081918129
:1093E0000E94334E08950E94A96108950E94A461CD
:1093F00008958EEC95E00E94552B86ED95E00E9435
:10940000552B0895CF93DF930E9450300097A9F019
:1094100086ED95E00E94742BEC01009729F10E94E3
:109420009330998388830E948E309B838A83CE01F8
:1094300004960E94CA2F8CAB17C08EEC95E00E9458
:10944000742BEC01009771F002960E94DC2F998337
:109450008883BE016E547F4FCE018E579F4F0E946E
:109460003A3102C0C0E0D0E0CE01DF91CF91089543
:10947000BC016E547F4F8E579F4F0E943A31089522
:10948000CF93DF93EC018EEC95E0BE010E94C52BDB
:10949000009719F08EEC95E009C086ED95E0BE01CD
:1094A0000E94C52B009729F086ED95E0BE010E9431
:1094B0009F2BDF91CF910895CF93DF93EC018EEC3A
:1094C00095E0BE010E94C52B009779F068817981F3
:1094D000CE0102960E940B31BE016E547F4FCE0129
:1094E0008E579F4F0E944B311CC086ED95E0BE0108
:1094F0000E94C52B0097A9F00E94E2306881798113
:109500008A819B810E940B318CA990E00E94A83037
:109510000E944A304CA9BE016C5F7F4F50E00E9410
:109520000764DF91CF910895CF93DF93EC018EEC28
:1095300095E0BE010E94C52B009719F0CE0102965E
:109540000CC086ED95E0BE010E94C52B009719F076
:109550008A819B8102C080E090E0DF91CF910895E5
:10956000FC0180819181089570E06F5B7F4F660FF1
:10957000771F680F791FCB010895E62FF0E0EF5BAE
:10958000FF4FEE0FFF1FE80FF91F808191810895B3
:10959000089582E992E10E94AA2D009721F082E9C4
:1095A00092E10E94952D0895E0917D12F0917E1236
:1095B000309711F00995089580E00895EF92FF9299
:1095C0000F931F93CF93DF937C018A01FC0180816D
:1095D0009181009731F0F3E08C309F0709F0FFC0D4
:1095E0002BC080E0E82FF0E0EE0FFF1FEE0FFF1F13
:1095F000E058FD4E118210828F5F843098F3809383
:109600007F128091BC099091BD09E0E8F2E1918B55
:10961000808B0E945D2A8093822282E992E160E43D
:1096200070E00E947F2D0E94FB508CE093E0F701D8
:109630009183808381E0D7C0623009F4B2C0633087
:1096400030F4662309F482C0613079F795C0673839
:1096500019F0683851F73AC010929A12C0E8D2E176
:1096600013C08A819B818017910741F48881998179
:109670000E943152198218821B821A82249680918C
:109680009A128F5F80939A1280919A12843048F3D5
:10969000E2E9F7E2848D958D8017910719F4158E14
:1096A000148E118EB09628E2E231F20798F3E8E2C8
:1096B000F8E2818592858017910711F41582148252
:1096C0003D9688E2EA3AF807A0F3AFCFE2E14239EB
:1096D0005E0709F0AACFCA010E94AA2D009709F4DB
:1096E000A4CF10929A122DC0F0E035E0EE0FFF1FCC
:1096F0003A95E1F7EE56F84D818D8823E9F082E93D
:1097000092E10E94952D80919A1290E025E0880FB9
:10971000991F2A95E1F78E56984D90939127809343
:10972000902782E00E94655280918322909184224A
:10973000009711F00E94D44A80919A128F5F809313
:109740009A12E0919A12E43078F26FCF41155105E8
:1097500009F46BCF509391274093902783E00E94A8
:1097600065528091832290918422009711F00E948B
:10977000D44A0E94C94A59CF4115510509F455CF21
:1097800050938D2740938C2785E00E9465528091ED
:10979000832290918422009709F447CF0E94D44AF3
:1097A00044CF8091832290918422009709F43DCF89
:1097B00080919422863031F48091AC2281FF02C0E6
:1097C0000E94C94A81E00E94655280918322909153
:1097D0008422009709F429CF0E94014D26CFF7017A
:1097E0001182108283E0DF91CF911F910F91FF9042
:1097F000EF90089590937E1280937D1208959C01BE
:109800004091BC095091BD0960E0E0E8F2E114C06C
:10981000808191818217930769F4828193818417F3
:10982000950741F460939B1211821082C9010E9436
:109830003152089534966F5F643050F360939B12F9
:10984000089540E0E0E8F2E116C0542F5F5F208108
:1098500031812115310569F440939C1291838083F5
:109860002091BC093091BD09338322830E944B5261
:1098700008953496452F443040F340939C12089548
:10988000FC018091BC099091BD09958F848F778FE1
:10989000668F0895FC018091BC099091BD09928763
:1098A0008187748763870895CF93DF93EA010E94CD
:1098B000BD51009749F02091BC093091BD09FC01D0
:1098C00032872187D487C387DF91CF9108950F9383
:1098D0001F93CF93DF9300D000D0CDB7DEB78C01BC
:1098E000AB018FEF89838A838B838C83CE010196B2
:1098F000B8010E94544C009719F0FC0115830483B1
:109900000F900F900F900F90DF91CF911F910F91BB
:1099100008958BEE95E062E040E050E00E940E2B4F
:1099200010928422109283220895AC018BEE95E070
:1099300061E00E94EB2A0895AC018BEE95E060E0B7
:109940000E94EB2A08950F931F93CF93DF938A0110
:109950000E943151EC01009759F08091BC0990911F
:10996000BD099D8F8C8F1F8F0E8FCE010E949C4C46
:10997000CE01DF91CF911F910F910895CF93DF9387
:10998000A0919027B0919127109719F0ED016C9656
:1099900005C0C0918C27D0918D27299680918B2767
:1099A00086FF22C010929D1240E0E0E8F2E116C06E
:1099B0008081918114962D913C9115978217930780
:1099C00059F482819381009739F040939D129983D5
:1099D00088831B821A8206C034964F5F443040F35E
:1099E00040939D120E94C94A88819981009731F065
:1099F0004A815B81609182220E940E2BDF91CF9180
:109A000008950F931F93CF93DF9380919422863014
:109A100009F074C0809183229091842225E08030E7
:109A2000920709F06BC0C4E9D2E0D0938422C093BE
:109A3000832202E000938D2214E910938E2210926B
:109A4000B0221092AF220E94F3508095909590938F
:109A5000B0228093AF2210929622109295220E94FB
:109A6000E2508095909590939622809395220E9443
:109A7000D44AD0938422C093832200938D221093E2
:109A80008E2290918E2780918F27E92FF82FDF016A
:109A9000A459BD4F8CE692E00D9001920197E1F739
:109AA00083EA92E26CE672E00E949F5080918722E6
:109AB0008093A322809188228093A422809189227E
:109AC0008093A52280918A228093A6221092B022B0
:109AD0001092AF220E94F350809590959093B022FF
:109AE0008093AF2210929622109295220E94E2500B
:109AF0008095909590939622809395220E94D44AC7
:109B0000DF91CF911F910F910895FC0120E030E08B
:109B100080E0A8E111C0419198E0542F5827B52F5B
:109B2000B17050FD8A278695B13009F4806846955A
:109B3000915099F72F5F3F4F2617370761F7089528
:109B40001F920F920FB60F920BB60F9211242F9304
:109B50003F934F935F936F937F938F939F93AF93B5
:109B6000BF93EF93FF938091940090919500909311
:109B70006F2280936E2281E0809360228091710039
:109B8000807D809371000E94D44980916022882357
:109B9000E9F1809194009091950020916E2230918E
:109BA0006F2282179307A0F480913422909135227E
:109BB000A0913622B09137228C57914EAF4FBF4FB4
:109BC0008093342290933522A0933622B09337228B
:109BD0008091940090919500821B930BA0E0B0E0DF
:109BE0004091342250913522609136227091372273
:109BF000840F951FA61FB71F8093342290933522A0
:109C0000A0933622B093372210926022FF91EF91F9
:109C1000BF91AF919F918F917F916F915F914F9184
:109C20003F912F910F900BBE0F900FBE0F901F9082
:109C300018959FB7F894E1E7F0E08081807D8083FC
:109C400088B38F6288BB10929000E1E9F0E0108247
:109C5000109292001092950010929400808185607D
:109C600080839FBF08952FB7F894909399008093B5
:109C7000980088B38F6288BBE1E7F0E08081826062
:109C800080832FBF0895CF93DF93FC01DB0185E034
:109C9000EB0119928A95E9F7858190E083709070C5
:109CA000009711F082E08C93878190E08370907030
:109CB000009721F082E012968C931297858190E0B4
:109CC00083709070009799F0878190E08370907016
:109CD000009769F02389348981859285281739078F
:109CE00031F481E0848312961C92129701C0148291
:109CF000C581C370C250C23028F4D0E0CB50DA4FD7
:109D0000888101C080E011968C931197E781E37000
:109D1000E250E23028F4F0E0EB50FA4F808101C0CD
:109D200080E013968C931397DF91CF910895CF9392
:109D3000DF9300D000D00F92CDB7DEB7BE016F5FCA
:109D40007F4F0E94434E89819A81890F8D5F9B814D
:109D5000890F9C81890F9D81890F0F900F900F9023
:109D60000F900F90DF91CF910895DF92EF92FF92C5
:109D70000F931F93CF93DF9300D000D000D0CDB7C7
:109D8000DEB78C017B01BE016F5F7F4F4E830E9467
:109D9000434E79816A81AB81BC81872F90E0039625
:109DA000860F911D8A0F911D8B0F911D2D81820FA2
:109DB000911D4E8150E0481759070CF498C0F801E6
:109DC000218130E02170307083E0220F331F8A95AB
:109DD000E1F7828190E08170907034E0880F991FE4
:109DE0003A95E1F7822B90819770892B438150E05F
:109DF0004170507095E0440F551F9A95E1F7842B00
:109E0000448150E04170507026E0440F551F2A9560
:109E1000E1F7842BF7018083F801258130E023707E
:109E20003070220F331F220F331F868190E0837022
:109E3000907054E0880F991F5A95E1F7822B978113
:109E40009295990F990F907C982BF7019183F801C7
:109E50008085F7018283723051F4F8018185F70122
:109E60008383F8018285F701848355E001C053E0C4
:109E700040E080E090E09801260F311D09C0F90113
:109E8000E80FF91FD384F701E70FF11DD0824F5F70
:109E9000742F750F0197461791F7972FA23089F409
:109EA0009701270F311DF8018389F9018083872FDE
:109EB0008F5F9701280F311DF8018489F901808394
:109EC0009E5F40E020E030E00B0F111D09C0F8015B
:109ED000E20FF31F5589F701E80FF11D50834F5F23
:109EE000842F890F215030404B1789F701C080E043
:109EF00026960FB6F894DEBF0FBECDBFDF91CF918F
:109F00001F910F91FF90EF90DF900895BF92CF9235
:109F1000DF92EF92FF920F931F93CF93DF937C0119
:109F2000B62EEA0182E0861708F0AEC0F701808104
:109F3000D82ED294D694D69463E0D622F1E0DF22D4
:109F4000F7019181292F269526952370C92EC29459
:109F5000C694C69473E0C722382F37703883382FE1
:109F600036953695369531703983382F3295317064
:109F70003A838295869581708B83DC822D83892F2D
:109F8000829583708E83CF8282818887222369F1B4
:109F90003381948180E0830F911D9A8789872230D5
:109FA00079F4CA010B9661EB74E00E94B928F701BD
:109FB00086818B8785818C878701095F1F4F20C031
:109FC00087010B5F1F4F2330D9F4F7013D96DA016B
:109FD00080E092911B969C931B978F5F119688301F
:109FE000C1F78701035F1F4F0BC087010D5F1F4F34
:109FF000CA010B9661EB74E00E94B9281A86198693
:10A00000CC2089F1DD2059F4F8012081918180E094
:10A01000820F911D9C8B8B8B0E5F1F4F04C0898517
:10A020009A859C8B8B8BF2E0CF1671F4CE0145960E
:10A0300061EB74E00E94B928F80181818D8B8081E9
:10A040008E8B0E5F1F4F17C0F3E0CF16A1F4085F91
:10A050001F4FD801FE0180E09E91958B8F5F319656
:10A060008830D1F708C0CE01459661EB74E00E94BC
:10A07000B9281C8A1B8A802F8E199B2D981B9FA79D
:10A080001EA70DA7B81608F480E0DF91CF911F91AD
:10A090000F91FF90EF90DF90CF90BF9008959C01BB
:10A0A00041505040460F571FFB010EC0B081A0E049
:10A0B0008181BD01680F711D260F371F26173707D5
:10A0C00010F42F5F3F4F3296E417F50778F3E4174B
:10A0D000F50749F4908180E0280F391F28173907C8
:10A0E00010F42F5F3F4FC9010895CF93DF93C091C4
:10A0F0008E22D0E0649730918D2220E0C20FD31FD2
:10A100009E01280F311DC90167E972E248E050E065
:10A110000E944F506FE972E2AE010E944F500097CB
:10A1200021F098278927982702C08FEF9FEFDF91B2
:10A13000CF9108959093A5128093A4120895FC01E5
:10A140004381460F40938A22872F99272281280F27
:10A1500020938922A181A093882250815093872245
:10A1600030E02817390748F48A2F8F5F80938822C0
:10A17000882319F45F5F50938722842F90E07070DA
:10A180008617970798F4809189228F5F80938922A0
:10A19000882361F4809188228F5F809388228823AE
:10A1A00029F4809187228F5F8093872208959C01F4
:10A1B000AB0180E090E0B9010E944F5098278927B9
:10A1C0009827089580E090E06BE872E244E150E067
:10A1D0000E944F50009721F09827892798270895CB
:10A1E0008FEF9FEF089586E00E947550089581E1FA
:10A1F0000E947550089580E0E82FF0E0EE0FFF1FF9
:10A20000EE5EF74D118210828F5F8430A8F380E0FC
:10A21000E82FF0E035E0EE0FFF1F3A95E1F7EE563C
:10A22000F84D118E8F5F843098F380E094E0909326
:10A23000A8128093A71240E08DE090E0242F30E038
:10A24000289FF001299FF00D389FF00D1124E85D43
:10A25000F74D158214824F5F4A3080F34093A61267
:10A260000895CF93DF93EC012091A7123091A812AB
:10A270002F5F3F4F8DE72030380710F020E030E1AE
:10A28000522F432FA0E012C0EA2FF0E0B5E0EE0F0E
:10A29000FF1FBA95E1F7EE56F84D818D882329F01E
:10A2A000848195818417950719F3AF5FA43061F716
:10A2B0003093A8122093A7121092A61280E0E0E03B
:10A2C000F0E01EC0A82FB0E055E0AA0FBB1F5A95C2
:10A2D000E1F7AE56B84D59969C915997992321F4C0
:10A2E0008093A612FD0110C0973049F4309731F0E9
:10A2F0005A962C915A97928D921708F4FD018F5F10
:10A30000843000F38093A612309799F182E0818F18
:10A310008091A91284878091AA1285878091AB12BF
:10A3200086878091AC12878788ED94E0938B828B2F
:10A33000958B848B81E090E0918B808B138E81E0F4
:10A34000828F83E0808F168A80E1878B8091A712AD
:10A350009091A812982789279827958384837783DB
:10A36000668388819981AA81BB8180839183A2833E
:10A37000B383CF01DF91CF9108950F931F93CF93B4
:10A38000DF93EC018B012091A7123091A8126DE0B0
:10A3900070E02F5F3F4F8DE72030380710F020E04E
:10A3A00030E1522F432FA0E011C08A2F90E0869F0A
:10A3B000F001879FF00D969FF00D1124E85DF74D99
:10A3C00084819581AF5F8417950719F3AA3069F7E7
:10A3D0003093A8122093A71240E02DE030E018C07F
:10A3E000542F5F5F842F90E0829FF001839FF00DD8
:10A3F000929FF00D1124E85DF74D848195810097BF
:10A4000031F44093A6129F01309749F424C0452FA0
:10A410004A3030F34093A61220E030E01CC0809117
:10A42000A7129091A812982789279827958384834B
:10A4300017830683209729F41082118212821382D7
:10A4400008C088819981AA81BB8180839183A2837E
:10A45000B38380E48087C901DF91CF911F910F9171
:10A46000089540E013C0E42FF0E0542F5F5FEE0F3B
:10A47000FF1FEE5EF74D208131812817390729F43F
:10A480004093A612118210820895452F443058F34C
:10A490004093A612089540E013C0E42FF0E0542F3B
:10A4A0005F5FEE0FFF1FEE5EF74D208131812115BA
:10A4B000310529F44093A612918380830895452F96
:10A4C000443058F34093A6120895AF92BF92CF92B2
:10A4D000DF92EF92FF920F931F93CF93DF93C09180
:10A4E0009027D0919127843009F4F1C123EB32E217
:10A4F00030938F2720938E273093862220938522B6
:10A50000833071F4898D90E08F7090708330910565
:10A5100009F074C088899989009709F031C78DC006
:10A52000823009F08EC08091AC128F5F8093AC12A4
:10A53000882399F48091AB128F5F8093AB128823AC
:10A5400061F48091AA128F5F8093AA12882329F464
:10A550008091A9128F5F8093A91210928422109289
:10A5600083221092272810922628898D873011F097
:10A57000853041F48A8D8F5F8A8F843109F000C75E
:10A58000198EFEC6882309F4FBC62889398921154E
:10A59000310509F44EC09A8D292F21502A8F992315
:10A5A00009F0EEC69B8D983031F0282F21502230D3
:10A5B00048F4953039F4198E80E880938B270E94F7
:10A5C000BE4C94C5953048F423E030E0092E02C01B
:10A5D000220F331F0A94E2F701C020E32A8F9F5F06
:10A5E0009B8F90E08F70907083309105E1F0843004
:10A5F00091054CF48130910509F469C382309105CD
:10A6000009F0BEC60DC08630910509F47EC58830BC
:10A61000910509F47AC58430910509F0B1C675C574
:10A620001092AC2257C384E080938B270E94BE4CCB
:10A6300092C58F70833009F0A3C688E080938B2782
:10A640004AC5853019F5E0918C27F0918D278481DA
:10A650009581009709F494C6109291271092902743
:10A660002C50304030938F2720938E2730938622B2
:10A670002093852210922728109226281092842257
:10A680001092832288E080938B271FC180918B22B8
:10A69000853409F075C610918D2200E080918E22DC
:10A6A000080F111D809183229091842280179107B9
:10A6B00008F466C61093842200938322809191222D
:10A6C00090E08F739070009709F05AC680919222A3
:10A6D000882309F055C64091222850912328A09044
:10A6E000F705B090F8054A155B0559F480912428C8
:10A6F000909125282091F9053091FA05821793074A
:10A70000A1F080919B2290919C228417950709F0DB
:10A7100037C620919D2230919E22809124289091CD
:10A7200025282817390709F02BC60E94E2502FEF81
:10A730008F3F920709F024C680919422863009F455
:10A740002EC18131D1F1813009F01AC680919F224A
:10A75000883009F015C610929F228091A122909115
:10A76000A2222FEF873F920710F0099601C00896AA
:10A770009093A2228093A122EBE8F2E280919722AB
:10A7800090919822A0919922B0919A2280939B2235
:10A7900090939C22A0939D22B0939E228091222888
:10A7A00090912328A0912428B0912528848795870B
:10A7B000A687B78780E48087C0C50C5110401093EE
:10A7C00084220093832287EA92E290938F278093DA
:10A7D0008E278091A5229091A622009739F00E94A1
:10A7E000F7502FEF8F3F920709F0CAC54091A12281
:10A7F0005091A2224115510509F4C2C588E298E2A0
:10A8000090938D2780938C2760919F227091A02236
:10A81000A091F905B091FA05C091FB05D091FC0516
:10A820000091FD051091FE05E0909722F09098228E
:10A83000C0909922D0909A222EC084819581009751
:10A8400021F14817590709F586819781009719F07A
:10A8500068177907D1F4208131812A153B0529F445
:10A86000828193818A179B07F9F02C173D0729F401
:10A870008281938180179107B9F0E216F30629F4DB
:10A8800082819381C816D90679F0CF010D969093F5
:10A890008D2780938C27E0918C27F0918D2788E27B
:10A8A000EA3AF80750F26CC510929127109290275F
:10A8B00082E080938B2787EA92E2909386228093AE
:10A8C000852210922728109226280E94BE4C809143
:10A8D000262890912728009709F452C59C01245EF0
:10A8E0003F4F309384222093832230938D222093F4
:10A8F0008E22E0918C27F0918D2720852093932242
:10A9000021E12093942208969827892798279093ED
:10A91000A4228093A3221092A6221092A5228481C1
:10A9200095819093A02280939F2286819781909316
:10A93000A2228093A1228091222890912328A09185
:10A940002428B09125288093972290939822A09351
:10A950009922B0939A2280819181A281B3818093C0
:10A960009B2290939C22A0939D22B0939E2283EBE6
:10A9700092E290938F2780938E270E94F7508095C4
:10A9800090959093A6228093A522009709F0D5C4B4
:10A990008FEF9FEF9093A6228093A522CEC40E94B2
:10A9A000F3502FEF8F3F920709F0EAC42091A122C4
:10A9B0003091A2222115310509F4E2C440919F2271
:10A9C0005091A0224115510509F4DAC4E091972273
:10A9D000F0919822A0919922B0919A22C2E9D7E2EF
:10A9E000698D6623A9F08C819D812817390781F430
:10A9F0008E819F814817590759F488819981E817FA
:10AA0000F90731F48A819B81A817B90709F47AC143
:10AA1000A09687E2C23FD80719F310F38091AC22C9
:10AA20008F738230B9F43093AE122093AD1240E0B0
:10AA30000DC0E42FF0E0EE0FFF1FEE5EF74D8081BA
:10AA400091814F5F2817390709F47DC0443088F39E
:10AA50004093A6128091AC2282FD92C484E180933F
:10AA6000AC2288E290E0909384228093832280E558
:10AA70008093AB228091A6229091AA229093A62245
:10AA80003091A5229091A9229093A5223093A922DA
:10AA90002091A4229091A8229093A4222093A822EE
:10AAA0009091A3229093A6124091A7224093A322B3
:10AAB0009093A7228F5F8093AA22882379F4832F13
:10AAC0008F5F8093A922882349F4822F8F5F809320
:10AAD000A822882319F49F5F9093A72280919F2238
:10AAE0009091A0229093AE128093AD122091A1225A
:10AAF0003091A2223093A02220939F229093A222F1
:10AB00008093A1228091972290919822A0919922DE
:10AB1000B0919A2280939B2290939C22A0939D2295
:10AB2000B0939E228091222890912328A0912428DE
:10AB3000B09125288093972290939822A0939922F0
:10AB4000B0939A22DFC31092A61280E0C0E0D0E05A
:10AB500022C0E82FF0E075E0EE0FFF1F7A95E1F7D5
:10AB6000EE56F84D918D992321F48093A612EF01B2
:10AB700016C0973079F4209721F0228D9A8D921784
:10AB800048F4C82FD0E065E0CC0FDD1F6A95E1F7EF
:10AB9000CE56D84D8F5F8430E0F28093A612209776
:10ABA00009F4EEC3D0939127C093902783E08A8F56
:10ABB000888F1E8A84E08F8B1B8E8091A1229091BA
:10ABC000A2229D838C8380919F229091A0229F83BB
:10ABD0008E838091972290919822A0919922B09192
:10ABE0009A2288839983AA83BB8381E0898F80918D
:10ABF000A9128C878091AA128D878091AB128E87C3
:10AC00008091AC128F8781E090E0998B888B809146
:10AC1000A6228B878091A5228A878091A42289878A
:10AC20008091A322888781E090E00E94FC5A809165
:10AC3000AB22282F30E0207F3070213531050CF415
:10AC400046C082958F7090E00597880F991F880FF6
:10AC5000991F3091AF1220E031C0E557FD4D30A56E
:10AC6000332329F42093A6121092AF1230C0313052
:10AC700011F42F5F23C03230E9F441A54430D1F400
:10AC80002093A6123093AF1292A580E023A530E066
:10AC9000282B392B3093AE122093AD12C90124E03A
:10ACA000893D920710F088ED94E09B8B8A8B9D8BF9
:10ACB0008C8B0DC041A5442331F0240FE22FF0E02E
:10ACC000E817F90754F22093A6123093AF1280E1EF
:10ACD0008093AC228091AC2282608093AC2282E08F
:10ACE0008093B32284E08093B4228093B52288EDD0
:10ACF0008093B6228CE290E090938422809383220A
:10AD000080E6ADC2D0939127C093902710928B27F5
:10AD10004091AC2250E042FF03C0198E80E248C24D
:10AD20008091AB2282958F70880F880F8093A61236
:10AD30009801281B310924513040309384222093FC
:10AD40008322862F90E08F7090708230910539F4C5
:10AD5000CA018F7390708231910551F429C08130FE
:10AD6000910531F4CA018F7390708230910501F121
:10AD70002115310529F4CA01837090700097C1F044
:10AD80009091A3228885981709F05FC29091A42220
:10AD90008985981709F059C29091A5228A8598173C
:10ADA00009F053C29091A6228B85981709F04DC2E5
:10ADB00044FF4AC0688979896115710509F444C066
:10ADC000CE010C960E949F503091A722809187223D
:10ADD0003817D1F52091A822809188222817A1F553
:10ADE0009091A92280918922981771F58091AA22C9
:10ADF00040918A22841741F53C872D879E878F8753
:10AE00008B8D8823D1F42E89888D9A8D891B922F62
:10AE1000969596959695891B280F2E8B87FD819583
:10AE20009F89392F36953695931B980F9F8B822FCC
:10AE3000869586958695890F888F81E080938B27EC
:10AE4000888D8A8F198A188A498D50E0CA018F70BF
:10AE500090708430910509F4B0C18530910564F497
:10AE600082309105C9F1833091050CF0B6C0813074
:10AE7000910509F085C211C08630910509F4DDC144
:10AE8000863091050CF4B9C18730910509F4DDC114
:10AE90008830910509F074C285C180918B2780FFAD
:10AEA00014C083E0898F80E480938B27198A188AE5
:10AEB0008091832290918422009709F408C122E4B2
:10AEC00020938B270E94FC5A02C18091AC228F7381
:10AED000823009F055C2FBCE80918B2780FF72C073
:10AEE0008091AC228F73823109F06CC08091AB22CB
:10AEF000282F30E0207F3070213531050CF446C01A
:10AF000082958F7090E00597880F991F880F991F81
:10AF10003091AF1220E031C0E557FD4D30A533230D
:10AF200029F42093A6121092AF1230C0313011F4E0
:10AF30002F5F23C03230E9F441A54430D1F420938F
:10AF4000A6123093AF1292A580E023A530E0282B03
:10AF5000392B3093AE122093AD12C90124E0893D04
:10AF6000920710F088ED94E09B8B8A8B9D8B8C8BE5
:10AF70000DC041A5442331F0240FE22FF0E0E81783
:10AF8000F90754F22093A6123093AF1283E0898F11
:10AF90008091A32288878091A42289878091A5220D
:10AFA0008A878091A6228B8781E090E00E94FC5ADC
:10AFB00082E480938B27198A188A10928422109237
:10AFC000832285C080E280938B270E94BE4CE09153
:10AFD0009027F0919127118E3DCD8091AC2280FF7A
:10AFE00025C044FD23C088899989009709F0C8C10C
:10AFF000809183229091842201960E94FC5A209194
:10B000008B27822F806180938B2780918322909160
:10B010008422009719F0226120938B270E94BE4C56
:10B0200081E090E0998B888B88E06DC085FF1CC023
:10B030009091B12280E02091B22230E0282B392B70
:10B0400080918E2790918F27820F931F90938F2747
:10B0500080938E278091832290918422821B930B70
:10B0600090938422809383228091832290918422E2
:10B07000009749F044FD07C020918B272260209360
:10B080008B270E94FC5A9091AD2280E02091AE2245
:10B09000820F911D9093AE128093AD122C893D8941
:10B0A0002817390710F0009721F43093AE1220933F
:10B0B000AD128091AD129091AE129B8B8A8B8091D4
:10B0C0008B2790E083709070009709F459C110921B
:10B0D0002728109226280E94BE4C20918B2725FFFE
:10B0E00007C01092272810922628198E84E1AEC03E
:10B0F00024FF0DC0109227281092262881E090E0AE
:10B10000998B888B84E0898F1B8E81E19FC0809111
:10B110002628909127280097E9F020FF02C0198A7D
:10B12000188A288939892115310581F42A893B89B2
:10B130002817390720F43093272820932628809158
:10B14000262890912728998B888B04C03093272834
:10B15000209326281B8E80918522909186229093A1
:10B160008F2780938E2780912628909127280097FB
:10B1700059F088899989009739F0889690938422AC
:10B180008093832288E10BC080918B2781FFF8C0D8
:10B1900088E290E0909384228093832280E18093E0
:10B1A000AC225CC080918B2780FFEAC0198E80E1C1
:10B1B00080938B270E94BE4CE3C0809183229091A4
:10B1C0008422009711F00E94FC5A9091AC22809149
:10B1D0008B2790FF0BC080FF06C087E0898F1A8EF7
:10B1E000198A188A19C086E0898F16C080FF1EC090
:10B1F00085E0898F198A188AC3C080918322909133
:10B200008422009711F00E94FC5A8091AC2280FFAA
:10B210000DC087E0898F1A8E81E090E00E94FC5A71
:10B2200080E180938B270E94BE4C0FC080918322C7
:10B2300090918422009749F4A3C080918B2780FFCE
:10B240009FC087E0898F1A8E9BC080E18093AC22DB
:10B2500088E290E0909384228093832280E580931B
:10B26000AB2288858093A72289858093A8228A852E
:10B270008093A9228B858093AA228C858093A32218
:10B280008D858093A4228E858093A5228F858093BF
:10B29000A62286E0809394228C819D819093A022A7
:10B2A00080939F228E819F819093A2228093A122DE
:10B2B0008091222890912328A0912428B0912528BC
:10B2C0008093972290939822A0939922B0939A22E8
:10B2D00088819981AA81BB8180939B2290939C2233
:10B2E000A0939D22B0939E22898D84FF05C0109269
:10B2F000AE221092AD2206C084E08093AD2288ED8C
:10B300008093AE2280E48093932280918322909157
:10B31000842290938D2280938E221092B2221092DA
:10B32000B1221092B0221092AF220E94F350809569
:10B3300090959093B0228093AF2285E480938B22E6
:10B3400010928C2210929222109291228091A4123B
:10B350009091A51201969093A5128093A4129093B8
:10B360008F228093902210929622109295220E9412
:10B37000E25080959095909396228093952204C0F8
:10B38000109284221092832210928B27DF91CF910A
:10B390001F910F91FF90EF90DF90CF90BF90AF90F3
:10B3A000089598278927982708950F931F93DC0104
:10B3B000CB011A2F0B2F20E030E098278927982700
:10B3C000A0E0B0E0DC0199278827082B192B2A2B55
:10B3D0003B2BB801C9011F910F910895FC012091E9
:10B3E0008522309186228BE897E2821B930BAB017A
:10B3F000861797070CF4AC01141615065CF44093FD
:10B40000262850932728E217F30721F0C901BF012E
:10B410000E9407640895CF92DF92EF92FF920F93FC
:10B42000CF93DF93CDB7DEB760970FB6F894DEBF4A
:10B430000FBECDBF002309F45AC029873A874B8736
:10B440005C876D877E878F87988B80E2801B49851C
:10B450005A856B857C851816B4F019821A821B8276
:10B460001C82992787FD9095909581959F4F04C0E8
:10B47000440F551F661F771F8A95D2F74D835E8351
:10B480006F8378872CC06A017B01002E04C0CC0C2E
:10B49000DD1CEE1CFF1C0A94D2F7C982DA82EB8213
:10B4A000FC826A017B0104C0F694E794D794C794A8
:10B4B0008A95D2F7D701C6014D855E856F8578895B
:10B4C00004C0440F551F661F771F0A95D2F7842BBF
:10B4D000952BA62BB72B8D839E83AF83B8872981AD
:10B4E0003A814B815C816D817E818F8198856096E8
:10B4F0000FB6F894DEBF0FBECDBFDF91CF910F9195
:10B50000FF90EF90DF90CF900895A0E1B0E0EBE8DE
:10B51000FAE50C94206129873A874B875C876D8711
:10B520007E878F87988BA982BA82CB82DC82ED825C
:10B53000FE820F8318874D855E856F8578898D81A2
:10B540009E81AF81B885481759076A077B07C8F005
:10B5500084179507A607B70790F049855A856B852C
:10B560007C8589819A81AB81BC81481759076A071C
:10B570007B0738F084179507A607B70720F482E009
:10B5800003C080E001C081E06096EAE00C943C6179
:10B5900080E880936100109261000E94BF350E9494
:10B5A0007B2A0E941E3A809132209091332000978E
:10B5B00029F001979093332080933220C09034205B
:10B5C000D0903520E0903620F09037200E94C3388C
:10B5D000DC01CB01C816D906EA06FB0601F30E947E
:10B5E000C338DC01CB018093342090933520A093A5
:10B5F0003620B0933720D3CFBC0180919027909113
:10B60000912708960E949F50E0919027F0919127F2
:10B6100080918722808780918822818780918922EA
:10B62000828780918A22838708952F923F924F923A
:10B630005F926F927F928F929F92AF92BF92CF92C2
:10B64000DF92EF92FF920F931F93CF93DF93CDB7CB
:10B65000DEB765970FB6F894DEBF0FBECDBF4C01C5
:10B660007F876E87FC0117821682838181FD04C06B
:10B6700076C34C855D8504C01E010894211C311CD5
:10B68000F4019381EE85FF8593FD859193FF819170
:10B69000FF87EE87882309F45EC3853241F493FD6A
:10B6A000859193FF8191FF87EE87853259F490E071
:10B6B000B4014C8B5D8B0E945A644C895D895D8717
:10B6C0004C87D7CFFF24DD2410E01032B0F48B324A
:10B6D00069F08C3228F4803251F0833271F40BC05F
:10B6E0008D3239F0803349F411602CC0126014603F
:10B6F00029C0186027C0106125C017FD2EC0282F53
:10B7000020532A3098F416FF08C08F2D880FF82E8A
:10B71000FF0CFF0CF80EF20E15C08D2D880FD82EE1
:10B72000DD0CDD0CD80ED20E10620CC08E3221F46E
:10B7300016FD11C3106406C08C3611F4106802C0E7
:10B74000883659F4EE85FF8593FD859193FF8191AD
:10B75000FF87EE87882309F0B8CF982F9554933050
:10B7600018F41061805E06C0982F9556933008F04B
:10B77000A2C11F7E16FD02C0E6E0FE2E1F738536B5
:10B7800011F4106406C0863611F4106802C0F1107E
:10B79000FA9417FF07C0FBE3FF1548F0EF2CE39482
:10B7A00027E00DC027E02F1530F02F2D07C027E030
:10B7B0007CE3E72E04C027E067E0F62EEE24CA0102
:10B7C00004969D878C87FA016081718182819381C3
:10B7D000A1010E2D0E9417635C01C9802C2D30E061
:10B7E000398B288BC0FE03C0388933FF06C011FD9A
:10B7F00006C012FF06C000E205C00DE203C00BE266
:10B8000001C000E0888999898C709070009709F4D4
:10B810003CC0002311F084E001C083E08D1558F492
:10B82000D81A13FD09C080E290E0B4010E945A6466
:10B83000DA94C9F701C0DD24002329F0802F90E0BD
:10B84000B4010E945A64888983FD05C033ECE32E5D
:10B850003BE0F32E11C02FEBE22E2BE0F22E0CC0BA
:10B860000115110509F0805290E0B4010E945A645C
:10B870000894E11CF11C04C0012F10E0007110704D
:10B88000F7018491882361F763C217FF0EC0EA0CA9
:10B89000F889F4FF04C08A81813309F4EA941E1404
:10B8A0004CF528E02E1548F12CC016FD2AC08F2D2E
:10B8B00090E08A159B0544F03CEFA3163FEFB306DA
:10B8C0001CF0106801C0FA94FF2049F0E2E0F0E0BB
:10B8D000EC0FFD1FEF0DF11D80818033A1F317FFE9
:10B8E00010C0EF2CE3948F2D90E0A816B90644F415
:10B8F000FA1807C0EE24E39404C098E0E92E01C0D2
:10B90000FF2417FF07C01A141B043CF495012F5F96
:10B910003F4F05C025E030E002C021E030E00023C9
:10B9200011F02F5F3F4FFF2029F08F2D90E00196FF
:10B93000280F391F8D2D90E02817390714F4D21ADB
:10B9400001C0DD24612E7724C301897090700097B7
:10B9500049F406C080E290E0B4010E945A64DA948F
:10B96000DD20C1F7002329F0802F90E0B4010E9470
:10B970005A6463FC09C006C080E390E0B4010E94F1
:10B980005A64DA94DD20C1F717FF48C08501B7FE7D
:10B9900002C000E010E04424552495012E1931091D
:10B9A0003B8B2A8B3501601A710A620C731C6F2D58
:10B9B00070E0EE24FF24E61AF70A3FEF0F3F13076B
:10B9C00029F48EE290E0B4010E945A64A016B106F8
:10B9D00054F02A893B89201731072CF4F301E40D38
:10B9E000F51D818101C080E3015010400894411C85
:10B9F000511C0E151F052CF090E0B4010E945A64F2
:10BA0000DCCF0A151B0541F49A81963320F4953357
:10BA100019F4388934FF81E390E049C08A81813389
:10BA200011F09FEEC92290E0B4010E945A64FF20F9
:10BA300089F08EE290E0B4010E945A6412E0F101B4
:10BA4000E10FF11D1F5F808190E0B4010E945A64F4
:10BA5000FA94A9F764FE03C085E490E002C085E68D
:10BA600090E0B4010E945A64B7FC05C0A114B1046F
:10BA700041F4C4FE06C0B094A194B108B3948DE221
:10BA800001C08BE290E0B4010E945A6480E305C0DB
:10BA90008F5FE6EFFFEFAE0EBF1EFAE0AF16B10408
:10BAA000BCF790E0B4010E945A64C501C096B4018D
:10BAB0000E945A644DC1833631F0833789F0833553
:10BAC00009F059C022C09A012E5F3F4F3D872C8755
:10BAD000FA018081898381E0E82EF12C510113C0A5
:10BAE0009A012E5F3F4F3D872C87FA01A080B180DD
:10BAF00016FF03C06F2D70E002C06FEF7FEFC5012E
:10BB00000E9420647C011F7714C09A012E5F3F4F72
:10BB10003D872C87FA01A080B18016FF03C06F2DEE
:10BB200070E002C06FEF7FEFC5010E94F7637C01F8
:10BB3000106813FD1CC006C080E290E0B4010E94B2
:10BB40005A64DA948D2D90E0E816F906A8F30FC038
:10BB5000F50117FD859117FF81915F0190E0B40118
:10BB60000E945A64D110DA940894E108F108E114B3
:10BB7000F10471F7EDC0843611F0893671F59A0140
:10BB800017FF0AC02C5F3F4F3D872C87FA01808149
:10BB90009181A281B3810BC02E5F3F4F3D872C87DF
:10BBA000FA0180819181AA2797FDA095BA2F012FD4
:10BBB0000F76B7FF08C0B095A095909581959F4FDF
:10BBC000AF4FBF4F0068BC01CD01A1012AE030E0BA
:10BBD0000E946265E82EE21841C0853721F41F7E7D
:10BBE0002AE030E020C0197F8F36A9F0803720F49A
:10BBF000883509F0B0C00BC0803721F0883709F0D4
:10BC0000AAC001C0106114FF09C0146007C014FF6E
:10BC100008C0166006C028E030E005C020E130E032
:10BC200002C020E132E0CA0117FF09C004969D87D7
:10BC30008C87FA01608171818281938108C00296AC
:10BC40009D878C87FA016081718180E090E0A1017D
:10BC50000E946265E82EE218012F0F7706FF09C0E7
:10BC60000E7FEF1430F404FF06C002FD04C00F7E07
:10BC700002C01E2D01C01F2D802F90E004FF0CC0BC
:10BC8000FE01EE0DF11D2081203311F4097E09C063
:10BC900002FF06C01E5F05C086789070009709F00D
:10BCA0001F5FA02EBB2403FD12C000FF0DC0FE2CA1
:10BCB0001D1550F4FD0CF11A1D2D06C080E290E018
:10BCC000B4010E945A641F5F1D15C0F304C01D1506
:10BCD00010F4D11A01C0DD24A4FE0FC080E390E06F
:10BCE000B4010E945A64A2FE1FC0A1FE03C088E5F1
:10BCF00090E010C088E790E00DC0C5018678907094
:10BD0000009791F0A1FC02C080E201C08BE207FD28
:10BD10008DE290E0B4010E945A6406C080E390E096
:10BD2000B4010E945A64FA94EF14C0F3EA94F1014A
:10BD3000EE0DF11D808190E0B4010E945A64EE2066
:10BD4000A9F706C080E290E0B4010E945A64DA9438
:10BD5000DD20C1F78ECCF4018681978102C08FEF80
:10BD60009FEF65960FB6F894DEBF0FBECDBFDF9193
:10BD7000CF911F910F91FF90EF90DF90CF90BF90E8
:10BD8000AF909F908F907F906F905F904F903F907B
:10BD90002F9008955058BB27AA270ED044C135D103
:10BDA00030F03AD120F031F49F3F11F41EF42AC153
:10BDB0000EF4E095E7FB20C1E92F46D180F3BA17D6
:10BDC000620773078407950718F071F49EF55EC14A
:10BDD0000EF4E0950B2EBA2FA02D0B01B9019001A6
:10BDE0000C01CA01A0011124FF27591B99F0593FEA
:10BDF00050F4503E68F11A16F040A22F232F342F32
:10BE00004427585FF3CF469537952795A795F0407F
:10BE10005395C9F77EF41F16BA0B620B730B840B94
:10BE2000BAF09150A1F0FF0FBB1F661F771F881F4C
:10BE3000C2F70EC0BA0F621F731F841F48F48795A4
:10BE400077956795B795F7959E3F08F0B3CF939593
:10BE5000880F08F09927EE0F979587950895A8D039
:10BE600008F481E008950CD0DEC0D6D040F0CDD0EB
:10BE700030F021F45F3F19F0BFC0511108C1C2C0BA
:10BE8000E3D098F39923C9F35523B1F3951B550BD0
:10BE9000BB27AA2762177307840738F09F5F5F4F9D
:10BEA000220F331F441FAA1FA9F333D00E2E3AF0DE
:10BEB000E0E830D091505040E695001CCAF729D0F8
:10BEC000FE2F27D0660F771F881FBB1F2617370747
:10BED0004807AB07B0E809F0BB0B802DBF01FF2777
:10BEE00093585F4F2AF09E3F510568F085C0CFC040
:10BEF0005F3FECF3983EDCF3869577956795B795B1
:10BF0000F7959F5FC9F7880F911D9695879597F9CB
:10BF10000895E1E0660F771F881FBB1F6217730744
:10BF20008407BA0720F0621B730B840BBA0BEE1F59
:10BF300088F7E0950895E89409C097FB3EF4909542
:10BF40008095709561957F4F8F4F9F4F9923A9F0F2
:10BF5000F92F96E9BB279395F69587957795679581
:10BF6000B795F111F8CFFAF4BB0F11F460FF1BC0C5
:10BF70006F5F7F4F8F4F9F4F16C0882311F096E958
:10BF800011C0772321F09EE8872F762F05C0662306
:10BF900071F096E8862F70E060E02AF09A95660FBF
:10BFA000771F881FDAF7880F9695879597F9089578
:10BFB000990F0008550FAA0BE0E8FEEF16161706BA
:10BFC000E807F907C0F012161306E407F50798F022
:10BFD000621B730B840B950B39F40A2661F0232B3B
:10BFE000242B252B21F408950A2609F4A140A695B7
:10BFF0008FEF811D811D089597F99F6780E870E09C
:10C0000060E008959FEF80EC089500240A941616CE
:10C01000170618060906089500240A941216130636
:10C02000140605060895092E0394000C11F48823C4
:10C0300052F0BB0F40F4BF2B11F460FF04C06F5FE0
:10C040007F4F8F4F9F4F089557FD9058440F551FB6
:10C0500059F05F3F71F04795880F97FB991F61F08A
:10C060009F3F79F087950895121613061406551F01
:10C07000F2CF4695F1DF08C0161617061806991F6D
:10C08000F1CF86957105610508940895E894BB2762
:10C0900066277727CB0197F908950BD0C4CFB5DF7A
:10C0A00028F0BADF18F0952309F0A6CFABCF112402
:10C0B000EECFCADFA0F3959FD1F3950F50E0551F47
:10C0C000629FF001729FBB27F00DB11D639FAA27ED
:10C0D000F00DB11DAA1F649F6627B00DA11D661F3C
:10C0E000829F2227B00DA11D621F739FB00DA11D5D
:10C0F000621F839FA00D611D221F749F3327A00D17
:10C10000611D231F849F600D211D822F762F6A2FB2
:10C1100011249F5750408AF0E1F088234AF0EE0F37
:10C12000FF1FBB1F661F771F881F91505040A9F744
:10C130009E3F510570F060CFAACF5F3FECF3983E71
:10C14000DCF3869577956795B795F795E7959F5FAB
:10C15000C1F7FE2B880F911D9695879597F9089545
:10C16000629FD001739FF001829FE00DF11D649FDB
:10C17000E00DF11D929FF00D839FF00D749FF00D67
:10C18000659FF00D9927729FB00DE11DF91F639F08
:10C19000B00DE11DF91FBD01CF0111240895AA1BA7
:10C1A000BB1B51E107C0AA1FBB1FA617B70710F0A2
:10C1B000A61BB70B881F991F5A95A9F780959095D4
:10C1C000BC01CD01089597FB092E07260AD077FD03
:10C1D00004D0E5DF06D000201AF4709561957F4FFA
:10C1E0000895F6F7909581959F4F0895A1E21A2E34
:10C1F000AA1BBB1BFD010DC0AA1FBB1FEE1FFF1F0B
:10C20000A217B307E407F50720F0A21BB30BE40B5A
:10C21000F50B661F771F881F991F1A9469F76095A1
:10C220007095809590959B01AC01BD01CF0108955B
:10C230002F923F924F925F926F927F928F929F9236
:10C24000AF92BF92CF92DF92EF92FF920F931F9324
:10C25000CF93DF93CDB7DEB7CA1BDB0B0FB6F894D5
:10C26000DEBF0FBECDBF09942A88398848885F8415
:10C270006E847D848C849B84AA84B984C884DF8086
:10C28000EE80FD800C811B81AA81B981CE0FD11D6A
:10C290000FB6F894DEBF0FBECDBFED0108958F92AB
:10C2A0009F92AF92BF92CF92DF92EF92FF92CF9385
:10C2B000DF93EC0188819981AA81BB810097A10558
:10C2C000B10521F484E299EDABE5B7E0BC01CD0105
:10C2D0002DE133EF41E050E00E94956749015A019A
:10C2E00027EA31E440E050E00E94B0606B017C013D
:10C2F000C501B4012CEE34EF4FEF5FEF0E94B06048
:10C30000DC01CB01C80ED91EEA1EFB1EF7FE08C0D9
:10C310008FEF9FEFAFEFBFE7C80ED91EEA1EFB1EDF
:10C32000C882D982EA82FB82C6019F77DF91CF91D2
:10C33000FF90EF90DF90CF90BF90AF909F908F9045
:10C3400008950E944F6108958FEF95E00E944F611C
:10C350000895A0E0B0E08093FF0590930006A093BD
:10C360000106B093020608953F924F925F926F923A
:10C370007F928F929F92AF92BF92CF92DF92EF9275
:10C38000FF920F931F93CF93DF9300D000D0CDB7D0
:10C39000DEB72B017A016115710529F0DB018C9361
:10C3A00011969C931197E114F10439F097012250F2
:10C3B00030402332310508F0FCC06C01860108943E
:10C3C000C11CD11CF80130803601832D90E00E9401
:10C3D000EF63009799F7FDE23F1661F4D8011196DB
:10C3E0003C90119792E0692E712C600E711ECC2446
:10C3F000C3940BC0BBE23B1639F4F801318082E0F4
:10C40000682E712C600E711ECC24E114F10421F011
:10C41000F0E1EF16F104F9F480E3381691F4D3015A
:10C420008C91883711F0883561F4F301318082E016
:10C4300090E0680E791E92E0C92AB0E1EB2EF12C53
:10C440000AC0E114F10439F4A0E33A16D1F0AAE0ED
:10C45000EA2EF12C30C0BAE0EB16F10461F1E0E114
:10C46000EE16F10429F0F8E0EF16F104B1F409C07A
:10C47000FFEF8F2EFFEF9F2EFFEFAF2EFFE0BF2EBF
:10C4800022C078E0E72EF12CEFEF8E2EEFEF9E2EFC
:10C49000EFEFAE2EEFE1BE2E16C09701442737FD19
:10C4A0004095542F6FEF7FEF8FEF9FEF0E94F66064
:10C4B00049015A0108C069E9862E69E9962E69E9A1
:10C4C000A62E69E1B62E40E000E010E020E030E06A
:10C4D000C701AA2797FDA095BA2F89839A83AB83BA
:10C4E000BC8350EDD52ED30C99E09D1570F4832DAF
:10C4F00081548A3118F499ECD92E06C0832D8156C7
:10C500008A3168F589EAD82ED30C8D2D90E08E15EE
:10C510009F052CF54F3FF9F080169106A206B30651
:10C52000B8F0C901B80129813A814B815C810E9430
:10C53000B0608B019C018D2D90E0A0E0B0E0080F71
:10C54000191F2A1F3B1F081719072A073B0710F45A
:10C550004FEF01C041E0D3013D903D01C2CF4114F6
:10C56000510489F0442339F0089461087108F201FC
:10C570007182608208C0C1FE06C0C3010297D20169
:10C5800011969C938E93C0FE07C030952095109510
:10C5900001951F4F2F4F3F4F47FF0FC082E290E0A2
:10C5A0009093B1288093B0280FEF1FEF2FEF3FEF4C
:10C5B00004C000E010E020E030E0B801C9010F90B5
:10C5C0000F900F900F90DF91CF911F910F91FF90DF
:10C5D000EF90DF90CF90BF90AF909F908F907F9023
:10C5E0006F905F904F903F900895662777270C9447
:10C5F000FB65FC0188279927E89421912032E9F313
:10C60000293010F02E30C8F32B3241F02D3239F49E
:10C61000689404C00E945264820F911D219120539E
:10C620002A30C0F31EF4909581959F4F08952830CD
:10C6300008F027E03327DA01990F311D87FD91605B
:10C6400000966105710539F432602E5F3D9330E349
:10C650002A95E1F708959F3F30F080387105610514
:10C6600009F03C5F3C5F3D93913008F08068911D7C
:10C67000DF93CF931F930F93FF92EF92192F987F21
:10C680009695E92F96959695E90FFF27EF5DF34F65
:10C6900099273327EE24FF24A701E701059008948A
:10C6A000079428F4360FE71EF81E491F511D660F28
:10C6B000771F881F991F0694A1F70590079428F407
:10C6C000E70EF81E491F561FC11D770F881F991FBF
:10C6D000661F0694A1F70590079428F4F80E491FE9
:10C6E000561FC71FD11D880F991F661F771F0694FD
:10C6F000A1F70590079420F4490F561FC71FD81FB4
:10C70000990F661F771F881F0694A9F784911095CB
:10C71000177041F0D695C79557954795F794E794CC
:10C720001A95C1F7E7ECFBE06894159015913591E7
:10C730006591959105907FE27395E118F10A430B9D
:10C74000560BC90BD009C0F7E10CF11E431F561F51
:10C75000C91FD01D7EF4703311F48A95E6CFE8949A
:10C76000015030F0080F0AF40027021708F4202FB8
:10C770002395022F7A3328F079E37D932A95E9F700
:10C7800010C07D932A9589F60694979567953795FD
:10C7900017951794E118F10A430B560BC90BD009F2
:10C7A00098F023957E9173957A3308F070E37C932B
:10C7B0002013B8F77E9170617D9330F0839571E31B
:10C7C0007D9370E32A95E1F71124EF90FF900F918C
:10C7D0001F91CF91DF91992787FD90950895911131
:10C7E00089C3803219F089508550D0F70895FC0133
:10C7F0000590615070400110D8F7809590958E0F8C
:10C800009F1F089540EB52E10E942B640895FB01A5
:10C81000DC0102C001900D9241505040D8F70895BC
:10C82000DC0101C06D9341505040E0F70895FB01D9
:10C83000DC018D91019080190110D9F3990B0895B5
:10C84000FC016150704001900110D8F780959095DF
:10C850008E0F9F1F0895FA01A191B081009719F4DE
:10C860001097E1F0CD01DC01CD010D90002011F415
:10C87000C00113C0FB012191222319F02015D9F723
:10C88000F3CFFB012191201519F41E92119606C0D9
:10C890002223C1F70D900020A1F7D001FA01A19346
:10C8A000B08308957AE0979F902D879F802D910DFA
:10C8B000112408950F931F93CF93DF938C01EB0105
:10C8C0008B8181FF1BC082FF0DC02E813F818C8137
:10C8D0009D812817390764F4E881F9810193F98370
:10C8E000E88306C0E885F985802F0995009731F423
:10C8F0008E819F8101969F838E8302C00FEF1FEF71
:10C90000C801DF91CF911F910F910895CF93DF93CD
:10C91000CDB7DEB7FE013596619171918091AC285B
:10C920009091AD28AF010E94155BDF91CF910895E2
:10C93000CF93DF93CDB7DEB7FE013596619171914C
:10C940008091AC289091AD28DC0113962C9113971F
:10C95000286013962C93AF010E94155BE091AC28E0
:10C96000F091AD282381277F2383DF91CF91089514
:10C970006091AC287091AD280E945A6408950F937D
:10C980001F93CF93DF938C01E091AC28F091AD28F9
:10C99000838181FF1AC0C0E0D0E005C009950097EF
:10C9A00011F0CFEFDFEFF80181918F016091AC289A
:10C9B0007091AD28DB011896ED91FC9119978823B1
:10C9C00069F78AE00995009711F0CFEFDFEFCE010C
:10C9D000DF91CF911F910F9108950F931F93CF93E4
:10C9E000DF93CDB7DEB72E970FB6F894DEBF0FBE3C
:10C9F000CDBF0D891E898F89988D26E02C831A83DF
:10CA0000098397FF02C080E090E801979E838D83A1
:10CA1000AE01455E5F4FCE010196698D7A8D0E9411
:10CA2000155B4D815E8157FD0AC02F813885421705
:10CA300053070CF49A01020F131FF80110822E966F
:10CA40000FB6F894DEBF0FBECDBFDF91CF911F911F
:10CA50000F9108950F931F93CF93DF93CDB7DEB758
:10CA60002E970FB6F894DEBF0FBECDBF8C0186E0C7
:10CA70008C831A83098377FF02C060E070E86150FD
:10CA800070407E836D83CE010196BA01A9010E9498
:10CA9000155B4D815E8157FD0AC02F813885421795
:10CAA00053070CF49A01020F131FF80110822E96FF
:10CAB0000FB6F894DEBF0FBECDBFDF91CF911F91AF
:10CAC0000F910895FA01AA27283051F1203181F100
:10CAD000E8946F936E7F6E5F7F4F8F4F9F4FAF4F86
:10CAE000B1E03ED0B4E03CD0670F781F891F9A1F99
:10CAF000A11D680F791F8A1F911DA11D6A0F711D4D
:10CB0000811D911DA11D20D009F468943F912AE058
:10CB1000269F11243019305D3193DEF6CF01089540
:10CB2000462F4770405D4193B3E00FD0C9F7F6CF71
:10CB3000462F4F70405D4A3318F0495D31FD405239
:10CB4000419302D0A9F7EACFB4E0A69597958795CF
:10CB500077956795BA95C9F70097610571050895AE
:10CB60009B01AC010A2E069457954795379527955A
:10CB7000BA95C9F7620F731F841F951FA01D0895F2
:10CB8000DC01CB01FC01F999FECF06C0F2BDE1BD8D
:10CB9000F89A319600B40D9241505040B8F708957C
:10CBA000F999FECF92BD81BDF89A992780B5089575
:10CBB000A8E1B0E042E050E00C94C265DC01CB019A
:10CBC00003C02D910E94E96541505040D0F708956F
:10CBD000262FF999FECF1FBA92BD81BD20BD0FB699
:10CBE000F894FA9AF99A0FBE019608950E94E865A2
:10CBF000272F0C94E9656F927F928F929F92AF924C
:10CC0000BF92CF92DF92EF92FF920F931F93CF9339
:10CC1000DF935B016115710521F0DB018C931196A7
:10CC20009C937C01E7010894E11CF11C08816701D9
:10CC3000802F90E00E94EF630097A1F70D3241F43E
:10CC4000098142E0C42ED12CCC0EDD1E11E009C0BA
:10CC50000B3231F4098132E0C32ED12CCC0EDD1E13
:10CC600010E0E6012197CE0161EC7CE043E050E06A
:10CC70000E947D670097D1F4E6012296CE0164EC14
:10CC80007CE045E050E00E947D67009711F4E601EA
:10CC90002796A114B10419F0F501D183C08330E0C7
:10CCA00020E090E8112309F40DC107C1CE0169EC21
:10CCB0007CE043E050E00E947D67009759F4A114A6
:10CCC000B10409F4FCC0C6010296D50111969C93EB
:10CCD0008E93F5C040E050E060E070E08824992435
:10CCE00000530A3090F51260212F30E0C90188709E
:10CCF000907012FF06C0009769F50894811C911C82
:10CD000029C0009719F0089481089108DB01CA0135
:10CD1000D2E0880F991FAA1FBB1FDA95D1F7480FE1
:10CD2000591F6A1F7B1F440F551F661F771F400F37
:10CD3000511D611D711D4839B9E95B07B9E96B07E0
:10CD4000B9E17B0738F0146005C00E3F39F413FDDC
:10CD500043C01860F60101916F01C2CF053311F095
:10CD60000531D1F5D601EC91ED3211F4106108C016
:10CD7000EB3229F0C601019621E030E008C0D6016F
:10CD80001196EC911197C601029622E030E0E05333
:10CD9000EA3020F06C01C21AD30A1EC0DC0120E088
:10CDA00030E0FCE020383F075CF4C901880F991F90
:10CDB000880F991F280F391F220F331F2E0F311D87
:10CDC000ED91E0536D01EA3060F314FF03C030953C
:10CDD00021953F4F820E931EC12FD0E011FF08C056
:10CDE000A114B10429F0C6010197D5018D939C933C
:10CDF000CB01BA010E949B5F6B017C01CE01837065
:10CE000090708330910521F4F7FAF094F7F8F094DC
:10CE1000C701B60120E030E040E050E00E942F5F03
:10CE2000882309F445C097FE07C090948194910827
:10CE30009394C8EFDCE002C0C0EEDCE098EE692E0F
:10CE40009FEF792E6C0E7D1E20E2A22EB12C0FC01A
:10CE5000FE010591159125913491C701B601A901F3
:10CE600098010E944D606B017C018A189B088A140E
:10CE70009B0474F72497B594A794C615D705B9F702
:10CE8000C601D7012A2F220F2B2F221F2F3F51F02F
:10CE9000BC01CD0120E030E040E050E00E942F5F77
:10CEA000882331F482E290E09093B1288093B028F7
:10CEB0003C2D2D2D9E2D8F2D06C08FEF04C030E010
:10CEC00020E090EC8FE7B901AC01872F922FA52FBE
:10CED000B42FBC01CD01DF91CF911F910F91FF9035
:10CEE000EF90DF90CF90BF90AF909F908F907F900A
:10CEF0006F900895992788270895FB01DC01415020
:10CF0000504088F08D9181341CF08B350CF4805E9C
:10CF1000659161341CF06B350CF4605E861B611109
:10CF200071F3990B0895881BFCCF97FB092E0526FA
:10CF30000ED057FD04D05AD90AD0001C38F45095B1
:10CF40004095309521953F4F4F4F5F4F0895F6F72D
:10CF500090958095709561957F4F8F4F9F4F089565
:04CF6000F894FFCF73
:10CF6400263A202573205B414444523D252D642EEE
:10CF7400252D64205345513D252D6420525353499A
:10CF84003D252D75204C51493D252D752044525089
:10CF94003D252D642E253032645D0A005363686597
:10CFA40064756C6564206576656E74206174203DDB
:10CFB400256C642066756E633D25780D0A00536305
:10CFC400686564756C6564206576656E74206E6F43
:10CFD400773D256C64206E6578743D256C640D0A7C
:10CFE4000028457874507772290000737461747551
:10CFF400733D3078253032780A2000312E302046B7
:10D0040069726D77617265205665722E20322E38F2
:10D0140020323031322D30382D3235006565707252
:10D024006F6D006F6E006F6666004F6E00613100B9
:10D03400726573657400613200765F696E006175B4
:10D04400746F00666C75736800414444523D252D2D
:10D05400642E252D64205345513D252D64205253C3
:10D0640053493D252D75204C51493D252D750A0008
:10D074007472696D0043683D252D6420547850779F
:10D08400723D252D640A004572726F722054582037
:10D094004C656E6774683D25640A0049443D00256B
:10D0A400303278002050533D25640020543D252D16
:10D0B400362E3266002054313D252D362E32660040
:10D0C40020545F4D43553D252D352E3166002056A5
:10D0D4005F4D43553D252D342E3266002050303DA2
:10D0E400252D6C58002050305F543D252D372E33AC
:10D0F40066002050313D252D6C58002055503D25AB
:10D104002D6C58002052483D252D342E31660020C8
:10D11400565F494E3D252D352E32660020565F411F
:10D12400313D252D352E32660020565F41323D2596
:10D134002D352E326600263A2025730A006C656E62
:10D14400203D2025640A0025303258006C656E3D70
:10D1540025640A006E04580442042A040E040000E4
:10D16400536C6565702070726F63657373000000A3
:10D1740000048F0E0000000062726F6164636173CB
:10D18400742070726F636573730000001804702359
:10D1940000000000737464696E2070726F636573BD
:10D1A400730000003404A70D00000000666F6F20B8
:10D1B40070726F636573730000004C0464080000B0
:10D1C4000000636D642070726F6365737300000008
:10D1D4006204B3220000000002003C008F0261627E
:10D1E400636465666768696A6B6C6D6E6F7020094D
:10D1F4000D008E041A22FFCC3B22FFCC3BED478A64
:10D204003C01001000BA0600000D0040003A067A06
:10D21400060000E628DA28181000000000457665AC
:10D224006E742074696D6572000000BD04CE2C001C
:10D23400000000020306070A0B0E0F436F6E7469A9
:10D244006B6920322E3500C600C500C400C100C27F
:10D2540000000000CE00CD00CC00C900CA000000D0
:10D264000000000002000000008E3900000000529F
:10D2740046323330206472697665720000000F050F
:10D284003E3E000000009B3CD83B8D3ECF3F2E3DF0
:10D29400313C3C3A363A263B173C0001010101017E
:10D2A400010101010101010101010052696D6500E3
:10D2B4004B0540410B4161646174612E6E756D20B4
:10D2C400776179206F75742074686572653A2025DA
:10D2D400640A00794278428244A645D8430080C05B
:10D2E400E0F0F8FCFEFF6E756C6C6D616300860502
:10D2F400524637463D46434649464F467369637333
:10D304006C6F776D6163009C056347C7465C465349
:10D31400466D4759464374696D65722070726F6338
:10D32400657373000000B505E24700000000BA0011
:10D334000800390C410C3500020011121312544339
:10D34400502F495020737461636B000000DE05DECA
:10D354004A00000000020800000000FFFFFFFF0178
:04D3640000000000C5
:00000001FF
